:020000040800F2
:1000000000500020251C0108C11C0108C11C01086A
:10001000C11C0108C11C0108C11C0108000000002E
:10002000000000000000000000000000C11C0108EA
:10003000C11C010800000000C11C0108ED8C000873
:10004000C11C0108C11C0108C11C0108C11C010818
:10005000C11C0108C11C0108C11C0108C11C010808
:10006000C11C0108FD8C0008C11C0108C11C01084D
:10007000C11C0108C11C0108C16E0008C11C010897
:10008000C11C0108C11C0108C11C0108C11C0108D8
:10009000C11C0108C11C0108C11C0108C11C0108C8
:1000A000C11C0108C11C0108C11C0108C11C0108B8
:1000B000C11C0108C11C0108C11C0108B71D0008B2
:1000C000BB1D0008B51D0008B91D0008C11C0108B2
:1000D000C11C0108B96E0008B16E0008C11C0108FE
:1000E000018D0008C11C0108C11C010800000000AE
:1000F0000000000000000000000000000000000000
:0C01000000000000000000005FF808F1A3
:100110002DE9F04FA3B003F02BFC18B903F05CFEFF
:1001200003F04CFCB34D03F0EDFC2B78B24C43F0E4
:1001300001032B70002309930A930B934FF4E013F0
:100140000C932368AD4F43F48033B87B2360A369DD
:1001500043F01003A361236803F400330A93099B5F
:10016000013309930A9B1BB9099BB3F5A06FF2D128
:10017000236813F4003300F0548302230B93A04B45
:10018000A0491A6842F010021A601A6822F00302AD
:100190001A601A6842F002021A606368636063685A
:1001A0006360636843F480636360974B1A68043B41
:1001B00022F070425A60954A1160616821F47C1106
:1001C0006160596841F000415960D96821F40041EB
:1001D000D9604FF4E0110C910B999846012900F079
:1001E000408302290ED138B10C9BB3F5801F40F03B
:1001F00030834FF4A0130C930C9B61680B4343F4C2
:1002000080336360236843F08073236023689E011A
:10021000FCD5636823F003036360636843F0020363
:100220006360636803F00C03082BFAD16368784EAF
:1002300003F00C03042B00F01883082B00F0178345
:10024000704B33606368734AC3F30313D25C336843
:100250004FF00009D34033600B9B6F4A6B60D8F8B6
:1002600008306E4BDFF8D4A1DA60A269049342F043
:100270000102A261626A22ABAA60626A504642F041
:1002800080726262A2690DF1880B42F01C02A261C9
:100290004FF6FF7223F8402D194603938DF84A90CC
:1002A00006F0ECFA03995E4806F0E8FA03995D4817
:1002B00006F0E4FA02228DF837204FF400724FF076
:1002C00010032BF8542D8DF836305046CAF8102004
:1002D000594606F0D3FA544903984A6842F000722E
:1002E0004A6007F011FA129A5049049BB2FBF1F2EE
:1002F0004F49DFF84CC10A604FF47A714D4AC2F899
:100300000090C2F804903268B2FBF1F24A49013A17
:100310004A60F02283F823200723C1F808900B607D
:10032000BB68039ECCF800303A4B03F1100EBEE8D8
:100330000F000FC6BEE80F000FC6BEE80F000FC6C5
:100340009EE80F0086E80F00A369402243F01003E7
:10035000A361A36943F01003A361A36943F01003F1
:10036000A361A36943F00803A361A36943F00803F1
:10037000A361A36943F00403A3611023CAF81430F6
:100380002023CAF81430CAF814204FF48042C8F869
:1003900010204FF40052C8F810204FF40042C8F863
:1003A00010201F4A5361134610225A61CDF810A045
:1003B000E246AEF140030593039B09F1040153F8B3
:1003C0000900194409F1080906F058FAB9F1400F7B
:1003D000F2D1DAF800301B0734D597F82431012B1D
:1003E00030D8AA6897F8253112F0805901F0AD8015
:1003F00028E000BF6C0D002000100240A00F00207C
:100400000020024000127A00041001404000002049
:100410000C000020DCA701080005FA0500ED00E053
:10042000000C0140001001400000014040420F005C
:10043000E42000208820002010E000E000080140B7
:10044000D01400204FF400536420C8F8143008F092
:10045000EAFB4FF48043A022C8F814300021C448BE
:1004600015F08CFCE369C34A43F00703E361A36919
:10047000DFF83C8343F4006343F00C03A361BE4BFD
:1004800000211A600222BD4B40461A701822DAF889
:10049000006015F073FC0021012388F8001088F833
:1004A0000C3097F805801422584615F067FCB8F117
:1004B0000E0FC6F3801904D008F0EF08B8F1080F4A
:1004C00002D101238DF83E3097F97E31012B01F0E6
:1004D0005F8097F98631012B01F05B8000238DF856
:1004E0003930C6F340038DF83A30C6F340338DF807
:1004F0003430C6F3C0338DF8373016F400638DF80E
:100500003C9007D097F81831A3F1020EDEF10003FA
:1005100043EB0E038DF83830C6F30043B7F8D40030
:100520008DF83D30C6F3C00306F0010106F0080265
:100530008DF83630C6F38043F604ADF842008DF8EE
:100540003B3048BFB7F8DC00B7F8E03048BFADF843
:100550004200B3F5FA7FADF84030C4BF0023ADF8D8
:10056000423097F868318DF835102B730023A5F8C9
:100570000D309DF83E30002B14BF0223002301B93B
:1005800002B101334FF0000B059A02EB83031B6DA0
:100590009A1E1A3306920793069A32F8023F069281
:1005A0004FF6FF72934240F0928104220026744B72
:1005B000DFF800C2DFF800E21A7006EB0C0706EB6A
:1005C0000E031036402E0FCB87E80F00F5D16D4B90
:1005D0006D4FD3F800E06D4B3A681E6800236C48FD
:1005E00002F4805CBCF1000F00F05382B6F90410F5
:1005F00020F8131001330C2BF4D150035CBF0122FF
:10060000644B4FF0000058BF1A702B7843F004037E
:100610002B7001F003FA3D68102205F0020500215D
:100620005D4815F0ABFBDDB1049B01201A680F2576
:10063000002300FA03F131F0080104BF990005FA24
:1006400001F103F1010308BF8A43082BF1D1049B98
:1006500001251A600322504B1A7007229D70DA7030
:1006600063684E4E43F4404363606369304643F031
:1006700001036361A36943F40073A36106F0CAFF39
:10068000474B00241293474B304613934FF480732B
:1006900018934FF48063199320231A934FF4005357
:1006A000039915951B93149416941C94179406F0B3
:1006B00093FF33683C4943F0010333604B68013DCD
:1006C00023F4702323F480734B608A68374BEDB2B8
:1006D000134043F4602343F002038B60CB6A20464F
:1006E00023F4700343EA0555CD6201231F254FF023
:1006F000070E294E821994784CB310F806805C1CC2
:10070000B8F1090FE4B292F803C040F2C581A8F134
:100710000A02D1F80C9002EB42020EFA02FA29EA20
:100720000A090CFA02F242EA0902CA60062B00F238
:10073000E58103F1FF3C4A6B0CEB8C0C05FA0CF3E2
:1007400022EA030308FA0CF21A434A6323460430F0
:100750001028CFD1144B9A6842F480729A609A683C
:1007600042F001029A609A6842F008029A6025E01D
:10077000202100201C110020C41D00206C0F00202F
:100780001C2100206C0C0020D0140020680C0020DC
:10079000A81D0020640D00208B1F002008000240CF
:1007A0004C2401409C1F002000240140FDF7F1FF74
:1007B000700F0020A00C00201CA901089A681107E6
:1007C000FCD49A6842F004029A60BA4B9A685207C5
:1007D000FCD4B94D9A68B5F9E80042F4A0029A60D9
:1007E000002800F0A8810022B44B1A7010F01AFF04
:1007F000B34910F06BFF1290B5F9EA0010F012FF48
:10080000AF4910F063FF1390B5F9EC0010F00AFF48
:10081000AB4910F05BFFAB491490039802F06EFFF8
:1008200093E1226842F0010222600993236803F0F9
:1008300002030A93099B013309930A9B1BB9099B85
:10084000B3F5A06FF2D123689B0701D5012395E48E
:10085000FEE70C9BB3F5E01F7FF4CEAC4FF4001322
:10086000C9E4636843F46013CBE41368E9E46368A4
:100870006168C3F38343C80303F1020302D4924ABD
:100880005343DEE461681268890348BF5208F7E702
:100890000693049BC8F8109078205E6108F0B8F9C0
:1008A000049BC8F8149078201E6108F0B1F9069BEB
:1008B000013397F825219342EADBAB6813F08053AC
:1008C0007FF4C0AD87F8253103F07CFABAE5DAB2DF
:1008D0007E4916018F199DF839101B0A11B1023A91
:1008E000012A12D99DF83A204AB1059A0498324457
:1008F000516E814203D1B2F86820082A05D0022B3C
:1009000009D19DF83430002B4CD1079B069A9342B5
:100910007FF442AE49E6012B41D19DF83530002BE2
:10092000F3D0FF2385F8543085F85530059B4FF000
:1009300000081E4496F86D30B6F868208DF84A30ED
:1009400002230399706E85F858806F668DF84B30DE
:10095000ADF8482085F81080C5F81480C5F81880D7
:10096000C5F81C80C5F8508085F8568085F85780FA
:1009700005F084FF424696F86A10306E05F054FE8A
:10098000384602F00DF8524B524AAB66524BC5F84E
:100990007080EB66111F384606F036FAB5E7022B79
:1009A000DAB243D14FF01C0901235FFA8BF109FB46
:1009B00001F905EB090888F85830059B4FF0000A4B
:1009C0001E4496F86D30B6F868208DF84A30022340
:1009D00088F859B00399706E88F85AA088F862A018
:1009E000C8F864708DF84B30ADF8482005F046FF2C
:1009F000524696F86A10306E05F016FE384601F041
:100A0000CFFF364B3649C8F86830364B09F114022F
:100A100009F110090A44C8F86C30C8F870A04944BC
:100A2000384606F0F1F90BF1010B6EE7032A7FF46B
:100A30006CAF9DF83B302C4E63B100234FF6FF7234
:100A4000082195F80E80384605F053FF274B46F8ED
:100A5000280013E0BDF8401095F80E80B1F5FA7F3C
:100A6000BDF842300FDD224A3846B2FBF1F20821D0
:100A700092B205F03EFF1F4B46F82800C360AB7BE7
:100A80000133AB7341E71C4AB2FBF1F2012192B290
:100A9000D9E7BEF90410ABE50A6908EB480A0EFA7B
:100AA0000AF922EA09090CFA0AF242EA09020A6181
:100AB0003CE600BF00240140A00F002044000020BD
:100AC00035FA8E3C681D002000093D003CA8010855
:100AD00079620008D80D00205163000825680008DD
:100AE000C40D002051620008EC2000206163000862
:100AF00000127A007163000840420F000C2B0DD8E1
:100B0000DA1FD1F830C002EB820205FA02F32CEAB8
:100B1000030308FA02F21A430A6317E60D3BCA6A96
:100B200003EB830305FA03FC22EA0C0208FA03F341
:100B30001343CB620AE6B5F9EA30002B7FF453AEDB
:100B4000B5F9EC30002B7FF44EAE4FF0000BC44EE5
:100B5000C44C10225946C6F800B0C6F804B0C6F816
:100B600008B0C14884F838B1B5F8F0A095F8EF9016
:100B700095F8F78015F002F92320A4F839B1C4F8EC
:100B80003CB1C4F840B1C4F844B1C4F848B108F06D
:100B90004AF80DF121020121752001F0C5F800B3DA
:100BA000B24B0DF12202C4F84031B14B0121C4F81F
:100BB00044314323584684F83C3101F0B5F89DF8A0
:100BC000223003F07E038DF82230002800F0FC80F4
:100BD000682B40F0F980012384F839311D2384F813
:100BE0003C31002094F83921A24B042A1870039359
:100BF00040F0D8849C49A04B40F2FD1C0B609F4BF9
:100C000004914B609E4BCB609E4B1A689B4642F012
:100C1000010EC3F800E04FF0010E4B460A2B28BF2F
:100C2000002340F202290EFA03F111EA090940F00B
:100C3000C18411EA0C0F00F0BD84934B42F0030213
:100C400083F80090914BCBF800203360904B736099
:100C5000DBF800309B0701D5336898474FF0000957
:100C6000049B50461B689847CA468A4E86F800A0E7
:100C7000B8F1000F04D0A8F10203022B00F2E980C2
:100C800022AB03F8409D012200210C2001F014F852
:100C9000002800F0DE809DF84830482B40F0D980D5
:100CA0007D4B7E4A1A607E4A5A6006233370DBF819
:100CB000003043F00803CBF8003095F8E4300BB176
:100CC000039A137095F8E5300BB16F4A137095F8DD
:100CD000E63003B1337095F8F830042B00F2E6806B
:100CE0004FF0010909FA03F212F0160865D112F06B
:100CF000090F00F0D9800A2007F095FF0DF12303BA
:100D00004A46A021772000F0D7FF0646002854D09D
:100D10004A461E21772001F00CF84FF42F6007F0AF
:100D200077FFC146DFF87CA1A8F1600112AB022277
:100D3000C9B277208DF848908DF8499000F0BCFF3B
:100D40009DF848209DF8493043EA022328F80A30EC
:100D500008F10208B8F1100FE6D100231946B4F8E3
:100D60005A2102F00F0E02F47F42A4F85A2121F01A
:100D700001002044B0F84C01002818BF002611F0F3
:100D8000010F1ABFC0B2434083EA1023082013F4B6
:100D9000004F18BF83F4C05301384FEA4303F6D124
:100DA00001311029E3D142EA0E02A4F85A2126B9F2
:100DB000C3F303339E4500F0068494F8383143F0C2
:100DC000200384F8383176E09DF8213003F07E036B
:100DD000682B8DF8213036D10223062184F8393171
:100DE000039AD4F84031084698479DF84D309DF855
:100DF0004B209B00520002F0020203F00403134355
:100E00009DF8492002F001021343DAB263B1012ACE
:100E100003D1002384F83A31E3E6022A01D1012309
:100E2000F8E7022007F009FFD4F840310DF1230262
:100E300001210C2098479DF8233013F00F03F0D0C8
:100E4000042BECD1E5E7702B04BF042384F839317F
:100E5000C7E6B8F1010F7FF630AF4FF0000805E7A5
:100E6000780B00206C0D0020F4150020291D0008CF
:100E7000AD1D0008200B0020751900088D18000812
:100E800090C1793D74150020840B00206119000881
:100E9000D1180008180B0020100B0020396400083E
:100EA00095630008B80E0020012B86D08C4A136889
:100EB00043F0040313606368012B02BF94F83831D8
:100EC00043F0400384F8383194F838610EB130466D
:100ED000A8E723784FF0100843F0020323704FF483
:100EE0000053804C63614FF480432361B8F10108E3
:100EF00012D0E368192083F40053E360E36883F4BD
:100F00008043E360E36883F40043E36007F08BFE13
:100F1000192007F088FEE9E74FF480434FF40058AA
:100F200023614FF40043C4F8108023616C4B1A68AE
:100F3000994612F0080F09D06B4BC4F814801B6857
:100F400098470122694BC4F810801A70684B694CAD
:100F50001B68187B10F066FB674910F0B7FB674908
:100F600010F0ACFA02F055FB8046208810F05AFBD6
:100F7000414610F0ABFB18F097FD614B18802088BC
:100F800010F050FB01465F4810F054FC5E4910F031
:100F90009DFB5E4B584918605D4B5E4CD86810F065
:100FA00095FB5D4910F092FB5C4B1B221860FF2102
:100FB000204614F0E3FE002201212270D9F800201F
:100FC000574B12F0020F1970204604D061700321B4
:100FD00019700221A170510704D519784C1C1C709E
:100FE0000324445412F00A0F40F003833C68A20625
:100FF00004D51A78511C1970072181546A79082A7E
:1010000001D00E2A04D11A78511C19700B21815479
:101010000C271A788754511C670748BF0232C9B29F
:10102000197044BF1A7010224FF0120748BF425483
:101030001A78511CC9B287546705197004D595F800
:101040009071002F40F0E382A70504D51A78511C57
:10105000197015218154E10504D51A78511C1970B5
:101060001A238354982200212E4814F087FE012071
:1010700007F0E4FC4FF04C0ADFF8A880DFF8A8B0D6
:10108000002853D0012E51DC0AFB06F908EB0907B2
:1010900097F84A4014B10136F6B2F1E7032203791A
:1010A00001210BEB830390F90000D3F8803100920B
:1010B0000194224607F066FC039060B14C22214661
:1010C000384614F05BFE039B48F8093001231E44A8
:1010D00087F84A30F6B2012007F090FCD0E700BF55
:1010E0007415002000100140100B0020181500207E
:1010F0008C1700204800002035FA8E3CDB0FC93FDA
:10110000A81700200AE81C410000C842A8160020C9
:10111000F4150020150F0020BD37863588170020F4
:10112000140F0020D00B0020DCA70108AF4AB04B01
:10113000B04C1A600023A646AF49B0480B808B70B4
:10114000AF4902600E68AF4AB5F82A01DFF8408364
:10115000AD4F06F1790113700FFA80FCD8F800202A
:1011600024F813C002F5167247F823200133122B1E
:10117000F4D1A64CC9362768FA0458BFB5F930C176
:10118000AEF806C00B7883B98A78CB789A420CD235
:10119000EAB1013A02EB820202EB820202F56173CC
:1011A0004A789BB204322EF812300431B142E9D1B0
:1011B0003B0721D595F82461062E17D8DFE816F0F5
:1011C0000F0078007B00A600C000DA00DA000133CF
:1011D00003EB830303EB830303F56173E0E745F25D
:1011E000F0528B4B1A8001F04DFC28B9082002F018
:1011F00089FB884A884B1A602368884A13F4804F19
:1012000004D01221864811708349086042F2010619
:10121000334203F0010103F400500FD044F620667E
:101220007B4B1E8020B108237E4813707A4B1860D8
:1012300021B10C237C491370774B196013787B4ED6
:10124000043B537007F0C8FC794BDFF848921860F4
:101250006B79784D052B04BF4FF4C872764BDFF8DD
:10126000388208BF1A80754A754B1A60754A764BEA
:101270001A60764A764B1A604FF47A72754B1A8070
:1012800000232B6033602B68002B40F00D81232757
:1012900007F0A2FC03F004F80A2007F0C4FC013FA9
:1012A000F6D1D9F800302B60D8F85C313360EAE72A
:1012B00042F6F82295E742F6F822554B00011A80D3
:1012C0000A2390FBF3F00023634AA0F5B06042F8D4
:1012D00023000133122BFAD14F4A6049402011609C
:1012E0004E4A137007F0AAFB00283FF47FAF01239A
:1012F000072790F900005A4A8DE88800594B402191
:1013000007F040FB003018BF01206EE742F6F822DC
:101310003F4B40201A80544A3F4B1A6010223F4BEB
:101320001A7007F08BFB00283FF460AF0123002602
:1013300090F900004D4A8DE848004FF4E133DEE7B4
:1013400042F6F822324B40201A80494A324B1A604A
:101350000822324B1A7007F071FB00283FF446AFA9
:101360000023012190F90000424A8DE80A004FF461
:10137000E133C4E742F6F8220C27254B3E481A8099
:10138000264B3E491F7000233D4A062EDFF80C8194
:10139000DFF80CC1DFF80CE103700B7013701BD089
:1013A0001B2388F8003005234FF4E1368CF80070D9
:1013B0008EF80030334A184B40201A6007F03EFB8D
:1013C00000283FF413AF0122002390F900008DE8BC
:1013D0000C0033462C4A92E721238EF8006088F8EF
:1013E00000308CF80070294EE4E700BFBC100020EC
:1013F0002C160020D4140020642000205820002047
:1014000084150020410A0020440A0020D014002046
:10141000720C0020AD82000818000020C8140020C3
:101420007D8200089D8200088D8200083C16002005
:10143000940B0020401600207E1500209A99193F39
:10144000BC1600208FC2F53DB81600206F12033C79
:10145000B0160020721500207C1E00204D8200086E
:10146000AD840008A08601003982000809840008C4
:1014700021820008C18300080A1E0020051F0020E9
:10148000041F00204D810008B182000890D00300A5
:101490001C150020441600206C0D0020061F0020A3
:1014A000091E0020071F0020DFF8AC9100230F2742
:1014B000C846DFF8A8A12B6033604FF0050B07F09A
:1014C0008BFB02F0EDFE0A2007F0ADFBBBF1010B38
:1014D000F5D12A68DAF80030013F03EB02013268E7
:1014E000D9F85C3129601A443260E6D10F2092FBB2
:1014F000F0F23260484A91FBF0F11378296043F032
:1015000008031370454A137823F00203137040F662
:10151000020223681A4209D0414A424B1A60032250
:10152000414B1A70414B1F80414B1F800122414BA0
:101530009B682360404B1A7098F8003063F07F037B
:1015400088F8003023B0BDE8F08F013B092B3EF650
:1015500079AF4FF480431422C8F8143008268DF870
:101560004A2002220399354806938DF84B20ADF8A6
:10157000486005F083F9049B3C201E6107F053FB93
:10158000069BC8F810304B464FF40049FFF791B95D
:10159000002307EBC303B3F88031003318BF0123E6
:1015A000FEF79DBF94F8383143F0020384F83831D8
:1015B000FFF791BB012B4FF000093FF62EAB204BFC
:1015C0001870FFF745BB42F21073A4F86031A4F81D
:1015D00062311C4BC4F864311B4BC4F868311B4B9F
:1015E000C4F86C311A4BC4F870311A4BC4F874311A
:1015F0005CE4042105241A788154511CC9B2445476
:10160000D11C197006210232D2B28154EEE40232AA
:101610001A701322425417E5801500206915002026
:10162000AE100020941D00208C1D0020981D00206D
:101630009A1D0020A00F0020640D0020000801402A
:10164000840B0020EB350008DD350008E13500088B
:10165000D93500083D3400086C0D002044160020E8
:10166000894B70B51A68908A80B2C1B2CE0739D55D
:10167000118821F400610904090C1180118889B2D4
:1016800041F48061118000211971597919B3997958
:1016900009B301219971D979022901BF118889B251
:1016A00041F400611180197A41F001011182DA7967
:1016B00093F90410013291420CD100229A715A7AA6
:1016C00032B119688A8822F440721204120C8A809E
:1016D00000225A7670BD197A01F0FE011182FF22B4
:1016E0001A71E4E78D073ED5BFF35F8FD879C0B29A
:1016F000012818D15979B1B19979A1B1118821F492
:1017000080610904090C1180BFF35F8F118B118870
:10171000587289B241F400711180918889B241F404
:1017200080619180C3E7118BBFF35F8FD979022964
:101730000FD1597969B1997959B1118821F4806132
:101740000904090C1180918821F480610904090CB5
:10175000E7E7D9790329E0D159790029DDD09979D2
:101760000029DAD0EFE74C0751D501215972597998
:10177000002938D09979002935D0D97993F9040016
:10178000022911881ED921F480610904090C1180F5
:10179000148ADD68E4B22C54C1B2108880B240F4DF
:1017A00000701080881C1871108A013149B2C0B2D3
:1017B0006854918889B241F4806191801188CE0586
:1017C000FCD474E789B241F400711180148ADD6899
:1017D000E4B22C54C1B2148A481C40B2E4B22C5476
:1017E00003311971EAE7997909B9197C39B111887E
:1017F00089B241F40071118019790131F1E7118842
:1018000089B241F48071118001219971D6E711F0FC
:1018100040011AD093F90460118ADD68C9B2F4B2AC
:10182000A955601C40B2DD79C11C8D42187105D1EB
:10183000918821F480610904090C9180DA79904241
:101840007FF435AF02341C7131E705067FF52FAF09
:1018500093F90400441C0AD05C69411C205C49B225
:101860001082D879197188427FF421AF6BE7197122
:10187000197E1182597900297FF465AFD979002941
:101880007FF415AF5FE700BFE40E002037B50F4BC4
:1018900004465D686A4606211878A847A0B19DF8FD
:1018A00000209DF8013043EA022323809DF80220A6
:1018B0009DF8033043EA022363809DF804209DF8DD
:1018C000053043EA0223A38003B030BDA80E0020F8
:1018D00013B50F4B04465B686A4606213B209847C8
:1018E000A0B19DF800209DF8013043EA0223238037
:1018F0009DF802209DF8033043EA022363809DF89F
:1019000004209DF8053043EA0223A38002B010BDF5
:10191000A80E002013B50F4CA27EC2B90E4B1B6857
:10192000ABB11A681AB10D49886902438A619A8875
:101930009868ADF8042002228DF8072004220DEBF0
:1019400002018DF8062004F099FF0123A37602B06E
:1019500010BD00BFE40E0020B40E002000100240B5
:1019600008B5FFF7D7FF4FF48052014B1A8008BD2E
:101970004800002070B50446FFF7CCFFB4F5807F27
:101980003DD0BB2C3DDC612C3DDC292C3DDC132CF7
:101990003DDC092C3DDC002C0CBF002506251E4C2F
:1019A0008021A3686B209847642007F03CF9A36866
:1019B000072168209847642007F035F9A3680021C3
:1019C0006B209847642007F02EF9A36818211B208C
:1019D0009847A36810211C209847A36829461A201D
:1019E0009847A36804211D209847A3680021192067
:1019F0009847A3681221BDE870403720184700259A
:101A0000CDE70125CBE70225C9E70325C7E7042574
:101A1000C5E70525C3E700BFA80E0020012828BFA1
:101A200001202DE9F04F4FF0140E06460EFB00F397
:101A3000704FDFF8D881F918F8586F4B88F81B60A1
:101A4000DC690A69C8F800002243DA6182880D89DE
:101A500022F440721204120C82800222B1F80AA011
:101A60004C6889B045EA0A09C4F8109003A92046D9
:101A70000193ADF80C908DF80F208DF80EE004F076
:101A8000FDFE019B00974FF0080B1F46A268154210
:101A900000F0A2800A20656107F0BAF825610A20EB
:101AA00007F0B6F8BBF1010BF0D1C4F814A00A207E
:101AB00007F0AEF865610A2007F0AAF825610A2050
:101AC00007F0A6F80222C4F810A08DF80F201C22FF
:101AD00003A920468DF80E20ADF80C9004F0CEFE40
:101AE000D8F80040454A03A894423A690BBF42F433
:101AF000001242F480023A613A610BBF3A693A69D6
:101B000022F4001222F480023A61A38823F4407385
:101B10001B041B0CA38023889BB243F0010323808A
:101B2000A58805F0F1FD059B354A364825F03F05AF
:101B3000B3FBF0F0B3FBF2F3002B08BF01232D043D
:101B40002D0C0543ADB2A58021884FF4967221F08B
:101B500001010904090C21804FF47A716FEA4343B3
:101B6000424392FBF1F26FEA534301329BB292B2CD
:101B70002284A383238800259BB243F001032380A2
:101B80002388009A23F4816323F002031B041B0CB7
:101B900023804FF4804323811423012403FB062672
:101BA000737B03A88DF80C308DF80D508DF80E5016
:101BB0008DF80F4000F0D6FE337B9DF80F208DF896
:101BC0000C308DF80D508DF80E504AB103A800F07E
:101BD000C9FE09B0BDE8F08F0A2007F019F855E7F3
:101BE0005A09094903F01F0304FA03F3203241F8AC
:101BF0002230EEE7A4A90108001002400054004082
:101C0000804F120040420F0000E100E0E40E00208F
:101C100010B5204C2368998A89B211F4706F1CBFEB
:101C20000122227711F4E06F1ED01A8B9A88890561
:101C300022F480624FEA02424FEA12429A8013D4A1
:101C40001A88920510D41A88D00517D51A88D1059C
:101C5000FCD41A8892B242F400721A801A88920553
:101C6000FCD4E07EFFF7DAFE2268938A23F47063E7
:101C70001B041B0C93820023637610BD1A8892B25A
:101C800042F400721A809A8822F440721204120CF4
:101C90009A80E9E7E40E0020054A08B5138801336D
:101CA0009BB21380034BD87EFFF7B8FE002008BD1F
:101CB000100F0020E40E002010B44000194CC0B2F8
:101CC000207221760120002121746071E27160761A
:101CD0002068E3606361217710B383889B0515D486
:101CE0000388D9050DD447F230530288920503D5F5
:101CF000013BFAD110BCCFE703889BB243F4807359
:101D0000038083889BB243F44073838047F230534F
:101D1000627E12B1013BFBD1ECE7207F80F0010035
:101D200010BC7047E40E002013460A4601466820A6
:101D3000C2E713B51C4B400002ACC0B2187204F8E5
:101D4000012D19760122002118681A745C615971FD
:101D5000DC60DA715A76197770B18288920517D4EF
:101D60000288D4050FD447F230520188890505D581
:101D7000013AFAD1FFF790FF02B010BD028892B28B
:101D800042F480720280828892B242F44072828071
:101D900047F23052597E11B1013AFBD1EAE7187F80
:101DA00080F00100E8E700BFE40E00200A4601468B
:101DB0006820BEE754E453E42AE729E738B504462F
:101DC00024200D4606F0B0FD4D2006F0ADFD002CA0
:101DD00014BF21203E2006F0A7FD0022064C284615
:101DE00023689A7106F0A0FD236893F84900BDE8C6
:101DF000384006F099BD00BFA01D0020014600201C
:101E0000DCE749282DE9F84F00F06E8300F2A98045
:101E10002C2800F0C4843ED8052800F0158220D874
:101E2000022800F0FC8105D8012800F0EB81002099
:101E3000BDE8F88F032800F000820428F7D10E20B7
:101E4000FFF7DCFF0A2006F081FD0024C14D285D6C
:101E5000013406F069FD0A2CF9D1012006F076FD67
:101E6000E8E1262800F072840AD8222800F0DD83F9
:101E70002428DCD10420FFF7C1FFB74B98680CE29F
:101E8000282800F078842A28D1D10120FFF7B6FF56
:101E9000B14B5879C0E13B2800F0C08337D83628D1
:101EA00000F0E48429D8322800F0A9843428BED177
:101EB0004820FFF7A3FF00250626A84F3C6806FB35
:101EC000054494F8CE0006F02FFD94F8C90006F002
:101ED0002BFD94F8CA0006F027FD94F8CB0006F01D
:101EE00023FD94F8CC0006F01FFD013594F8CD00D9
:101EF00006F01AFD0C2DE1D19CE1382800F0368463
:101F00003A2894D10420FFF779FF0020C5E1422848
:101F100000F08A8412D83D2800F0BD82402886D186
:101F20000820FFF76BFF00248B4D631993F81C0109
:101F3000013406F0F9FC082CF7D17BE1452800F0CC
:101F4000AF8446287FF473AF0D20FFF757FF0020C2
:101F500006F0EAFC002006F002FD002006F0FFFC7F
:101F6000D3E7702800F0C68200F2A280682800F053
:101F7000438258D8642800F0828124D84B2800F08E
:101F80002E844D287FF453AF754D00262878754C6C
:101F900000EB4000C0B2FFF731FF2B7802349E42C5
:101FA00080F0488114F8020C06F0BEFC14F8010C15
:101FB000013600EB800000EB800000F2EE2080B2E2
:101FC00006F0C4FCE9E7652800F06A8166287FF422
:101FD0002EAF1220FFF712FF634B00251B88634CC6
:101FE000B3F5806FD4BF0126082604F1220737F924
:101FF0001500013590FBF6F080B206F0A7FC032D2A
:10200000F5D1208D06F0A2FC608D06F09FFCA08D1E
:10201000574C06F09BFC208806F098FC608806F080
:1020200095FCA0881AE76D2800F0058212D869286F
:1020300000F0EE816C287FF4FAAE4E4C0620FFF7DC
:10204000DDFE208806F082FC608806F07FFC4A4BAB
:10205000188803E76E2800F0F9816F287FF4E7AE57
:10206000464C0B20FFF7CAFE23680025187806F0BF
:102070005BFC2368587806F057FC23682B441879DA
:10208000013506F051FC032DF7D12368D87906F00D
:102090004BFC2368987806F047FC2368D87806F054
:1020A00043FC2368588906F051FC2368187AB3E092
:1020B0007B2800F0028435D8742800F0838010D883
:1020C000722800F0E18273287FF4B1AE0820FFF798
:1020D00095FE0124E0B2013406F026FC092CF9D16A
:1020E000A8E0752800F08E8277287FF4A0AE1F4C00
:1020F00000262079FFF782FE4FF00C08204D671D67
:1021000023799E4280F096800023F05D08FB03F265
:102110005119525D824200F0F28301331C2BF5D13C
:102120000136EDE7F02800F0038331D87C2800F079
:10213000CA83A0287FF47BAE0C20FFF75FFE114B13
:10214000186806F00CFC104B186806F008FC0F4BE2
:102150001868A2E070B40108A00F002084150020C8
:10216000C8140020D410002048000020100F0020C8
:10217000001500205C1D0020781500205815002057
:1021800044AA0108E8F7FF1FECF7FF1FF0F7FF1F55
:10219000FE2800F0BE82FF287FF449AEC34A002328
:1021A00011880122C24C2384114240F0088101337E
:1021B0009BB25200092B92B2F6D10220FFF71EFE0D
:1021C000208C4BE600264FF0010AB94F4FF0000B70
:1021D000DFF810933B795B4540F34C82B54B0C25FF
:1021E0001BF80340002305FB03F202EB090012F881
:1021F0000920A24200F0708301331C2BF3D10BF1B4
:10220000010BE7E70320FFF7F9FD002006F08CFB48
:10221000022006F089FB002006F086FB0AE005207C
:10222000FFF7ECFD0024A44D285D013406F07CFB93
:10223000052CF9D10120BDE8F88FFFF7DFFD012063
:1022400006F072FB0020E4E71A20FFF7D7FD002418
:102250009A4D285D013406F067FB0B2CF9D1002460
:10226000974D285D013406F05FFB082CF9D100245E
:102270000020013406F058FB072CF9D1DAE70720DB
:10228000FFF7BCFDE72006F04FFB8E4B587906F0B8
:102290004BFB002006F048FB042006F060FBC9E77A
:1022A0000B20FFF7ABFD814B814C188806F04EFBED
:1022B0002088012580B206F049FB834B053418685D
:1022C000C0F3C003C0F380029B0043EA4203C0F3A3
:1022D00040021343C0F3401243EAC20300F010006F
:1022E000184306F033FB794B34F8032C1968784B0C
:1022F00002F001001B7814F8016CC3F3800343EA79
:102300004003C2F3400043EA800302F008000343A5
:10231000C2F3800043EA0013C2F3801043EA401383
:1023200001F04000034301F08000034301F480709A
:102330000343C2F3001043EA4023C2F3401043EAD0
:102340008023C2F3002043EAC02301F480500343FA
:1023500001F40050034301F48040034301F40040C2
:10236000034301F48030034301F40030034301F4DC
:102370008020034301F40020034301F48010034351
:10238000C2F3402043EA4053002001F00071C2F341
:1023900080220B4343EA82630246B24209D2115DB6
:1023A00005FA01F119421CBF05FA02F10843013296
:1023B000F3E706F0D4FA434B93F8F4042CE7013B1F
:1023C000072B05D8DFE803F007090C0E10121416CE
:1023D00001232384F1E60223FBE74FF48073F8E73F
:1023E0008023F6E74023F4E72023F2E71023F0E709
:1023F0000823EEE70423ECE71020FFF7FFFC00249E
:10240000344D285D013406F08FFA102CF9D111E714
:10241000314D00242878314E400000F0FE00FFF7D7
:10242000EDFC2B789C42BFF405AF36F8140006F0A3
:102430008DFA0134F5E70820FFF7E0FC64201C4C1E
:10244000A36C584306F08BFAE06C26E70720FFF7F1
:10245000D5FC234B164C1888FF28A8BFFF20C0B21C
:1024600006F062FA206D80F3100080B206F06EFA7A
:10247000B4F8540006F06AFA124B93F8193133B1EC
:102480000A20A36D584380F3100080B2E6E4A06DEB
:1024900000F30F00F9E70B4C0220FFF7AFFC94F8B4
:1024A000740106F041FA94F87301B5E67015002046
:1024B000100F0020150F00206AB401087BB401083A
:1024C00087B40108A00F00207415002060150020BB
:1024D000691500203E0F0020C8140020D4140020ED
:1024E0008E1D002044AA01080220FFF787FCC74B7D
:1024F0009889B3E4C64C1E20FFF780FC23680025B2
:102500001B78022B6BD1DFF81483C24FC24E2368B5
:1025100005F1080253F8220041460FF0D7F817F0F2
:10252000C3FA80F30800C0B206F0FEF9236839460A
:1025300003EB8503D86A0FF0C9F817F0B5FA80F3FA
:102540000800C0B206F0F0F9236805F10E0231462A
:1025500053F822000FF0BAF817F0A6FA80F308003B
:10256000C0B2013506F0E0F9032DD0D1AB4E072DF6
:10257000236827D13146586C0FF0A8F817F094FA69
:1025800080F30800C0B206F0CFF923683146986C9A
:102590000FF09CF817F088FA80F30800C0B206F03C
:1025A000C3F9236893F84C000FF038F817F07CFA61
:1025B000FF28A8BFFF20C0B2013506F0B5F90A2DEB
:1025C000D5D137E62B44587806F0AEF923682B4472
:1025D000D87A06F0A9F923682B44587DECE72368E4
:1025E0002B44587806F0A0F923682B44D87A06F0DB
:1025F0009BF923682B44587D013506F095F90A2D87
:10260000EDD117E62F20FFF7F9FB854C14F8010FE9
:1026100000283FF40FAE06F087F9F7E70120FFF737
:10262000EDFB7B4B1B681878F6E55020FFF7E6FBC7
:1026300000250C27DFF8D8817A4ED8F8004004EB4B
:10264000850494F87930013507FB0363187A06F0A6
:102650006BF994F87A0006F067F994F87B0006F0BD
:1026600063F994F87C0006F05FF9142DE5D1E1E5FB
:102670004644C4E5BAF1000F3FF4DCADF0B2FFF719
:10268000BDFB4FF0000AA1E5604C1620FFF7B6FB3A
:10269000B4F82A0106F05AF9B4F8D00006F056F959
:1026A000B4F8D20006F052F9B4F8D40006F04EF9AE
:1026B000B4F86C0106F04AF9002006F035F9002064
:1026C00006F032F9002006F02FF994F8190106F00F
:1026D0002BF994F8260106F027F9002006F024F9DA
:1026E0004B4B1B68B3F956000A2390FBF3F080B202
:1026F00006F02CF994F80E0106F016F994F8120180
:1027000006F012F994F8110106F00EF994F813018D
:1027100082E50820FFF772FB002006F017F9002081
:1027200006F014F9002006F011F90020FFF796BB1F
:10273000374C0420FFF762FB2368B3F85A0006F019
:1027400005F92368B3F85800FFF788BB2F4C062023
:10275000FFF754FBB4F8E80006F0F8F8B4F8EA0024
:1027600006F0F4F8B4F8EC00FFF778BB0420FFF7AC
:1027700045FB264CBEE7254C0720FFF73FFBB4F88E
:10278000140106F0E3F8B4F8160106F0DFF894F847
:10279000180106F0C9F8B4F81A01FFF75FBB1B4C2B
:1027A0000C20FFF72BFB94F8240106F0BDF8B4F8D9
:1027B0002E0106F0CBF8B4F82A0106F0C7F8B4F8F9
:1027C0002C0106F0C3F894F8250106F0ADF8B4F832
:1027D000300106F0BBF8B4F83201FFF73FBB0B4CF9
:1027E0000420FFF70BFB94F86A0106F09DF894F8BB
:1027F0006B0106F099F8B4F86C01FFF72FBB0120CC
:10280000FFF7FCFA014B93F8260105E5A00F002025
:10281000841500200000C84200007A4400002041D6
:10282000CBA9010844AA0108434C1020FFF7E6FA9F
:10283000607906F079F8A06806F091F894F8240120
:1028400006F072F8B4F8E80006F080F8B4F8EA0090
:1028500006F07CF8B4F8EC0006F078F8B4F814014F
:1028600006F074F8B4F81601FFF7F8BA334D324C9D
:1028700095F85C0004F11006C0EBC000C0B2FFF791
:10288000BDFA94F97E0195F9603083423BD095F909
:102890006C30834237D00834A6423FF4CBACF0E72B
:1028A0001320FFF7ABFA0024254D285D013406F014
:1028B0003BF80B2CF9D1FFF750BB0220FFF79EFA33
:1028C000204BFFF7C5BB0320FFF798FA1E4B187883
:1028D00006F03CF81D4BA6E64568284613F024FD9B
:1028E0008046BAF1000F7FF4C3AE2C46631B9845B7
:1028F0007FF785AC14F8010B06F016F8F6E7087AB6
:1029000006F012F80CE4C0B206F00EF8B4F880013C
:1029100006F01CF894F8820106F006F894F883019A
:1029200006F002F894F8850105F0FEFF94F88401A2
:1029300005F0FAFFAFE700BFA00F0020100F002046
:102940007BB4010846000020C01D002010000020BC
:1029500010B505F0DFFF84B205F0DCFF04EB0020CA
:1029600080B210BD0C4B0D49DB68DB43C3F302237F
:10297000C3F104024378934002781B018818DBB24C
:1029800080F800330123500902F01F0203FA02F21B
:1029900041F82020704700BF00ED00E000E100E0BA
:1029A00073B505460124002601220021006804F0C9
:1029B000BCF92A6801A813889BB243F00103138075
:1029C000EB7A8DF805408DF804308DF806608DF8AF
:1029D0000740FFF7C7FFEB7A1B2B0BD1192301A888
:1029E0008DF804308DF805408DF806608DF80740AD
:1029F000FFF7B8FF02B070BD10B5124C12220021D3
:102A000004F5CA7013F0BAF905230022042001214D
:102A100084F89A3184F89C3184F8A23184F8A43186
:102A2000522384F8962184F89B0184F89D2184F830
:102A30009E1184F8A30184F8A52184F89431A4F8A8
:102A4000981110BD880F00200C4B03F1E802C3F869
:102A50003425C3F8381500F1500302781AB981788B
:102A6000C278914208D304309842F6D10023044A38
:102A700083F00103137070470123F8E7880F0020EB
:102A80001400002007B51C4B03F5A862C3F83C25D1
:102A900093F83C212AB3012A0AD1032183F8421575
:102AA000072183F844250C2283F8431583F8402539
:102AB000124A134B40205A6005F0C0FF70B101224A
:102AC000002390F9000040218DE80C004FF4E13321
:102AD0000C4A05F057FF003018BF012003B05DF825
:102AE00004FB022183F84215032183F8442583F86F
:102AF00043150722DAE700BF880F0020F5810008A0
:102B0000140000207983000800210120FFF756B946
:102B10000B4AD2F8483513F4805FB2F952350AD027
:102B2000B2F84221111A8B4208DD10448342B4BF2F
:102B3000002001207047B2F84401F7E701207047F8
:102B4000880F00202DE9F041424CD4F87025F2B1F5
:102B5000D4F8743504F27E569B1A3F4A04F2845529
:102B600093424FF000033FD804F5AF6030F91320D3
:102B700036F91370590097426F5EC8BF26F81320CC
:102B8000974203F10103B8BF6A52032BEED194F8C8
:102B900090353BB3B4F87A35B4F81C21B4F81A1167
:102BA0009B1AB4F822215343B4F81E2118B2B4F88A
:102BB0007C359B1AB4F824215343B4F878251BB212
:102BC000521AB4F820114A430A2112B292FBF1F2D0
:102BD00093FBF1F3A4F8782590FBF1F2A4F87C358F
:102BE000A4F87A25BDE8F08104F28A574FF0020874
:102BF0003846C4F8703504F58C7C36F913E035F9A5
:102C000013200EEB020191FBF8F1A2EB0E0202EB96
:102C1000820227F813200133032B2CF8021FECD17A
:102C2000B4F98C25B4F98A350A211344B4F98E25F8
:102C30000A4E134400225943835EB51803EB430345
:102C400091FBF3F30232062AA5F80831F4D101F022
:102C5000B9F89CE7880F00207FC3C901A00F0020AE
:102C60002DE9F04FB84C85B0D4F8943580460193E7
:102C700094F89835002702930023B44E04F29C5B2D
:102C80000093DBF80420002A69D092F80090B9F193
:102C9000000F64D0DBF808300199CB1A002B0DDB54
:102CA00001F5FA73CBF808300123009903FA01F11A
:102CB00094F8CC3523EA010384F8CC35029B002B31
:102CC0004DD09BF8003051780433DBB2002940F03E
:102CD000458204EB4303B3F94C15B4F8423103F1D8
:102CE000C800814226DD957894F8CC35009A1341CE
:102CF000DB0734D4002DCCBF0220012005F050FFAB
:102D000009F1FF33132B41D8DFE813F033004900FA
:102D1000540064007C008400E2004801A701D20155
:102D2000FD014000640071008400E2004801D90008
:102D30003F019E01C83B994202DA95786D42D3E784
:102D40000123009A03FA02F294F8CC3523EA020335
:102D500084F8CC35019B03F5FA73CBF80830009B5F
:102D60000BF10C0B0133042B00938AD105B0BDE8A5
:102D7000F08F98F800301D44FA2DA8BFFA2525EAF7
:102D8000E57588F80050404605F09CFE0123009A46
:102D9000934094F8CC25134384F8CC35DFE798F8BA
:102DA00001301D44642DA8BF642525EAE57588F827
:102DB0000150E8E798F80330D4F834151D44642D29
:102DC000A8BF642525EAE57588F80350404605F05C
:102DD0003BFEDBE798F805302B44642BA8BF642347
:102DE000B9F10D0F23EAE37388F80530CED098F8D7
:102DF00004301D44642DA8BF642525EAE57588F8D4
:102E00000450C3E798F806301D4485F3080588F898
:102E10000650BBE7D4F838A59AF80020022A35D12D
:102E200028460EF0FFFB4A490EF004FDDAF82410A4
:102E30000EF044FB394603900EF0E6FD20BB039AEA
:102E4000314610460EF0FEFD039A00B13246B9F14C
:102E50000F0FCAF8242099D028460EF0E3FB3C4916
:102E60000EF0E8FCDAF820100EF028FB3946054693
:102E70000EF0CAFD50BB314628460EF0E3FD00B10E
:102E80003546CAF8205081E73A46E0E79AF8022032
:102E90002A44C82AA8BFC822B9F10F0F22EAE27259
:102EA0008AF802203FF472AF9AF801201544C82D29
:102EB000A8BFC82525EAE5758AF8015066E7D4F869
:102EC00038A59AF80020022AEED1C5E73D46D8E79A
:102ED000D4F838A59AF80020022A3DD128460EF0F1
:102EE000A1FB31460EF0A6FCDAF830100EF0E6FA3F
:102EF000394603900EF088FD60BB039A31461046B8
:102F00000EF0A0FD039A00B13246B9F1100FCAF8D5
:102F100030203FF43BAF28460EF084FB31460EF0E4
:102F200089FCDAF82C100EF0C9FA394605460EF085
:102F30006BFD88BB314628460EF084FD00B1354656
:102F4000CAF82C5022E700BF880F00200000C842BA
:102F5000000020413A46D8E79AF80C202A44C82AB3
:102F6000A8BFC822B9F1100F22EAE2728AF80C2039
:102F70003FF40CAF9AF80B201544C82DA8BFC82504
:102F800025EAE5758AF80B5000E7D4F838A59AF8D9
:102F90000020022AEED1BEE73D46D1E7D4F838A59D
:102FA0009AF80020022A36D128460EF03BFB8749CA
:102FB0000EF040FCDAF83C100EF080FA394603902F
:102FC0000EF022FD28BB039A314610460EF03AFD62
:102FD000039A00B13246B9F1110FCAF83C203FF410
:102FE000D5AE28460EF01EFB78490EF023FCDAF829
:102FF00038100EF063FA394605460EF005FD50BB59
:10300000314628460EF01EFD00B13546CAF838504C
:10301000BCE63A46DFE79AF816202A44C82AA8BF39
:10302000C822B9F1110F22EAE2728AF816203FF4A1
:10303000ADAE9AF815201544C82DA8BFC82525EABD
:10304000E5758AF81550A1E6D4F838A59AF800205D
:10305000022AEED1C5E73D46D8E7D4F8389599F86D
:103060000030022B19D128460EF0DCFA58490EF038
:10307000E1FBD9F828100EF021FA394605460EF08A
:10308000C3FC40B9314628460EF0DCFC00B13546A1
:10309000C9F828507AE63D46FAE799F803301D440E
:1030A000C82DA8BFC82525EAE57589F803506DE647
:1030B000D4F8389599F80030022B19D128460EF033
:1030C000B1FA31460EF0B6FBD9F834100EF0F6F92D
:1030D000394605460EF098FC40B9314628460EF0B8
:1030E000B1FC00B13546C9F834504FE63D46FAE729
:1030F00099F80D301D44C82DA8BFC82525EAE575EF
:1031000089F80D5042E6D4F8389599F80030022B32
:1031100019D128460EF086FA2C490EF08BFBD9F80F
:1031200040100EF0CBF9394605460EF06DFC40B963
:10313000314628460EF086FC00B13546C9F84050AD
:1031400024E63D46FAE799F817301D44C82DA8BF7C
:10315000C82525EAE57589F8175017E601297FF497
:1031600015AEB9F10C0F7FF411AE40F6330104EB4C
:103170004303B3F94C354FF496658B42A8BF0B4619
:103180009078B3F5617FB8BF4FF4617395FBF0F5AC
:10319000A3F5617393FBF5F594F8CD35EDB2AB4231
:1031A0003FF4F4AD032DD4BF2B460223094A84F823
:1031B000CD3509FB032303F2F643C4F8D03500F004
:1031C000B1FB681CC0B205F0EBFCDFE500007A44FF
:1031D00000002041A00F00202DE9F3410E46002100
:1031E00090460B46934C0746B4F84651B4F8440158
:1031F00004F24C5E3EF911209B088242C4BF63F08A
:103200007F03DBB20131AA42B8BF43F04003042977
:10321000F0D194F8D4259A4252D194F8D515F929D1
:1032200002D8013184F8D515834D84F8D4352B7834
:1032300093B9D4F8D835DA074FD5002F44D10023FD
:10324000C4F8DC3502F0D0FF94F8E13584F8E0757D
:10325000DB0701D505F0DEFD94F8D535142B2CD114
:103260002B78B3B194F8D4355F2B06D194F8E135BF
:1032700013F0040748D005F00DFE56B194F8D4358C
:103280007D2B06D194F8E13513F0040742D005F008
:1032900001FE94F8E13513F004020ED194F8D43510
:1032A000572B3DD14FF47A73A4F8EA35D4F8EC35B6
:1032B00013F0080301D1A4F8F03502B0BDE8F081A5
:1032C000002284F8D525AFE7D4F8E435012BC3DC20
:1032D000B4F8E835DF06BFD4BCE7042000F0DFFA1D
:1032E000032000F0DCFA94F8E1355807B4D594F8DF
:1032F0009835002BB0D0B8F1000F02D005F0CAFD10
:10330000AAE7002FA8D1F9E70B2005F023FC84F8E9
:10331000D575B2E70B2005F01DFC84F8D575B8E72C
:10332000D4F84815490719D55A2B17D194F8F23516
:103330002BB1012384F8F22584F8F335BDE794F826
:10334000F43583F0010384F8F4352BB10C2002B07E
:10335000BDE8F04105F0FEBB0D20F8E75D2B48D03D
:103360005B2B55D05E2B55D1032043E00EB17E2B55
:103370005BD094F8D435972B04D14FF4C873A4F8DC
:10338000F6359AE7A72B06D194F8F83543F00403F5
:1033900084F8F83591E70022BB2B019218D1022363
:1033A000ADF80630D4F8FC35BDF80410B3F8582059
:1033B0000A44A3F85820BDF80610B3F85A200A446E
:1033C000A3F85A2000F0FEFC002384F8D53574E7FA
:1033D000B72B02D14FF6FE73E2E7BE2B03D10223D7
:1033E000ADF80430DEE7BD2B7FF467AF4FF6FE7318
:1033F000F6E70120C5B26B1E84F80C3500F0DEFA4A
:1034000000F080FB284602B0BDE8F04105F0C8BBE3
:103410000220EFE7562B01D100F0D4FC2B78002BD3
:10342000A7D094F8D4356F2BA0D102B0BDE8F041FD
:1034300005F0F0BC880F0020140000202DE9F04FAB
:103440001E460027864600208C46614987B04B897E
:103450000C894FEA032AB6EB0A0A67EB000BA4FBC0
:103460000A6704FB0B77B1F80480F40944EA476467
:103470004FEA08460592A219CC884FEAE715A4FB4B
:103480000A6704FB0B77B1F802804FEA162444EA7E
:1034900007644FEAC83645EB000314EB06084FEA11
:1034A000272545EB00098889CDE90223A0FB0A45C1
:1034B00000FB0B55E00D40EA452010F5FA634FEA9A
:1034C000E55141F10004B3F5FA6FCDE9003474F130
:1034D00000035DDA0523A0FB034503FB015504FB54
:1034E00001F300FB0533A4FB00451D446F104FEAB8
:1034F0003406DDE90223921B4FEA940663EB0703CF
:1035000046EA8576AF104FF0FF35324CB8EB06082F
:10351000CDE90223DDE9002369EB0709A242AB41B3
:1035200023DA40F6AC5400250019694100FB01F391
:10353000A0FB000101EB4301CD00C400041B45EAE0
:10354000507561EB0505DDE9022312196B41CDE9E8
:1035500002230B23A0FB034503FB01556D104FEA2B
:103560003404B8EB040869EB05090AFB0BF3AAFB6A
:103570000AAB0BEB430B4FEADA7040EA4B00DDE994
:1035800000344FEAEB711B1A64EB0104CDE90034FF
:10359000059BA3FB080103FB0911DDE90234460D7D
:1035A00046EAC126F31A4FEA615767EB0404DB0BC6
:1035B00043EA4443BEF1000F01D0CEF80030BCF125
:1035C000000F02D0009BCCF8003007B0BDE8F08FB0
:1035D000B80E002024FAFFFF03F093BB03F091BB69
:1035E000012248217720FEF7A4BB01225821772031
:1035F000FEF79FBB80EAE073A3EBE0738B4206DB30
:10360000002801DD401A704702D0084470470020AE
:10361000704770B504460EF035FA2030402859D86E
:103620002D4E2E4D314620460EF00CFA60B92C4E30
:103630002A4D314620460EF0E7F958B1204629467A
:103640000DF03CFF0446F4E7204629460DF034FF18
:103650000446E7E7234920460EF0F4F900282CD071
:10366000204920460DF028FF01461E480DF024FF9A
:103670000446214620460EF029F805461A490EF068
:1036800025F81A490DF018FF29460EF01FF81849C1
:103690000DF014FF29460EF019F816490DF00CFF35
:1036A0002946064620460EF011F8014630460EF037
:1036B0000DF821460DF002FF70BD0F4920460EF0B7
:1036C000A3F90028D5D0074920460DF0F7FE0146A2
:1036D0000948CBE7002070BDDB0F4940DB0FC94034
:1036E000DB0F49C0DB0FC93F9A7C2E36FAAF4F394A
:1036F0003587083CA4AA2A3EDB0FC9BF2DE9F04F4D
:10370000056885B00C4681463A4928460DF0D6FE3C
:10371000FFF77FFF80462846FFF77BFFD9F804506C
:103720000646344928460DF0C9FEFFF772FF0746EA
:103730002846FFF76EFFD9F8089005462D49484600
:103740000DF0BCFEFFF765FF82464846FFF761FFBC
:103750004146814650460DF0B9FF4146019048462A
:103760000DF0B4FF5146029030460DF0AFFF4946D0
:10377000039030460DF0AAFF3946834650460DF0BF
:10378000A5FF4946206007F100400DF09FFF039917
:103790006060A56028460DF099FF02990DF08EFE3D
:1037A0005946E06028460DF091FF014601980DF062
:1037B00083FE3946206106F100400DF087FF019934
:1037C000606128460DF082FF014658460DF074FEF8
:1037D0000299A06128460DF079FF03990DF06EFE65
:1037E0004146E06138460DF071FF206205B0BDE84A
:1037F000F08F00BFDB0FC93F2DE9F04104468AB0CE
:103800002768084601A96668A568FFF777FF019950
:1038100038460DF05BFF0499804630460DF056FFA8
:10382000014640460DF04AFE0799804628460DF0B5
:103830004DFF014640460DF041FE0299206038469A
:103840000DF044FF0599804630460DF03FFF0146DC
:1038500040460DF033FE0899804628460DF036FFAD
:10386000014640460DF02AFE0399606038460DF08F
:103870002DFF0699074630460DF028FF01463846D1
:103880000DF01CFE0999064628460DF01FFF014663
:1038900030460DF013FEA0600AB0BDE8F0810123B0
:1038A000034A03FA00F0138823EA000010807047EF
:1038B000701500200123034A03FA00F0138818430F
:1038C000108070477015002010B5064C228822EA3F
:1038D00000008242208002D0012005F061F920889A
:1038E00010BD00BF120F002010B5054C22881043F8
:1038F0008242208002D0012005F052F9208810BDBC
:10390000120F0020024A936823EA0000906070477B
:10391000A00F0020024A936818439060704700BFD0
:10392000A00F002038B50F4C1925206805F0CAF803
:10393000002220680C4C072A0ED002FB02F3A3F1F0
:103940001901037A4B4303F6C413534393FBF5F376
:1039500024F812300132EEE70449BDE8384005F0A2
:1039600073B800BF58150020A40B00207010002071
:1039700010B5104B1A786A2A1AD140F21C52598895
:10398000914215D11A79BE2A12D193F81A25EF2A3D
:103990000ED10022084C13F8010B80EA0201A34269
:1039A000C9B203D1831A5842584110BD0A46F2E702
:1039B000002010BD00F801081CFD01082DE9F743A7
:1039C00004F086FF6A234A4E40F21C513370BE2336
:1039D0003371EF2386F81A3500231846718086F874
:1039E0001B35F25C01338B4280EA0200F9D186F884
:1039F0001B05042700203F4C3F4BDFF80491636018
:103A000003F188336360013F17F0FF0739D0342397
:103A10003A4DE36005F17848A8F5FC38C8F309038E
:103A2000002B3BD000234FF4005056F80880019340
:103A300003F0B4FE0428E6D123694FF4005043F0AC
:103A4000010323611FFA88F32B8003F0A7FE0428EB
:103A500042D1AB1C0193019B4FEA1848A3F80080A8
:103A60004FF4005003F09AFE2369042823F0010369
:103A70004FEAC3434FEAD3432361C4D104354D45D4
:103A8000C8D11C4A0428136943F08003136102D192
:103A9000FFF76EFF38BB042005F0CFF84FF430205D
:103AA00003F07CFE0428AED123694FF4302043F0AC
:103AB000020323616561236943F04003236103F03E
:103AC0006DFE2369042823F002034FEAC3434FEA43
:103AD000D3432361A6D096E7236923F00103DB04D7
:103AE000DB0C23618FE704F0DDFE03B0BDE8F0835B
:103AF000A00F0020002002402301674500F80108C4
:103B00001CFD01082DE9F041FFF732FF10B9032039
:103B100005F093F8914C04F0DBFE40F21C52904902
:103B200020460BF055FD94F8F4344FF48E71022BBF
:103B3000C4BF002384F8F43494F8F424894D01FBC5
:103B400002F303F5D07020442344286093F8F40175
:103B500001FB02420228C4BF002083F8F40192F85E
:103B6000F431814A13700C2202FB03437F4A03F2B3
:103B7000F643136046F20902A3681A4200F0E5809A
:103B8000A368D80703D54FF40050FFF7BBFEA36826
:103B9000590409D50820FFF7B5FE4FF40050FFF790
:103BA000B1FE0120FFF7AEFEA3681A0706D54FF459
:103BB0000050FFF7A7FE0120FFF7A4FEA3689B04B7
:103BC00012D54FF40040FFF79DFE94F81831012BF9
:103BD00003D14FF40060FFF795FE4FF48030FFF7FC
:103BE00091FE4020FFF78EFE94F872312BB194F8CD
:103BF000763113B1002384F876310020FF27024686
:103C00005B4E5C4B1E602318B3F880114B1003F021
:103C100077334FEAA10C0CF0333CCB1AA3EB0C0327
:103C20004FEAE10C0CF0113CA3EB0C0303EB231364
:103C300003F00F3393FBF7FC11F0010ECCEB0C2CCF
:103C400018BF0132A3EB0C0318BFD2B2012B07DD62
:103C5000022B7FD1BEF1000F7CD011F0BC0F79D0C8
:103C600008301028CFD1013A012A73D8FFF75AFE45
:103C700030220021404812F081F829683F4F01F1BD
:103C80007900FEF7E1FE3E4BA7F126081F602B6886
:103C9000187802F0B9FA3B4B07F174021A606422FB
:103CA00094F86A11384B4A43C8325A6000229A602D
:103CB000DA601A615A619A61DA6183F8202083F828
:103CC0002120324BBA1D1A60314BA7F11E021A6037
:103CD000304B8037C3F800802F4BB4F8F2001F60E0
:103CE0002E4B1E600DF09AFC2D4E7060B4F8F4005F
:103CF0000DF094FC2D68B06095F85C3005F164021D
:103D0000337095F87830B5F81601737094F8753102
:103D10003373244B1E60244B1A600DF083FC014664
:103D200022480DF087FD22490DF0D0FC214B186090
:103D3000214B1D60214B05F211151D60204BC3F86E
:103D40000080BDE8F04104F0ADBD4FF40050FFF736
:103D5000E1FD15E7FEF750FE88E700BFA00F002049
:103D600000F8010884150020551500205815002082
:103D7000BC100020582000202415002096100020A0
:103D8000240B00202816002064200020342000206E
:103D9000680C00206C0C00209C0C0020600D0020A2
:103DA0008C1500208C170020C017002000006144F3
:103DB0004C3D0F44980C0020C41600208C0C0020B1
:103DC000940C002008B5FFF7F9FDFFF79BFEBDE856
:103DD0000840012004F0E4BE2DE9F04FEC4C85B022
:103DE00040F21C520021204611F0C8FF0021E94E8C
:103DF00004F5D0733360E84B04F2F6421970E74BD8
:103E00004FF480401A606A23237003236371FFF725
:103E100081FD4FF40060FFF77DFD0220FFF77AFD82
:103E20004FF48070FFF776FD4FF41673A4F8F2306C
:103E3000FA23A4F8F4302A23A4F8F030C823A4F815
:103E4000FA30012384F8EE3084F810312B2384F803
:103E50001131232384F81231242384F813311023E1
:103E6000A4F816311E232022A4F814314FF4AF73A6
:103E700084F8F620A4F81A310E22022384F80E21C9
:103E800084F81831002705230A2284F8F414A4F8D2
:103E9000FE10A4F8FC10A4F8001184F8E41084F8D3
:103EA000E51084F8E610A4F8E810A4F8EA10A4F8E5
:103EB000EC1084F8EF1084F8F71084F8F81084F808
:103EC0000F2184F8911184F89011C4F89471C4F80A
:103ED000987184F89F3140F2DC53A4F82A3140F203
:103EE0004C43A4F82C3140F26C73A4F82E3140F20C
:103EF0007533A4F8303140F643032546B24684F8C2
:103F00009C1184F89D1184F89E1184F8241184F882
:103F10002511A4F832310329CCBF0123002384F8F2
:103F2000343114BF1E2305230131122984F83531A1
:103F300004F10204EFD14FF47A73A5F85831A5F8D3
:103F40005C31A5F86031A5F86431A5F8D43040F2B1
:103F50007E53C820A5F8D83040F2EA534FF4FA62F5
:103F6000A5F87801A5F8DA3040F24C4040F2B4539D
:103F700000264FF001084FF01E0919214FF0050BE4
:103F8000A5F85A21A5F85E21A5F86221A5F86621B9
:103F9000A5F8D000A5F8D22040F2DC5044F25062DF
:103FA000A5F8DC30322385F875110391A5F8D60009
:103FB0000290A5F8DE30A5F8E02085F8279185F875
:103FC000298185F8738185F8768185F8778185F870
:103FD0007A8185F8266185F8286185F8686185F819
:103FE000726185F874B1A5F8E2300193FEF704FD23
:103FF00040F6AC52DAF800400399AA81AE73E17141
:1040000021214FF0260E23226174532184F801E010
:10401000E27284F802E022734FF00F0E5022E17634
:104020000A21E27084F805E046224FF0220EA174C6
:104030007821627384F806E064224FF00E0EA172BC
:104040002D214FF05A0C227184F810E022774FF0A6
:10405000350E282221754FF4FA7184F8159084F8F2
:10406000169084F8189084F81AE084F808C0267036
:1040700084F817B0A673E6736676627284F81E80C1
:10408000A4F84E1046494FF07F59A163E1634549BA
:10409000DFF824E1A1624FF07E5161634249C4F828
:1040A0002CE0A1644B21C4F830E00298DFF80CE169
:1040B000C4F82090C4F8249084F84C1084F8506020
:1040C00084F8516084F852602764C4F844E084F8AE
:1040D000536085F8F6C4A5F800054FF0410C0320A5
:1040E000019B85F8F7C485F8F834102385F8FB1494
:1040F00085F8FA1485F8F96485F8FD6485F8FE649E
:1041000085F8FC64A4F85860A4F85A6084F87960D3
:1041100084F87A0084F87E0084F88100022084F814
:104120007B3084F8833084F8883084F88B30152312
:1041300020214FF0300C84F88200042084F868308D
:104140001A4B84F87D80E366194B84F878802367E6
:10415000DFF86C80174BDFF86C9084F87C1084F8E3
:104160007F6084F880C084F8841084F8850084F827
:10417000866084F8876084F889B084F88A6084F85F
:104180008C10A4F8566084F85C00C4F860E01BE072
:10419000A00F002084150020551500205815002080
:1041A0008FC2F53C00002040000040409A99193F22
:1041B000F6287C3F1F856B3FCDCCCC3E0000A04055
:1041C000FCA9010890B4010884F8642084F86520F3
:1041D000636708F1080A16F80910002948D150232E
:1041E00084F81231282384F813314FF44873A4F86B
:1041F00016310A2384F8111184F8141184F8181167
:1042000040F2145285F86A31C823A5F86C2185F86C
:104210006B3185F86E11A5F870316B181031C0291B
:104220001F61FAD121464FF48E7218480BF0D0F975
:1042300021464FF48E7216480BF0CAF9154B1A68D6
:10424000154B1168C5F8021551685960916899605D
:104250001168C5F80E1551681961916859610123FB
:1042600085F81033022385F82C3405B0BDE8F08FB3
:104270000A4816F021FA30B150453EBFA0EB0800C5
:10428000401980F81C610136A5E700BF5C120020D0
:104290007813002058150020A2140020FCA9010862
:1042A00070B5354C2369C01A00280ADB002323614E
:1042B000237D3BB1012B21D004F08EFC23691844EF
:1042C000206170BD2D4DAB68984758B1A369184463
:1042D000E369A0610133202BE36101BF1023400893
:1042E000A061E361236A01332362EB6898470123ED
:1042F00023756B88226913442361DDE71F4D2B6909
:10430000984758B1636A1844A36A60620133802BEE
:10431000A36201BF402340086062A362236A0133A5
:10432000052B236224D16B6898470023E26923623E
:104330002375A369616AB3FBF2F3A26AB1FBF2F1E0
:104340000A468BB9E36A89B9226B00216E69616202
:10435000A161A162E1610A480A49B0470A4B1A68A3
:104360000A4B1A602B88C5E7E362ECE72163ECE7B0
:10437000EB689847F6E700BF8C150020CC0E0020B4
:1043800044160020C80E00201C1500203416002002
:104390002DE9F04F87B00393974B07461E88029193
:1043A00016F00206019212D0944BB3F90060B3F9F3
:1043B0000230002EB8BF7642002BB8BF5B429E424F
:1043C000B8BF1E46B6F5007FA8BF4FF400760025A3
:1043D000DFF854B207F1010A0421884B4FEA45097E
:1043E00033F91520864B520033F91530002B93FB1F
:1043F000F1F1B8BF5B42B3F5206F00F3F3805BF8D7
:104400002500531A0344B3F57A5FA8BF4FF47A53DB
:104410007C488342ACBF4BF825304BF825005BF855
:1044200025009AF80A40C0114443A0119AF80040B0
:10443000714B54431B884FEA85089B0700900AF193
:10444000010A4FEAA4143BD0019B5B429A4203DB72
:10445000019B9342A8BF134642F2107E6A4A6B4802
:1044600039F902209B1A039A32F91520134458F89F
:1044700000201A447245A8BF7246DFF8BCE17245BD
:10448000B8BF724648F80020387A4343387FDB11C2
:1044900000EB8000C0F1000E734503DB8342A8BF30
:1044A00003469E46BB7CA4EB0E045A43009B1213AA
:1044B000981A7043744302EB602300930EEB64245C
:1044C000534B97F851205B5D5943A4EBA1146AB19B
:1044D000504920464144059204910DF0A3F8059AF5
:1044E000049904F00FFC0DF0CDFA04460420444B6F
:1044F00039F90310484B39F9032029F803108A1AB7
:1045000092FBF0F219180C3358F801E058F8030048
:1045100048F801207044104497F8502048F803E010
:1045200052B13E49049288440DF07CF8049A414609
:1045300004F0E8FB0DF0A6FA394B3A4A5B5D013511
:104540005843009B022D1C44A4EB601029F8020084
:104550007FF442AF0420029B99790F314B00274929
:10456000B1F904105943264B4911B3F9043000291D
:1045700093FBF0F3A1EB0303B8BF494232292A4869
:1045800034DC8468797B03FB0141284CA142A8BF3D
:104590002146274CA142ACBF81608460F9784B432F
:1045A00024499B11097803290ADDB7F84E10B1F5AB
:1045B000FA7F05DA4C42A3421BDB8B42A8BF0B46B5
:1045C00081686FF0FF0041F34F31B1F5807FA8BFE4
:1045D0004FF480718142ACBF5B181B18938007B009
:1045E000BDE8F08F00234BF8253018E700218160EB
:1045F000D4E72346E4E700BF120F0020E0160020B6
:10460000380F002080C1FFFF5C1D00203C170020F8
:1046100044170020EC160020C015002028170020A9
:104620005C17002034170020F8160020FEFFFF0F53
:10463000020000F01C210020F0D8FFFF2DE9F04F10
:1046400087B003938F4B0292B3F90020B3F9023085
:10465000002AB8BF5242002BB8BF5B429A42B8BF93
:104660001A460026B2F5FA7F1346A8BF4FF4FA7334
:104670008146B246B346344600930196824B6700AA
:104680001A8812F003003FD0022C39D07D4BD95F3D
:10469000029B49005B42994203DB029B8B42A8BF0D
:1046A0000B46642579496FF0040EC95F5B1A0399C4
:1046B00031F914100B4499F80810594391FBF5F1A6
:1046C00099F81C500EFB05FB594505DB05EB8505EC
:1046D0008D42A8BF0D46AB466D4D55F824100B44D6
:1046E00042F210718B42A8BF0B466A498B42B8BF99
:1046F0000B4699F8121045F824304B431B130193D5
:10470000012801D1022C36D15E4BA00033F907A05D
:10471000614B624ED95F81EAE173A3EBE173B3F5BC
:10472000206F00F3A180022C00F09780502505FB3C
:104730000AF509EB04035B7895FBF3F5042391FB81
:10474000F3F3EB1A35581D44B5F57A5FA8BF4FF463
:104750007A55534B9D42ACBF355033504F4B09EB0C
:10476000040153F824607D2396FBF3F3CE7A5E4375
:10477000402396FBF3F6910779D5022C77D04FF4BE
:10478000FA75009B009903FB0AF871430198C3F581
:10479000FA720BFB028800FB021298FBF5F392FB06
:1047A000F5F53D4A3F4932F90780042298FBF2F2C1
:1047B00014F8018008FB02F86FF04F0298FBF2F842
:1047C00099F85120984472B13749404601EB840171
:1047D000059204910CF026FF059A049904F092FAD0
:1047E0000DF050F9804604202B4BD95F2F4BDA5F38
:1047F00003F1080E8A1A92FBF0F2D95314335EF8D3
:1048000024C053F824004EF824206044104499F842
:104810005020A10043F824C05AB1254B05921944F9
:1048200004910CF0FFFE059A049904F06BFA0DF068
:1048300029F9204B454413F804801F4B00FB08F076
:104840004FF0200890FBF8F00134281A032CD853BD
:104850007FF414AF07B0BDE8F08F8AEAEA73A3EBE8
:10486000EA73642B7FF762AF0023335076E7D307F8
:1048700004D5022C02D0019D5B4692E73546534693
:104880008FE700BFE0160020120F00205C1D002003
:104890003C170020F0D8FFFF380F0020F81600204A
:1048A00080C1FFFF44170020EC160020D415002023
:1048B000281700205C170020341700202DE9F04F46
:1048C00089B00593AA4B804618880C4604920CF0D8
:1048D000A5FEA8490CF0FAFEA74B02901B889B0787
:1048E0004CD5129BA54ADD8940F2E633B2F90000AF
:1048F000401B00F2F31199421146B1F9023040F227
:10490000E63198BF80EAE072A3EB050398BFA2EB03
:10491000E07203F2F31088BF4FF4FA72884230D885
:1049200083EAE370A0EBE3709042B8BF104698F8BA
:104930004C504DB3C0F5FA700CF074FE90490CF079
:1049400079FF4FF07E510CF0B7FD0646642090FBD6
:10495000F5F00CF067FE014630460CF0B7FE4FF064
:104960007E510CF0ABFD002107460DF04DF858B913
:104970004FF07E5138460DF065F830B14FF07E575C
:1049800003E04FF4FA70D2E70027231D00240393BD
:1049900008F120030193039B620013F8015B022CD2
:1049A00003930692774B55D1B3F904000A35684357
:1049B0000CF038FE74490CF03DFF0546734B620065
:1049C000985E0CF02FFE724B196C0CF07FFE0146C6
:1049D00028460CF071FD019B834653F8046B01934C
:1049E0006C4B185D0CF01EFE3146054658460CF027
:1049F0006DFE014628460CF069FE67490CF01AFF6F
:104A000098F8512082462AB1644901EB840104F0F0
:104A100079F98246594602980CF058FE019B604E87
:104A200099680CF053FE5F490CF050FE56F82410C4
:104A30000CF044FD5C49A50081460CF0E5FF002820
:104A400044D15A4948460CF0FDFF002840D0DFF819
:104A50005C913DE033F91460049B5842864203DBCD
:104A6000B342A8BF33461846514B62009B5EC01A42
:104A7000059B33F9143018440CF0D4FD49490CF06F
:104A8000D9FE3D4B8246B3F8009019F0010F04D0D7
:104A9000D8F844100CF01AFE8FE705F114007043AB
:104AA0000CF0C0FD38490CF0C5FE19F0020F0546A8
:104AB00084D0D8F8481050460CF008FE39460CF067
:104AC00005FE014628460CF0F9FC76E7DFF8D890A1
:104AD00046F80590374E5846A9590CF0EDFC45F8BC
:104AE00006B0069002994FF07E500CF0A3FE069B94
:104AF00019460CF0EBFD834606F10C03EA58183614
:104B0000A9591046079306920CF0D8FC59460CF0B0
:104B1000D5FC069A079BAA5198F85020864645F87E
:104B200003B022B12449294404F0ECF886467046CB
:104B300022490CF07FFE019B59690CF0C7FD154B13
:104B40000546185D0CF06EFD014628460CF0BEFDD2
:104B500011490CF06FFE1A4905460CF055FF98BB41
:104B6000184928460CF06EFF78B3164D2DE000BFB3
:104B7000E8200020BD378635120F0020D414002015
:104B80000000FA43E016002000004842380F0020E1
:104B9000C0150020E81600200000C842EC160020D6
:104BA000681700200000204100007AC300007A430B
:104BB0005C1D002004160020281700200000404043
:104BC000000096C3000096430E4D494650460CF037
:104BD00075FC29460CF072FC14F066FFB0F57A7F84
:104BE000A8BF4FF47A70084B62009842B8BF1846CD
:104BF0000134064B032C98527FF4CDAE09B0BDE8CA
:104C0000F08F00BF000096C318FCFFFF3417002090
:104C10000022044B1A605A600022034B1A605A604B
:104C2000704700BF3C170020601700202DE9F74FA8
:104C30005D4C5E4A94F821909046B9F1010F0CBF8B
:104C40004FF0000A4FF0030A594D11682F7801F018
:104C50008063584EDFF868B107F00407019394F8B9
:104C60002010052914D8DFE801F003203D5C71898C
:104C700037B1B9F1010F0BD0012184F82010EEE714
:104C8000019B4FF480606BB1FEF72EFE0023236181
:104C9000BAF1000F00F08480504603B0BDE8F04F39
:104CA00003F058BFFEF710FEF0E7B9F1010F01D194
:104CB0000521E2E70121E17002214FF4806084F8D0
:104CC0002010FEF711FEDBF868003368417864209D
:104CD00000FB013161612188052001312180FEF74F
:104CE000E9FDBCE7B9F1010F04BF052184F82010EC
:104CF0006FB14FF0020ADBF86C10B1F90E002E49CB
:104D0000088048808880DBF868004088C880306868
:104D1000616981423FD3002F3DD0B9F1010F9ED090
:104D2000B6E7297841F00201297004F0B3F8306841
:104D3000E1690144A161042184F820104FF48060EE
:104D4000FEF7C2FD0520FEF7AAFD88E7B9F1010FC5
:104D50000FD13068A16981429AD2184B197819B9DC
:104D6000D8F80010CB0793D4297821F002012970DC
:104D70009EE73268E3691344A36189E7DBF86800C2
:104D80003368C188642000FB01312161002184F86F
:104D90002010E170D2E742F21071E16103216CE76B
:104DA00003B0BDE8F08F00BF642000206015002034
:104DB000691500201C150020D414002014000020C8
:104DC000C015002042F20F732DE9F74FC14C266F3A
:104DD000861B9E4240F2B48044F620639E422067C8
:104DE00001D901F001FABC4D2B7853B1BB4B1B78B4
:104DF00013F0040705D10022B94B1A6001F0F4F951
:104E00002F70D4F87480D4F87890C14560D0D4F86D
:104E100080000CF007FC8246D4F884000CF002FC01
:104E2000014650460CF006FDE76F14F0C9FE8246BD
:104E3000A8EB09000CF0F2FBAA490CF047FC4FF07C
:104E40007C510CF0FFFD002840D1642007F5D547C8
:104E5000333797FBF0F00CF0E5FB51460CF036FCD5
:104E6000A1490CF033FCA1490CF030FCD4F8883097
:104E700007460A2B0DDC0023C4F88C00C4F89030E0
:104E8000C4F8940001F0B0F9D4F888300133C4F8C4
:104E90008830D4F898300F2B3FD1D4F89C3004EBF5
:104EA000830201330F2B08BF0023C4F89C300E236C
:104EB000D2F8A000C4F89830D4F890100CF0FEFAA4
:104EC000014638460CF0F8FAC4F8DC00C4F87880E3
:104ED000874B1F6827B3874B98680CF0A3FB80466D
:104EE00038460CF09FFB014640460CF0A3FCC4F88A
:104EF000E000D4F8E000D4F8E810C4F8E4000CF0C6
:104F0000E5FB7D4907460CF07FFD68B97B493846D3
:104F10000CF098FD48B1794F07E0D4F88C00CBE74E
:104F20000023C4F8E030E4E7734FC4F8E07001F008
:104F30005BF9D4F8EC30052B05DC0133C4F8EC3018
:104F400003B0BDE8F08F30460CF068FB6C490CF004
:104F500071FC0646D4F8DC80D4F8F01040460CF022
:104F6000B5FB31460CF0B2FBD4F8F4100CF0A6FA05
:104F70005B4F8146D4F8F810C4F8F40040460CF0BA
:104F8000A5FB31460CF0A2FB39680CF097FAD4F877
:104F9000FC10824640460CF099FB31460CF096FB23
:104FA000D4F890100CF08AFAD4F8E0108346C4F8D4
:104FB000900048460CF082FA31460CF087FB0190D5
:104FC0000AF0BEFD00224F4B0AF00EFE804650460E
:104FD00089460AF0B5FD02460B46404649460AF0AE
:104FE00051FC8046304689460AF0AAFD02460B462F
:104FF000404649460AF0F8FD8046D4F88C008946C0
:105000000AF09EFD02460B46404649460AF03AFC2D
:105010000CF0FEF90146C4F88C00064658460CF028
:105020004DFA01998046C4F8940050460CF046FAB7
:10503000386014F039FD344F3860404614F034FDC8
:10504000D4F8982031490E2A0860314B384621DCCB
:105050001F68013201370E2FC8BF00271F601F686D
:10506000C4F8982004EB8707C7F8A060076840F2EF
:105070003E60284ED4F8E480328802F21F3292B2A9
:10508000824205D8728802F21F3292B2824243D91C
:105090000020B8E01A6801320F2A1A6009D10022F4
:1050A0001A60D4F89C20C4F8A0600132C4F89C2097
:1050B000DCE704EB8202C2F8A060D4F89C20013245
:1050C0000F2A08BF0022F1E7D4F8080153E0C4F822
:1050D0000C616BE0C01500206815002069150020E8
:1050E000641500206F12833A8E2BEA410000C842FB
:1050F000D4170020C4170020000048C40000484412
:10510000002474490000E03F501D0020580F00208B
:105110001C0000205C1D0020444AD4F8149116782D
:1051200016F0040603D10A681432C4F800211B7972
:10513000002BC9D10868D4F8003105211B1AB3F53A
:10514000FA7FA8BF4FF4FA7339489842B8BF18469F
:10515000FEF750FAD4F804311B795843802390FBB2
:10516000F3F0B0F5967FA8BF4FF49670A3F5D67311
:105170009842B8BF18462023D4F80411C01B8A7A7D
:10518000424392FBF3F2B2F5967FA8BF4FF49672BA
:10519000A3F5A6739A42B8BF1A46002E97D0D4F84A
:1051A0000C310E7D00FB0630C4F80C01D4F80C3134
:1051B0002048B3F5161FA8BF4FF416138342B8BF9B
:1051C00003464FF40056C4F80C3193FBF6F3887F86
:1051D0009E180CF027FA4946824640460CF06EF9BC
:1051E000014650460CF072FA4FF06C510CF06EFA1A
:1051F0000CF048FC9628A8BF96206FF095039842C3
:10520000ACBF301AF01AC4F8100105213846C4F8B2
:105210001481FEF7EFF9002F074BB8BF7F42C82F6C
:1052200018607FF78DAE01232B7089E66915002089
:105230000CFEFFFF0080DAFF5C0F00202DE9F04735
:105240002F4E044635682F4928460CF037F9FEF7F3
:10525000E0F980462846FEF7DCF9766805462949DC
:1052600030460CF02BF9FEF7D4F982463046FEF7B3
:10527000D0F92168814650460CF028FA6768A66884
:105280003946044628460CF021FA49460CF01EFA2D
:10529000014620460CF012F93146044648460CF00F
:1052A00015FA41460CF012FA014620460CF006F9B8
:1052B0004146044638460CF009FA3146074628466E
:1052C0000CF004FA014638460CF0F6F8214614F0CA
:1052D00075FC0D490CF0FAF90C490CF0ABFA002101
:1052E0000CF0ECF80A490CF0A5FA14F0DDFB03B25F
:1052F000002BBCBF00F5B47003B21846BDE8F087C0
:10530000D8160020DB0FC93F0000E144DB0F494005
:10531000000020412DE9F04F87B00493854B0746EC
:105320001B8802929C0740F1D78040F2E632824807
:10533000109BDD89B0F900305B1B03F2F31494423B
:1053400004469CBF83EAE370A0EBE37040F2E633CF
:10535000B4F9022088BF4FF4FA70521B02F2F31422
:105360009C4200F2B68082EAE273A3EBE2738342CE
:10537000B8BF03460522C3F5FA7393FBF2F30A2282
:10538000643B5A433B7FDB105343642293FBF2F3AD
:10539000134423EAE3735BB200244FF06408DFF8A0
:1053A000BC9100930B1D019309F1100B019B61004F
:1053B00013F8012B022C01930391604B40F08E8077
:1053C000B3F90C501B3255436D115D4B62009B5E6F
:1053D000042293FBF2F307EB040A9AF80160ED1A3A
:1053E00005FB06F314F8096097F851205E4396FB1D
:1053F000F8F6F61172B15349304601EB840105927B
:1054000003910CF00FF9059A039903F07BFC0CF063
:1054100039FB06464C4B9AF80B2018884B4900FB89
:1054200005F3DB12534319F8042000115A4392FB91
:10543000F8F25BF824304FEA840C1A44B2F5001FEE
:10544000A8BF4FF40012424B9A42B8BF1A465313FA
:105450004BF824204FF6FF7292FBF0F0039351F8C3
:10546000243001F10C02EB1A434341F8245001F1BE
:10547000180552F824E09B1155F8240042F8243016
:1054800097F850207044184445F824E05AB124316C
:1054900001EB0C0505920CF0C5F8059A294603F0BE
:1054A00031FC0CF0EFFA9AF815306200434319F81A
:1054B00004000134584390FBF8F0039B032C1E4476
:1054C000244B06EB20269E527FF470AF07B0BDE858
:1054D000F08F4FF4FA734DE764235DE7083333F937
:1054E0001450029B69005B42994203DB029B8B4292
:1054F000A8BF0B4618496000095E5B1A049931F990
:10550000141019440B4B1B88D8070FD41B3255437A
:105510009B074FEA25157FF558AFBB7C009A4B439C
:10552000534393FBF8F305EB23154EE73D7A4D43C8
:105530002D114AE7120F0020D4140020D8160020A5
:10554000380F0020EC160020E8200020041700206F
:105550000000E0FF341700205C1D0020E81600204A
:105560002DE9F04F89B00693B04B0591B3F90810BF
:105570000492B3F90A200029B8BF4942002AB8BFF3
:1055800052429142B8BF11460026B1F5FA7F0A4651
:10559000A8BF4FF4FA720746B1463446019202960C
:1055A000039603F1200AA24B198811F003003AD0A8
:1055B000A04B650033F91420049B52005B429A42D1
:1055C00003DB049B9342A8BF13469B4A6FF0040978
:1055D000AA5E64259B1A069A32F9142013443A7A7B
:1055E0005A4392FBF5F23D7F09FB05F94A4504DB7E
:1055F00005EB85099145A8BF9146904D55F82420AB
:10560000134442F210729342A8BF13468C4A93424D
:10561000B8BF1346BA7C45F82430534301284FEAFB
:105620002333039333D0834B33F914300293854BE8
:1056300033F9142082EAE273A3EBE273B3F5206F2F
:1056400000F3E3805023029843433819407893FBDA
:10565000F0F3042092FBF0F29B1A5AF82420134432
:10566000B3F57A5FA8BF4FF47A53774A9342ACBF41
:105670004AF824304AF824207D235AF824603A1945
:1056800096FBF3F3D67A5E43402396FBF3F68A0744
:1056900040F1BF804FF4FA75019B0299039803FB18
:1056A00001F80199C3F5FA72714309FB028800FB06
:1056B000021298FBF5F392FBF5F562000792614A3E
:1056C000624932F91480042298FBF2F214F8018046
:1056D00008FB02F86FF04F0298FBF2F897F85120A0
:1056E00098446AB1583901EB840B404607920BF09D
:1056F00099FF079A594603F005FB0CF0C3F9804661
:105700000420504B6200D15E514B4FEA840BD25EB5
:1057100003F1040E8A1A92FBF0F203F10C0C600004
:10572000C1525EF824105CF824004EF8242008448E
:10573000104497F850204CF8241052B1203B9B4461
:1057400007920BF06FFF079A594603F0DBFA0CF053
:1057500099F9364A454402F1840111F80480610048
:1057600000FB08F04FF0200890FBF8F0013402F144
:105770005C032D1A022CCD527FF415AF0420059B3B
:1057800099790F314B00B2F90C1059432D4B491147
:10579000B3F90430002993FBF0F3A1EB0303B8BF86
:1057A000494232293CDC906A797B03FB010129489C
:1057B0008142A8BF014628488142ACBF91629062F5
:1057C000F9784B4325499B11097803290ADDB7F87D
:1057D0004E10B1F5FA7F05DA4842834223DB8B4253
:1057E000A8BF0B46916A6FF0FF0041F34F31B1F54E
:1057F000807FA8BF4FF480718142ACBF5B181B183B
:10580000A2F8603009B0BDE8F08F00234AF82430D8
:1058100032E7CB0759BF3546029B039D4B464CE709
:1058200000219162CCE70346DCE700BFD8160020D8
:10583000120F0020E01600205C1D00203C17002005
:10584000F0D8FFFF380F002080C1FFFF4417002071
:1058500048170020FEFFFF0F020000F01C2100206F
:105860002DE9F04F054690F850008BB00891059255
:105870000993002800F0B7803228A8BF32200BF02F
:10588000D1FE0146BA480BF0D5FF0446B94B188843
:10589000002808BF01200BF0C5FEB74906900BF0A9
:1058A00015FF0146019020460BF008FE01460198C5
:1058B0000BF0C0FFB14B07901B889B0740F1958010
:1058C000AF4BB3F90800B3F90A300028B8BF404223
:1058D000002BB8BF5B429842B8BF1846B0F5E17FD5
:1058E000A8BF4FF4E1700BF09DFEA6490BF0A2FF9C
:1058F00004904FF000090024CDF80890022CA24E2D
:1059000000F06F8136F914706300384603930BF092
:1059100089FE9E490BF0DAFE0CF0B4F80BF082FE23
:105920009B490BF0D3FE9B4B039033F914000BF013
:1059300079FE924B0646B3F8008018F0030F65D04D
:1059400001460BF0BBFD0CF09DF8059B5B429842B5
:1059500003DB059B8342A8BF03468F4A6100885E34
:10596000099A1B1A32F9140018440BF05BFE8246A8
:10597000287F0BF053FE89490BF0A8FE8346287A56
:105980000BF04CFE51460BF0A1FE85490BF09EFE3C
:105990000CF078F881460BF100400CF073F881456B
:1059A00005DB58460CF06EF84845A8BF48460BF09A
:1059B00039FEDFF820925146029001980BF086FEE6
:1059C00059F824100BF07AFD76494FEA840B824691
:1059D0000CF01AF860B9744950460CF033F848B12D
:1059E000DFF8C4A106E0714C50E70023049380E780
:1059F000DFF8B0A149F80BA0A87C0BF00FFE5146D0
:105A00000BF064FE6A490BF061FE814618F0010F4D
:105A100040F0E480002FB8BF7F42B7F5206F4FEA17
:105A2000840A7BDD0022634B43F824202B19D87AAB
:105A30000BF0F4FD5F4B53F824100BF047FE5E496A
:105A40000BF044FE18F0020F074615D002993046BD
:105A50000BF032FD04990BF039FE02990BF02EFD8C
:105A60004946064638460BF027FD04990BF02EFEFA
:105A700049460BF023FD0746DFF85C8118F8040067
:105A80000BF0D0FD03990BF021FE4C490BF01EFEEC
:105A9000014630460BF010FD95F85120824632B198
:105AA000A8F1580101EB840103F02CF98246444E21
:105AB000039856F824100BF0FFFC06F1080B01992F
:105AC0000BF0B8FE039B5BF8248046F82430414677
:105AD0000BF0F2FC07990BF0F9FD41460BF0EEFCE0
:105AE00039464BF82400804650460BF0E7FCA6F1FF
:105AF00018038246185D0BF095FD41460BF0E6FD5C
:105B000030490BF0E3FD014650460BF0D5FC13F095
:105B1000CBFF403E6300F0520134EFE62A493046A5
:105B20000BF0D4FD2B19074658780BF077FD014692
:105B300038460BF07FFE1F4F03990BF0BDFC019917
:105B40000BF0C4FD57F824100BF0B8FC1F49834636
:105B50000BF05AFF38B91E4958460BF073FF20B1BD
:105B6000DFF86CB001E0DFF864B047F80AB05DE739
:105B700083F9223EE8200020BD378635120F002031
:105B8000D81600200000E143380F00200000A03E9E
:105B9000CDCC4C40E01600205C1D00200000A04051
:105BA0006F12033C0000F0C10000F041AF4C593CC3
:105BB0000AD7A33D681700200AD7233CA69B443B85
:105BC00074170020F7CC92380000A043000040C3B7
:105BD0000000404360170020441700204F46029EFB
:105BE0004AE706980BF04EFF20F003000BF01AFD79
:105BF00073490BF01FFE089B95F853908046714C3B
:105C00009B79B9F1000F78D0B4F90C9089EAE97A60
:105C1000AAEBE97A0AFB03F06B4B90FBF3F0EB780D
:105C200064305843642390FBF3F00BF0FBFC0190CD
:105C3000B6F904000BF0F6FC4FF07A510BF046FD7C
:105C400013F032FF83460BF0EDFC019B19460BF07D
:105C50003DFD5E490BF0EEFD064648460BF0E2FCCA
:105C600031460BF029FC8BEAEB73A3EBEB73B3F536
:105C7000207F064602DCBAF1640F19DD0023A3621F
:105C800095F8512022B13046514903F03BF80646C1
:105C9000394630460BF012FC0BF0F4FE00B20BF06C
:105CA000C1FC13F001FFA4F860000BB0BDE8F08F59
:105CB000502000FB09F9E87899FBF0F0A0EB0B000D
:105CC0000BF0B0FC41460BF001FD0BF0DBFEA36ACC
:105CD0001844B0F57A5FA8BF4FF47A503D4B984214
:105CE000B8BF18467D23A06290FBF3F06B7B58434E
:105CF00080110BF097FC0746C2E7B4F90C705B000B
:105D000028337B43B6F904005F110BF08BFC4FF096
:105D10007A510BF0DBFC13F0C7FE381A0BF082FC53
:105D2000002FB8BF7F42322F064631DDC4F82890DD
:105D3000A36A6FF0FF005B13B3F5807FA8BF4FF439
:105D400080739842B8BF18460BF06CFC074630468B
:105D50000BF098FEEB78584380110BF063FC1E4B60
:105D600006461B78032B8BDDB5F84E80B8F5FA7F1D
:105D700086DA0BF087FEC8F10003984203DB80450A
:105D80004346A8BF034618460BF04CFC064677E78F
:105D9000687B0BF043FC31460BF098FC41460BF05E
:105DA00095FC0BF06FFEA36A18440C4B9842A8BFF9
:105DB00018460B4B9842ACBFA062A362B8E700BF85
:105DC00000803B45D81600200CFEFFFF0000A042DB
:105DD000F416002080C1FFFF1C210020FEFFFF0FF2
:105DE000020000F02DE9F04F93B002F0F5FE00271D
:105DF0000546574CDFF87081D4F8AC304646C31ADC
:105E0000184601930BF00AFCD4F8B0100BF05EFCBE
:105E1000C4F8AC503D46D4F8B430DFF850A11B783C
:105E2000049002934B4B0DF124091A8805930392B9
:105E300004F1B80B6B000693474B33F915000BF0D8
:105E4000F1FB04990BF042FC029B49F82500002B62
:105E50004FD018460BF0E6FB01464FF07E500BF09A
:105E6000E9FC014607904FF07E500BF025FB5BF8F4
:105E700025100BF02BFC06903AF915000BF0D2FB25
:105E8000079B19460BF022FC069A014610460BF0C0
:105E900015FB4BF825000BF0F5FD28F815006B00FD
:105EA00033F90830039A5B4393FBF2F30135032D7A
:105EB0001F44BFD164235F4397FBF2F7274B09A927
:105EC0001F60493F2648BFB2FDF796FC3B2F15D90E
:105ED000B4F9D0000BF0A6FBD4F8CC50014628460C
:105EE0000BF0B0FD1F4B002842D11A7822F00802B7
:105EF00041E03AF8153028F81530D0E7D4F8B4303E
:105F00004FF07E515F684FF0000A38460BF0D6FA2A
:105F100001464FF07E500BF08DFC8046104D36F957
:105F20001A000BF07FFB55F82A10834638460BF019
:105F3000CDFB014658460BF0C1FA41460BF0C6FBBB
:105F400045F82A000AF1010ABAF1030FE7D1BFE7C9
:105F5000D816002048000020380F00206C150020C3
:105F60009C17002080150020320F002050200020B8
:105F70001A7842F008022946D4F8C8001A7013F0C3
:105F80001DFED4F8C81080462060D4F8C400D4F8B0
:105F9000CCA000F1004508460BF098FB514607469F
:105FA00050460BF093FB014638460BF087FA13F08E
:105FB0007DFE0146284613F001FE824907466060D7
:105FC00040460BF083FB13F06FFD7F4D7D49288029
:105FD00038460BF07BFB13F067FD7C4B68801B6839
:105FE0001A0740F1B48009A97948FDF705FCD4F8F7
:105FF000B4304FF07E51D3F80880002540460BF0B6
:106000005DFA01464FF07E500BF014FC8146704F54
:10601000DFF8D0B13BF915000BF004FB57F8251061
:10602000824640460BF052FB014650460BF046FAC2
:1060300049460BF04BFB47F825000135032DE9D10C
:106040006348FFF7FBF8634B1880236803F10043B4
:106050000C93636803F100430D935E4BB3F90000AA
:106060000BF0E0FA5C4900F100400BF02FFB0E90C2
:10607000B6F900000BF0D6FA0F90B6F902000BF05B
:10608000D1FA1090B6F904000BF0CCFA0CA91190DB
:106090000FA8FDF7B1FBD4F8B4305B78012B40F0CA
:1060A0008D804E4B1B785B0714D4D4F8E0508DB133
:1060B0000823D4F8E400013D90FBF3F3C01A0BF081
:1060C000B1FA11990BF0FAF90BF0DCFCC4F8E050CE
:1060D000C4F8E4000823D4F8E40090FBF3F00BF0DC
:1060E000A1FA014611980BF0E7F911900F9813F0FF
:1060F000DBFCD4F8E8502978FDF77CFAD4F8EC30D2
:106100001844C4F8EC00109813F0CEFC2978FDF781
:1061100071FAD4F8F0301844C4F8F000119813F074
:10612000C3FC6978FDF766FAD4F8F430019A184494
:10613000D4F8F830C4F8F4001344C4F8F830D4F8B4
:10614000FC300133C4F8FC3013B0BDE8F08F244DAF
:1061500049462846FDF750FB2968D5F804900846C3
:106160000BF0B4FA4946074648460BF0AFFA014631
:1061700038460BF0A3F9D5F808800746414640465B
:106180000BF0A4FA014638460BF098F913F08EFD97
:10619000002107460BF02EFC70B9394628680BF039
:1061A00049FB3946286068680BF044FB3946686053
:1061B000A8680BF03FFBA860094842E7059B1888D8
:1061C0008DE700BF4C3D0F445C1D0020741500207E
:1061D000AC1700207815002035FA8E3C6915002098
:1061E00024000020001500200022064BC3F8EC20FC
:1061F000C3F8F020C3F8F420C3F8FC20C3F8F8205B
:10620000704700BFD816002001380A4B042804D874
:10621000DFE800F006080A0C0E00074ADA60704753
:10622000064AFBE7064AF9E7064AF7E7064AF5E7B2
:10623000064AF3E7240000203D46000815530008F5
:10624000BD480008914300086155000861580008E6
:1062500010F80A3C0133DBB20A2B00F80A3C07D9DC
:10626000002310F8131C034A22F8113000F80A3CEE
:10627000704700BFE81E0020314A70B5136C90686B
:10628000194440F68C23081A98429160D0605160FE
:10629000134639D9117892F94520914220D10A1F2D
:1062A000082A1DD893F84620182A03DC013283F807
:1062B000462001E083F8441093F9442091421BD119
:1062C00093F84700C0B100201E4C1F4D824209DCEC
:1062D00000241D480B2A0BDC20F812400132F9E79C
:1062E0000022E4E754F8046F25F810600130EDE770
:1062F0001648027801320270012283F847200022FA
:1063000083F845101A7070BD92F84710B9B140F289
:10631000DA51A0F2EF248C4208D811780B2905DC61
:106320000B1D0131117042F8230070BD0022104690
:1063300083F8472099180432302A0861FAD170BDD9
:106340007C0D0020880D0020E81E0020130A00208C
:10635000024A136C01330B44136470477C0D002018
:10636000024B53F820301B6819807047EC20002046
:10637000074B53F82030A1F57A701A6819894FF449
:106380007A73414391FBF3F189B21180704700BFEA
:10639000EC20002037B504466B46012202210C2078
:1063A000FBF78AFC10B9002003B030BD9DF8003027
:1063B000DA07F8D56B46072203210C20FBF77CFC9B
:1063C0000028F0D09DF806309B07ECD19DF80130F5
:1063D0009DF80000174D40EA032000B20BF022F9AF
:1063E00029680BF073F90BF04DFB9DF8033020800A
:1063F0009DF8020040EA032000B20BF013F969682F
:106400000BF064F90BF03EFB9DF8053060809DF8C1
:10641000040040EA032000B20BF004F9A9680BF075
:1064200055F90BF02FFB0122A0800A210C20FBF76D
:1064300080FCB9E73400002013B500220A210C20AB
:10644000FBF777FC142002F0EEFB0F220A210C2050
:10645000FBF76FFC0A2002F0E6FB01AB03221021E0
:106460000C20FBF729FC0A2002F0DDFB9DF904005B
:106470000BF0D8F84FF086410BF01EF84FF06E513C
:106480000BF024F94FF07E510BF018F825490BF072
:106490001DF9254C20609DF905000BF0C3F84FF065
:1064A00086410BF009F84FF06E510BF00FF94FF0E9
:1064B0007E510BF003F81B490BF008F960609DF961
:1064C00006000BF0AFF84FF086410AF0F5FF4FF0F1
:1064D0006E510BF0FBF84FF07E510AF0EFFF1149BF
:1064E0000BF0F4F80022A0600A210C20FBF721FC3D
:1064F0000A2002F098FB0DF10303012202210C2077
:10650000FBF7DAFB0DF10303012209210C20FBF755
:10651000D3FB01220A210C20FBF70BFC012002B067
:1065200010BD00BF0000F0413400002070B50546EA
:10653000046D8668A38986B023F400531B041B0CEA
:10654000A3818379697913F0020F14BF4FF40052CD
:10655000002213F0040F14BF4FF48060002011F0EC
:10656000010F14BF042300238907218A48BF43F089
:10657000080389B221F4405111432182A28922F4F7
:10658000B05222F00C021204120C02431343A381F6
:10659000A28A01A822F440721204120CA28201F015
:1065A000B3F8204A039B0499944218BF1946192254
:1065B000A3894A4313F4004F14BF7100B100B2FB2A
:1065C000F1F16426B1FBF6F3A2891801120406FB6F
:1065D00013131FD5DA003232B2FBF6F202F00702D3
:1065E00042EA00039BB22381AB792A6D13F0080FB6
:1065F000938A0BBF23F008039BB21B0443F00803EC
:1066000008BF1B0C938293899BB243F40053938180
:1066100006B070BD1B013233B3FBF6F303F00F037A
:106620000343DFE70038014010B57C4B1B78012B9A
:1066300014BF00240324038C002938D123F0010364
:106640001B041B0C0384018B038C89B221F0F30122
:1066500041F0010141EA0411714C9BB2A04242F0A9
:10666000010212D004F50064A0420ED0B0F1804FB8
:106670000BD0A4F59834A04207D004F58064A04262
:1066800003D004F58064A0420ED123F0020313432B
:1066900001830384038B23F00C031B041B0C038373
:1066A000038B9BB2038310BD23F00A03EFE7042999
:1066B00038D123F010031B041B0C0384018B038CC3
:1066C00021F440710905090D41F4807141EA04315A
:1066D000534C9BB2A04212D004F50064A0420ED0ED
:1066E000B0F1804F0BD0A4F59834A04207D004F548
:1066F0008064A04203D004F58064A0420CD123F052
:10670000200343EA021292B242F010020183028493
:10671000038B23F44063C0E723F0A00342F0100290
:106720001A43F3E708293DD123F480731B041B0CA3
:106730000384818B038C89B221F0F30141F00101C4
:1067400041EA0411364C9BB2A04212D004F5006419
:10675000A0420ED0B0F1804F0BD0A4F59834A042E7
:1067600007D004F58064A04203D004F58064A04201
:1067700012D123F4007343EA022292B242F48072EF
:1067800081830284838B23F00C031B041B0C838303
:10679000838B9BB2838310BD23F4206342F4807209
:1067A0001A43EDE723F480531B041B0C0384818BF5
:1067B000038C21F440710905090D41F4807141EA0F
:1067C0000431174C9BB2A04212D004F50064A042E1
:1067D0000ED0B0F1804F0BD0A4F59834A04207D072
:1067E00004F58064A04203D004F58064A0420CD17B
:1067F00023F4005343EA023292B242F4805281837E
:106800000284838B23F44063BFE723F400735B04AB
:106810005B0C42F480521A43F1E700BF780D002070
:10682000002C014038B510F80E2C044650F8043CFA
:1068300052B9012220F80C1C00F80E2C997A186825
:106840000222BDE83840EFE6002530F80C2C20F895
:106850000A1C891A89B220F8081C074A10F80F0C84
:1068600022F8101004F80E5C2A46997A1868FFF78F
:10687000DBFE04F8065C38BDE81E00202DE9F0437D
:1068800000234FF00F0E01260F8847FA03F2D207BC
:1068900023D58C784FEAD30814F0100F18BF91F865
:1068A000039003F0070504F00F024FEA850550F846
:1068B00028C018BF42EA09020EFA05F92CEA090CB1
:1068C000AA4042EA0C02282C40F828200AD1C268CB
:1068D00006FA03F422EA0402C2600133102BD4D179
:1068E000BDE8F083482CF8D1C46806FA03F22243CD
:1068F000F2E72DE9F743DFF89492164605464F4636
:1069000099F800400A46006831469846631C07F82B
:10691000043B00F00AFA2B8901A9ADF804301823D2
:106920008DF80630022368688DF80730FFF7A6FF60
:1069300095F80AE0240127442A684946BEF10C0F65
:1069400043D8DFE80EF00742424268424242A0428A
:106950004242D900138CDFF8389223F001031B0464
:106960001B0C1384138CB2F804C0108B4A4520F022
:1069700073004FEA00404FEA10409BB21FFA8CFCB4
:1069800040F070003ED009F500694A453AD009F55B
:1069900040694A4536D009F580694A4532D009F543
:1069A00080694A452ED023F0020343F00303A2F886
:1069B00004C01083A2F834801384138B23F00803DF
:1069C0001B041B0C43F0080313832B7B43B1B2F869
:1069D00044306FEA43436FEA53439BB2A2F844301A
:1069E00013889BB243F001031380BEF10C0F00F239
:1069F000B980DFE80EF0B3B7B7B7BEB7B7B7C2B765
:106A0000B7B7C60023F00E032CF4407C43F0030319
:106A10004CF4807CCBE7138CDFF8749123F01003E7
:106A20001B041B0C1384138CB2F804C0108B4A4552
:106A300020F4E6404FEA00404FEA10409BB21FFAB4
:106A40008CFC40F4E04015D009F500694A4511D0AE
:106A500023F0200343F03003A2F804C01083A2F80F
:106A600038801384138B23F400631B041B0C43F442
:106A70000063A9E723F0E0032CF4406C43F03003FB
:106A80004CF4806CE8E7138CDFF8049123F48073F6
:106A90001B041B0C1384138CB2F804C0908B4A4562
:106AA00020F073004FEA00404FEA10409BB21FFAFB
:106AB0008CFC40F0700016D009F500694A4512D0F0
:106AC00023F4007343F44073A2F804C09083A2F847
:106AD0003C801384938B23F008031B041B0C43F0AE
:106AE0000803938371E723F460632CF4405C43F460
:106AF00040734CF4805CE7E7138CDFF8949023F448
:106B000080531B041B0C1384108CB2F804C0938BAD
:106B100020F4005023F4E6431B0400041B0C000C7B
:106B20004A451FFA8CFC43F4E04340F4405003D044
:106B300009F500694A4503D12CF4804C4CF4804C93
:106B4000A2F804C09383A2F840801084938B23F4AE
:106B500000631B041B0C43F40063C2E70B1902F132
:106B600034005860384621448E818A6003B0BDE805
:106B7000F0830B1902F13800F3E70B1902F13C0026
:106B8000EFE70B1902F14000EBE700BFD817002038
:106B9000002C0140026D70B515880446ADB2A906FF
:106BA00006D5036B23B9C36AA3B1908880B2984716
:106BB0002B0620D5636AA26A9A42236D17D0511C16
:106BC000A069A162825C9A802369994213D3002351
:106BD000A36270BDE169928840694E1CD2B2E66141
:106BE0004254E169E268914228BFE361E0E7DA6874
:106BF00022F08002DA6070BD10B5046B0346C168F4
:106C0000406944B11A6C8C1A013A08BF0A46005D0B
:106C10001A64C0B210BD1A6A805C01328A4228BF71
:106C20002246C0B21A6210BD436B13B190F8440003
:106C30007047836A406A1B1A584258417047416A3C
:106C4000826A0369914238BFC9188A1A416B21B11F
:106C500049680A44591E8A4203D2581E801AC0B29B
:106C6000704700207047036B5BB15B68026C934216
:106C7000A3EB020301D3D8B27047C0681844C0B276
:106C80007047C369026A934237BFC068981AC01838
:106C9000801AF4E7836A8169426B1944D160416AC2
:106CA0008B4229BF0169CB1ACB1A53602ABF00233C
:106CB000536083624FF0000380F84430136838BF9C
:106CC000816243F0010313607047436A8269D154C3
:106CD000436A02690133934228BF00234362436B36
:106CE0001BB11B68DB0705D4D4E7026DD36843F002
:106CF0008003D36070474171FFF718BC8160FFF7D4
:106D000015BC07B5032201AB00217720FAF7D4FFA9
:106D10009DF805309DF804001B0243EA00439DF8EE
:106D20000600184303B05DF804FB254B10B5534330
:106D3000244A254C12680139B2FBF3F20388013A68
:106D4000A04289B292B29BB212D004F50064A04274
:106D50000ED0B0F1804F0BD0A4F59834A04207D0EC
:106D600004F58064A04203D004F58064A04202D1FF
:106D700023F070039BB2154CA04206D004F580644A
:106D8000A0421CBF23F440739BB203800E4B81854D
:106D9000984202850FD003F5006398420BD003F5AB
:106DA0004063984207D003F58063984203D003F50F
:106DB0008063984201D1002303860123838210BDA2
:106DC00040420F000C000020002C01400010004049
:106DD0000B4B800A98420FD004D8B0F5801F09D021
:106DE000FE207047074B984208D049339842F7D1AC
:106DF0000020704701207047022070470320704731
:106E00000100100002001000F8B504680546204695
:106E1000FFF7DEFF032841DCAB7A4FEAA30E39B956
:106E20000227A6899D08B6B2AF4026EA0706A681CA
:106E30000A2505FB00E51D4E46F82510043546F8E9
:106E40002520324631B199080223A5898B402B4376
:106E50009BB2A3812823434303F120011144EFF3A4
:106E60001286502585F312880425103313441F68B9
:106E700017B10F6019680431013D03F10403F6D125
:106E80000D60F3B283F31188282303FB0020036A0B
:106E90002BB1A3899BB243F00103A381F8BDA38961
:106EA00023F001031B041B0CF7E700BF2021002087
:106EB00000486FE69C18002000486BE6F0180020A0
:106EC0004FF400520A480B4B5A60D0F888201368E0
:106ED00023F001031B041B0C1360826FC36F9A42E3
:106EE00001D05430D6E6012380F89830704700BFB7
:106EF0009C180020000002402DE9F0431E469E4BE6
:106F00008DB09842894690469DF8507040F0D280EE
:106F10009A4B9B4AC3F85C805A6503F1A8029A66B3
:106F200003F5D472DA664FF480721A665A66954A8F
:106F3000C3F8A400C3F88820A2F54842403AC3F839
:106F40009C20914B9A6942F480429A615A6942F0BE
:106F500001025A6102238DF803304FF400733A079F
:106F6000ADF8003040F194801C23694687488DF8C5
:106F70000230FFF783FC01240E23002501A88DF8C1
:106F800004308DF805408DF807408DF80650FBF76A
:106F9000E9FC252301A88DF805408DF807408DF800
:106FA00004308DF80650FBF7DDFC794C00250123F9
:106FB000256284F84430E561A5626562C4F82C90CE
:106FC0006671C4F80880A7712046FFF7AFFAF20790
:106FD00029D5206B002800F0BD80E36C0395019358
:106FE0004FF480530A9380230693E3680595049336
:106FF0002023099363690795029308950B9500F088
:1070000009FB01A9206B00F0E7FA226B216D1368E0
:1070100043F0010313608B8A9BB243F040038B82E1
:1070200053689BB22364B30728D5606B002800F037
:107030009A80A36C002501934FF480530A93802318
:1070400006932369029504931023059503930795EE
:10705000089509950B9500F0DDFA01A9606B00F029
:10706000BBFA636B1A6842F002021A60226D5D601F
:107070005D60938A9BB243F0800393822046226D29
:1070800093899BB243F4005393810DB0BDE8F08324
:10709000B30706D5182369463C488DF80230FFF740
:1070A000EDFBF5077FF567AF4FF48063ADF8003077
:1070B00048235AE7374B98425BD1304B304AC3F8EC
:1070C00008801A604FF48072DA601A6103F52A7240
:1070D0005A6103F56A729A612F4A18659A64DA64F4
:1070E000294B3C07DA6942F40032DA615A6942F00E
:1070F00001025A614FF002038DF803304FF0040390
:10710000ADF8003016D51C23694620488DF80230B2
:10711000FFF7B4FB262300228DF80430012301A8D9
:107120008DF805308DF806208DF80730134CFBF7ED
:1071300019FC3BE7B00706D51823694613488DF8BC
:107140000230FFF79BFBF107E4D50823ADF80030D0
:107150004823D9E74FF6DF72236D1A80DA6842F0D0
:107160002002DA605FE7226DD36843F08003D360CA
:1071700084E7002089E700BF003801409C18002008
:1071800014AA010844000240001002400008014017
:10719000F01800200044004004440040084BDA6826
:1071A000D10709D4DA68520708D4DB6813F0100F4E
:1071B00014BF03200420704701207047022070474D
:1071C0000020024002680D4B5AB941F288329142C8
:1071D000A8BF11461429B8BF14211A6801601144D0
:1071E00041601A684168521A002AA1BF1A680368F0
:1071F0009B184360ACBF0120002070471C15002085
:10720000F8B505460026094F28460FF08DF8F4B270
:10721000A04206F1010607D9285D01F0A9FB2B5D0C
:107220003A7853403B70EFE7F8BD00BF441D0020A3
:10723000F8B5A44C6368013B062B00F2D380DFE86D
:1072400013F0070054008400E90003012401A001A9
:107250009D4DA2682B689D4E9B1A40F69802934262
:107260000AD93368012043F00803336000236360C8
:10727000BDE8F840FCF728BB0120FCF735FB4B22AA
:10728000934F3B681A715A71336883F00803336077
:10729000E368904E632B03DC4FF4FA63F380F8BD90
:1072A0000120FCF711FB227C552332B93A68537157
:1072B0004FF47A737380022307E0012A09D13A68F8
:1072C00053714FF4FA637380052363602B68636125
:1072D000F8BD032A3A68137103D14FF47A733380EF
:1072E000E9E74FF4FA633380EEE7784A0120136848
:1072F00083F008031360FCF7E7FA227C724B7549B0
:1073000040F201404AB9B4F91A204880B2F5E17F51
:1073100006DD032262601B68D9E7032A08800ED0CD
:10732000022262601B6862699B1AB3F5FA6F59D337
:10733000002363606361BDE8F84001F0ABBDB4F9C0
:107340001810B1F5E17FEBDDE4E7237C93B9B4F9E4
:107350001A30B3F5E17F46DD5C4A0120136883F003
:1073600008031360FCF7B0FA40F27E42594B5A8092
:10737000554BD7E7032B35D1B4F91830B3F5E17F7E
:1073800015DD524A0120136883F008031360FCF7EF
:107390009BFA4FF483624F4B1A804B4B62691B6818
:1073A0009B1AB3F5FA6F1DD3002363608FE79BB27E
:1073B000B3F5E17F16D8638BFA339BB2B3F5FA7F4E
:1073C00010D8424A0120136843F008031360FCF709
:1073D0008BFA4FF483623F4B1A803B4B1B6863610F
:1073E00004236360F8BD9BB2B3F5E17FFAD8238B29
:1073F000FA339BB2B3F5FA7FF4D8344A012013680C
:1074000043F008031360FCF76FFA40F20142314B7E
:107410005A80E2E72D4A0120136843F00803136005
:10742000FCF762FA4FF4FA622A4BDA804B22284BBF
:107430001B685A711A71244B62691B689B1A40F6CB
:10744000B8329342B0D8CBE70120FCF73DFA227C5A
:107450001D4B012A1F4940F2B77007D1B4F91A2019
:10746000488012F5E17F04DA062253E7022A0880F9
:1074700008D005221B68626062699B1AB3F5FA6F37
:1074800092D2F8BDB4F91820EBE7207C012823D173
:10749000B4F91A3013F5E17F59DA0C4A136883F016
:1074A00008031360FCF710FA40F23A72094B5A8055
:1074B000054B62691B689B1AB3F5FA6FBFF474AF92
:1074C000F8BD00BF441D00201C15002060150020E1
:1074D00058150020D4140020022883D1B4F91830A4
:1074E00013F5E17F14DA384A0120136883F00803AA
:1074F0001360FCF7E9F940F2B772344B1A80344B51
:1075000062691B689B1AB3F5FA6FBFF44DAFF8BD03
:1075100003F5E1739BB2B3F5C87F3FF663AF638BAE
:10752000FA339BB2B3F5FA7F3FF65CAF264A0120EF
:10753000136843F008031360FCF7D6F940F23A727F
:10754000224B1A80224B1B686361072349E703F52E
:10755000E1739BB2B3F5C87F3FF644AF238BFA3398
:107560009BB2B3F5FA7F3FF63DAF174A136843F07D
:1075700008031360FCF7B8F940F2B772134B5A8056
:10758000E0E7114A0120136843F008031360FCF799
:10759000ABF94FF4FA62237C012B18BF4FF4AF61B3
:1075A0000A4BDA804FF04B0218BF1980094B1B6859
:1075B0001A715A71064B62691B689B1AB3F57A7F80
:1075C000C3D900230DE700BF60150020D4140020AC
:1075D0001C150020581500208B6810B50C6A026835
:1075E00023430C6922F4FF4223434C6922F07002CA
:1075F00023438C692343CC6923434C6A23438C6A1D
:10760000234313430360CB6843600B6883604B687C
:10761000C36010BD036823F001031B041B0C03604F
:107620000023036043608360C360294B984204D108
:10763000284A536843F00F0326E0274B984204D1B1
:10764000244A536843F0F0031EE0244B984204D1CF
:10765000204A536843F4706316E0214B984204D1EA
:107660001C4A536843F470430EE01E4B984204D109
:10767000184A536843F4702306E01B4B984205D127
:10768000144A536843F4700353607047174B984291
:1076900004D1104A536843F07063F5E7144B9842E5
:1076A00001D1144AC5E7144B984201D1114AC8E7E9
:1076B000124B984201D10F4ACBE7114B984201D1AE
:1076C0000C4ACEE70F4B9842DFD10A4AD1E700BF00
:1076D00008000240000002401C000240300002404E
:1076E00044000240580002406C000240800002400A
:1076F00008040240000402401C040240300402401E
:1077000044040240580402401F4A10B5536803F075
:107710000C03042B21D0082B22D01C4B0360536890
:107720001B49C3F30313CC5C0368E3404360546814
:10773000C4F302240C5D23FA04F484605468C4F397
:10774000C2240C5DE340C3605268C2F3813211442D
:107750000A7CB3FBF2F3036110BD0E4B1B68DDE73F
:1077600053685168C3F38343C90303F1020302D48E
:1077700009494B43D2E7516811F4003F05490968B4
:1077800018BF4908F5E700BF0010024000127A0058
:1077900030AA01084000002000093D0010B5044651
:1077A000FFF7FCFC012806D10CB9052010BDFFF73E
:1077B000F5FC013CF6E7002C08BF052010BD0F4B7F
:1077C0001A6842F001021A6059680D4A0A405A606C
:1077D0001A6822F0847222F480321A601A6822F445
:1077E00080221A605A6822F4FE025A604FF41F0287
:1077F0009A604FF00062034B9A607047001002409D
:107800000000FFF800ED00E02DE9F8434C4C036860
:10781000023AE36183880D462384062A05D8DFE80F
:1078200002F06A6F747981858A00A38B0B80E38BE9
:107830006B80238CAB80434B1B79002B59D1B5F95E
:10784000000009F0EFFE8046B5F9020009F0EAFEFB
:107850000746B5F9040009F0E5FE616A06464046B0
:1078600009F034FF216B8146384609F02FFF0146AD
:10787000484609F023FEE16B8146304609F026FFB9
:107880000146484609F01AFE12F00EF9A16A288056
:10789000404609F01BFF616B8146384609F016FF30
:1078A0000146484609F00AFE216C8146304609F03F
:1078B0000DFF0146484609F001FE12F0F5F8E16AB5
:1078C0006880404609F002FFA16B8046384609F007
:1078D000FDFE0146404609F0F1FD616C0746304669
:1078E00009F0F4FE0146384609F0E8FD12F0DCF834
:1078F000A880BDE8F883E38B0B80A38B5B4297E7FE
:10790000A38B5B420B80E38BF8E7E38B5B420B803E
:10791000A38B8DE7A38B5B420B80E38B6B80238C67
:107920005B4287E7E38B0B80A38BF7E7A38B0B808E
:10793000E38B5B42F2E7E38B5B420B80A38BF8E7C0
:10794000441D00204000002010B53D4C00F0F4FD27
:1079500094F84830032BB4F84A3026D10A2B1CDDAA
:107960000023282084F8483001F05DF900F0E4FDA0
:10797000B4F84C0000F0C0FD226DD37890FBF3F01A
:1079800001300828A8BF0820537980B24343A4F8E7
:10799000543013795843A4F8560094F84830012B1A
:1079A0001CD00DD3022B3BD010BD0A2BF5DC0323DA
:1079B00084F848300023A4F85430A4F85630ECE79B
:1079C000B4F85420B4F84A309A4237DD012384F8E1
:1079D00048300820BDE8104001F0BCB8194A1378BF
:1079E00023F002031370B4F84A20B4F856309342DF
:1079F00004DD022384F8483007201CE0B4F854303A
:107A000001339A4216DD002384F84830B4F8583028
:107A1000B3F59B7F12DCBDE810400320FBF74ABFA3
:107A2000B4F85630B4F84A2001339A42E4DD012319
:107A300084F84830082001F08DF8E7E710BD00BF5A
:107A4000441D0020691500202DE9F047C54D8AB07E
:107A50002A682E4692F849304E2B00F0AF827FD82C
:107A6000372B00F00A834FD8292B00F0958220D8BD
:107A7000252B00F07682272B00F08082232B5AD111
:107A800000F048FF1328064610D8B74D0C272C6885
:107A900000F040FF0023B54907FB031292F808E00D
:107AA000864500F03B8301331C2BF5D1FBF72CF806
:107AB000A3E0332B00F0A982352B00F07A812D2B27
:107AC00039D100F027FFAA4C84F82401FAF740FFCF
:107AD000A4F82E01FAF73CFFA4F82A01FAF738FFC0
:107AE000A4F82C0100F016FF2B6884F825015B79BF
:107AF000082B40F38280FAF72BFFA4F83001FAF745
:107B000027FFA4F8320178E0412B00F084820BD8E3
:107B10003C2B00F0BD803E2B00F0AB80392B0AD10E
:107B200000F0F8FE924CDCE1442B00F0DE8204D839
:107B3000432B00F07B82002078E04A2B00F0A380EA
:107B40004C2BF8D100F0E6FE894C84F86A0100F075
:107B5000E1FE84F86B01FAF7FBFEA4F86C014CE03F
:107B6000D32B66D03DD8CD2B00F0E6811CD8CA2B94
:107B700000F09880CC2B00F04381C82BDBD15479E6
:107B80006408122C92D8002501AFA54255D3224695
:107B90000023784901A89C4255DC0021754B122A2C
:107BA00057D10123B37128E0CF2B00F06481C0F0DE
:107BB000CD81D02B00F0B881D22BBCD16E4B1B787D
:107BC00013F0040419D100F0A5FE694B0228D4BFBC
:107BD00083F8F40483F8F444FBF7F0FEFBF792FF1C
:107BE0000BE0D92B00F09B810BD8D62B00F08881BD
:107BF000D82B00F08F81D42B9DD10020FAF7FEF80E
:107C000013E0EF2B29D006D8DA2B94D1FAF7A0FE97
:107C10005A4B1880F1E7F22BEFD0FA2B8BD1564B51
:107C20001B785B07D8D5FAF76FFF01200AB0BDE8D3
:107C3000F087FAF78DFEA880DFE7FAF789FE27F8CC
:107C400015000135A1E730F8135021F81350013326
:107C5000A1E723F812100132A1E7434C2568FAF797
:107C600077FEA5F85A002468FAF772FEA4F85800C7
:107C7000C3E700F04FFE3E4C84F8740100F04AFE6A
:107C800084F87301B9E7FAF763FE394B9881B4E7DA
:107C9000354C256800F03EFE287023681878FEF702
:107CA000B3FAAAE7304C002523681B78022B6DD16C
:107CB000DFF8D090DFF8D080314F266800F02AFE40
:107CC00009F0ACFC494609F0B5FD05F1080A46F893
:107CD0002A00266800F01EFE05F10A0306EB830663
:107CE00009F09CFC414609F0A5FD7060266800F093
:107CF00011FE09F093FC394609F09CFD05F10E0ACE
:107D00000135032D46F82A00D7D11E4F072D2668CE
:107D100019D100F0FFFD09F081FC394609F08AFD18
:107D20007064266800F0F6FD09F078FC394609F029
:107D300081FDB064266800F0EDFD86F84C00013549
:107D40000A2DE3D159E700F0E5FD2E447070266856
:107D500000F0E0FD2E44F072266800F0DBFD2E44BA
:107D60007075ECE7A01D00208415002044AA0108CE
:107D7000A00F0020C41E002069150020460000202E
:107D800000007A44000020410000C842266800F04C
:107D9000C1FD2E447070266800F0BCFD2E44F072C8
:107DA000266800F0B7FD2E4401350A2D7075EDD11F
:107DB00023E700F0AFFD0B2804463FF677AECF4B2C
:107DC0001D6800F0A7FD03283FF670AE062303FBF5
:107DD000045484F8CE0000F09DFD84F8C90000F042
:107DE00099FD84F8CA0000F095FD84F8CB0000F0FE
:107DF00091FD84F8CC0000F08DFD84F8CD00FCE608
:107E00005379092B7FF752AEBD4C266800F082FDF6
:107E10003070266800F07EFD707000F07BFD6428F5
:107E2000A8BF64202368187100F074FD6428A8BFFF
:107E300064202368587100F06DFD2368987100F08C
:107E400069FD642828BF64202668F07100F062FD97
:107E5000B070266800F05EFDF0702668FAF778FDD5
:107E60002B6870815B790A2B7FF7C7AE246800F01E
:107E700051FD2072C1E6FAF76BFD6FF4AF64031990
:107E80009BB2A04CC62B98BFA4F82A01FAF760FD5C
:107E9000A4F8D000FAF75CFDA4F8D200FAF758FD78
:107EA000A4F8D400FAF754FDA4F86C0100F032FDF8
:107EB00000F030FD00F02EFD00F02CFD84F81901DB
:107EC00000F028FD84F8260100F024FD8B4B1D688E
:107ED000FAF73EFD00EB80004000A5F8560000F0E8
:107EE00019FD84F80E0100F015FD84F8120100F070
:107EF00011FD84F8110100F00DFD84F813017CE6FA
:107F000000240835FAF724FD25F814000134082C64
:107F1000F8D172E6FAF71CFDFAF71AFD6DE6FAF7EA
:107F200017FD85F8200068E6774B1B7858073FF56A
:107F300064AEFBF751FF4FE6734B1B7859073FF5D3
:107F40005CAE4FF4C872714B1A8056E66E4B1B78CC
:107F50005A073FF552AE6E4A137843F0040313708C
:107F60004BE60022674B9A60FAF7F2FC0446FAF7F8
:107F7000EFFC04EB0040FBF7CDFC3EE6FAF7E8FC33
:107F8000604CA4F8E800FAF7E3FCA4F8EA00FAF77A
:107F9000DFFCA4F8EC0030E6FAF7DAFC594CA4F860
:107FA0001401FAF7D5FCA4F8160100F0B3FC84F82C
:107FB0001801FAF7CDFCA4F81A011EE6032355793F
:107FC000B5FBF3F5122D3FF671AD002640F6CA0958
:107FD00040F2EE2819274F4CAE4204F10204BFF4E0
:107FE0000CAE00F097FC04F8020CFAF7B1FC48451F
:107FF000A8BF48464045B8BF4046A0F2EE2090FBDF
:10800000F7F0013604F8010CE6E700F083FC3D4B85
:1080100083F82601F1E500243A4D00F07BFC63195A
:108020000134082C83F81C01F7D1E6E500F072FC5E
:108030000023344CA360FAF78BFC0546FAF788FC62
:1080400005EB0040FBF766FC00F064FC84F82401BB
:10805000FAF77EFCA4F8E800FAF77AFCA4F8EA0044
:10806000FAF776FCA4F8EC00FAF772FCA4F8140115
:10807000FAF76EFCA4F81601BFE507255379B3FBA8
:10808000F5F5C5EBC5029B1A13F0FF0F7FF40EAD9B
:10809000EDB2013DEDB2FF2D3FF4AFAD00F03AFC83
:1080A000746A40B294F9023083421CD094F90A30C9
:1080B00083427FF4FBAC0123DB009A1CD4423FF4E3
:1080C000F5AC1C44A070FAF743FCA08000F022FC41
:1080D000A07100F01FFCE07100F01CFC607200F069
:1080E00019FC2072D5E70023E6E74FF480420A4BE3
:1080F0005A61012385F828307FE500BF84150020F0
:1081000058150020A00F0020691500207E150020C2
:1081100080150020D410002000100140137804EBDB
:10812000860484F8793000F0F5FB84F87A0000F0DA
:10813000F1FB84F87B0000F0EDFB296884F87C00FB
:1081400001F17900FAF780FC57E500BF0378994206
:10815000BABF024B33F8110000207047D01D002039
:108160000021F0B5224D0B462C4641F22106421863
:108170002A44127E83EA02230922013A07D013F42B
:10818000004F4FEA430318BF73409BB2F5E701313C
:108190001929ECD100F1190100F11A0521442544F7
:1081A0000E7E297E01EB062189B299421FD14FF440
:1081B000AF6694F839700138D5B2BD4202F10102C0
:1081C00012DA00EB4201C9B263180131214493F87D
:1081D00018E00B7E03EB0E239BB273431B1303F5D6
:1081E000487324F81530E7E7012384F83A30F0BDEE
:1081F000D01D002003788B420BD9074B89001A78D9
:10820000064B0B44D86B02B1400800F5777080B282
:1082100070470020704700BFCC140020D01D002004
:1082200007298FBF0020034B03EB8101C86E80B28A
:10823000704700BFD01D0020034B03EB4101B1F894
:108240008C00C008704700BFD01D002008B5084B47
:1082500003EB8101D1F8AC0009F0E0F9054909F020
:1082600035FA054909F02AF909F032FC80B208BD57
:10827000D01D00200000203F00005C44024B03EBB7
:108280004101B1F8F4007047D01D0020024B03EB10
:108290004101B1F818017047D01D0020024B03EBDB
:1082A0004101B1F818017047D01D0020002070472F
:1082B00070B5054600F090FC2E4CD4F83031C4F86F
:1082C0003001C31AB3F5FA5F82BF002384F834315A
:1082D00084F8353194F8343123B9A12D04BF01223B
:1082E00084F8352194F835212AB1E218EDB2013332
:1082F000157684F8343194F8345194F83631AB4221
:108300000AD194F83731052B07D0062B08D000236B
:1083100084F8353184F8343170BD0020FFF720FF38
:10832000637E1E2BF3D100200246013DC3B2AB4257
:1083300018DA092123441B7EDBB2013911F0FF0159
:108340000DD082EA0306F60745BF83F01803C3F396
:1083500047035B0843F08003C2F34702EDE70130B7
:108360001A46E3E725442B7E9A42D0D10320FFF73B
:10837000F7FECCE7D01D002010B5044600F02CFC21
:1083800041F288310D4BE4B2D3F83821C3F83801FB
:10839000821A8A4284BF002283F83C2193F83C2150
:1083A0000F2A03EB02010CBF0122013281F83D418B
:1083B00014BF83F83C2183F84D2110BDD01D00204F
:1083C00010B5044600F008FC41F288310D4BD3F89B
:1083D0005021C3F85001821A8A4284BF002283F8D8
:1083E000542193F85421142A03EB02010CBF0122FB
:1083F000013281F8554114BF83F8542183F86A2172
:1084000010BD00BFD01D002010B5044600F0E4FBF5
:10841000254BD3F86C21C3F86C01821AB2F57A6F40
:1084200084BF002283F8702193F870214AB9A82CE8
:1084300038D183F87121A3F87221991881F8754118
:1084400006E0022A02D183F87441F6E7242AF4D91F
:1084500093F8741101320231D2B249008A4283F892
:10846000702116DA082241F22101B3F87201E4B258
:1084700080EA042010F4004F02F1FF324FEA40007E
:1084800018BF484012F0FF0280B2F3D1A3F8720186
:1084900010BD01318A4201BF002283F87021012200
:1084A00083F8712110BD00BFD01D002010B5044617
:1084B00000F092FB40F6AC510E4BD3F89C21821A8F
:1084C0008A42C4BF002283F8A02193F8A021991802
:1084D00081F8A1411AB90F2C0BD1C3F89C010132CC
:1084E000D2B2192A83F8A0210CBF0122002283F8FE
:1084F000BA2110BDD01D002040F2AD1340F6FF722E
:108500004343B3FBF2F30A4A13800A4B1A681E2353
:1085100011784B4344F6FB7100FB03105378C3EB17
:108520000333B0FBF3F09378B0FBF3F080B2704705
:108530009C1D0020941D00202DE9F74F7A4C94F8E3
:10854000BC3104EB4303B3F8CC81784B1FFA88F8B5
:10855000A3F80080B4F9DA310A2B1CBF002384F899
:10856000D83194F8D831002B61D1714B4FF0974935
:10857000C4F8DC31C4F8E4314FF07E53C4F8E8317C
:108580006C4B4FF0000AC4F8EC316B4B4FF07C574A
:10859000C4F8F03140F2DC53C4F82C321023A4F8B4
:1085A0002A321823654D664AA4F82832C4F8E0211F
:1085B000EE1805F1300B4946286909F087F8514655
:1085C000019009F021FA019B3946002800F0A380B0
:1085D000184608F071FF09F0EBFAC6E908014946B0
:1085E00055F8040F09F072F85146019009F00CFAA1
:1085F000019B3946002800F09280184608F05CFF85
:1086000009F0D6FAE6E902015E45D4D10A23A4F8BE
:10861000DA31A8F2DC531B04C4F84832C4F85432EF
:10862000C4F84C32C4F85832012384F8D831434B93
:10863000D4F82CA2B4F92A52A8EB0A005A6A00FA1C
:1086400005F14A43186A4FEAE179D4F8487200FB11
:108650000922C4F84812A0FB0101D4F85462114465
:108660005A6CD3F8408072434FEAE67908FB09223E
:10867000A8FB06899144DA6AD4F858C27A43B0EB71
:108680000800C4F858629E6A61EB09014FEAE77975
:10869000D4F84CE206FB0922C4F84C72A6FB07672B
:1086A0001744DA6C36180CFB02F2986C4FEAEC793E
:1086B0004F4100FB0922A0FB0C01301A7646114401
:1086C00067EB0101F7171E6B5B6BC4F850E20EFB02
:1086D00003F306FB0733A6FB0E671F448019C4F89B
:1086E0005CC2B4F92822794108F064FE01236A1EB5
:1086F0009340C4F85402C01841EBE3712A4608F0D5
:1087000059FE10EB0A0080B2FFF7F6FE0D4B188001
:1087100003B0BDE8F08F184608F0D0FE5BE71846BE
:1087200008F0CCFE6CE700BFD01D0020901D00209B
:1087300056157D396350FABF0CE0743FA81F002026
:108740005615FD398E1D0020F8B53C4C0546B4F891
:108750006032322B4ED1D4F864321A88A4F86822E1
:108760005A889B88A4F86A22A4F86C320388A4F87B
:108770006E324388A4F8703200231946304AD4F888
:1087800064E202F10C06B4F860029F00322808BFD0
:1087900042F8231036F913C0D05926F8131060445C
:1087A000D0512EF813100133032BECD1B4F8603202
:1087B000012B19D14FF0000284F88622214A0C20A7
:1087C000137000F0C7F9D4F86432B4F868221A8044
:1087D000B4F86A225A80B4F86C229A80B4F86E32E7
:1087E0002B80B4F870326B80B4F86032013BA4F88F
:1087F000603201E0002BBFD1134B1A78E2B10022A6
:1088000032201A70D4F87432D4F8641293FBF0F367
:108810000B80D4F8783293FBF0F34B80D4F87C32A1
:1088200093FBF0F3094800881B1A8B802A806A802A
:10883000BDE8F840FBF7C6BAF8BD00BFD01D002068
:10884000442000207A1500207B15002048000020DD
:10885000114BD3F8883203EB4002117E29B1022973
:108860000DD00E4B33F810007047022805D90328AD
:10887000F7D10B4A1268D2040AD5D8897047507EC6
:1088800000EB800000EB800000F2EE2080B2704729
:108890004FF49660704700BFD01D0020D414002014
:1088A000D014002008B500F097F90222064B83F897
:1088B0009022064AC3F88C021268C3F89C22012257
:1088C00083F8B52208BD00BFD01D00201C15002074
:1088D00008B500F081F90222074B00F5B71083F8C4
:1088E0009022D3F89C2200F5587002F2DC52C3F8B3
:1088F0008C02C3F89C2208BDD01D0020044A536896
:1089000023B192F90020824200D11847704700BF7E
:1089100088200020034B1B68DA79511CD97113445D
:10892000187A7047A01D002010B50446054B21465B
:10893000986803681B689847034B1B689A795440F2
:108940009C7110BD88200020A01D002010B5044699
:10895000C0B2FFF7E9FF200ABDE81040E4E710B518
:10896000044680B2FFF7F2FF200CBDE81040EDE7AF
:10897000034B01469B681A6818461268104700BFEF
:1089800088200020F7B5044619480E4690F900509B
:108990001146A5421A469DF824E09DF8203007466E
:1089A00016D090F90C00A0421FD000201BE0114807
:1089B000CDF800E0FEF7A0FAA8B10C2303FB057385
:1089C00004711E7258600EE0CDF800E00A48F1E72D
:1089D00000250C2000FB0570007A0028E5D1002C52
:1089E000E5D0012CF0D003B0F0BD0125F1E700BFC8
:1089F000700F0020003801400044004070B5002591
:108A00000C490D4A0B7B1268012B05DD05B10B7378
:108A1000002070BD2346F7E75C1CDB00D618B68843
:108A2000E4B206424FF00105F4D002330C73D018C3
:108A300070BD00BF88200020C41D00200022014B13
:108A40001A73DBE7882000202DE9F04100240A2773
:108A50004FF47A761A4D82781FFA82FEA4EB0E0349
:108A60001BB2002B29DDC2F16402D2B203FB03FC6E
:108A700090F80380524308FB0CFC9CFBF2F2C8F117
:108A800064084244534393FBF7F30EEB8E0E03EB63
:108A90004E031BB26B800A88B1F802E00A34AEEBD9
:108AA000020E03FB0EF393FBF6F3A4B21344782CEF
:108AB00025F8023FCFD1BDE8F08108BF0122D5E7FC
:108AC0009420002030B5002340F6C4150A4C072B33
:108AD00010D003FB03F2A2F1190142784A4302F6D7
:108AE000C4125A4301784A4392FBF5F224F813204A
:108AF0000133ECE730BD00BFAE2000200F4B043047
:108B000033F9102040F633039A42A8BF1A461923BE
:108B1000B2F5617FB8BF4FF461720878584300F234
:108B20008330904208DA4878584300F2833090420C
:108B3000B4BF00200120704700207047D4140020EB
:108B40000022034B83F834209A639A871A64704793
:108B50008820002070B408B970BCF1E70E4A0023E9
:108B60000C25114605FB03F4A65C864209D10B4B8C
:108B7000186C50B1224455784278954205DB70BCA0
:108B800070470133102BEDD1F9E70022214419641D
:108B90009A879A63F3E700BF94AB0108882000200E
:108BA0004000142870B4A8BF142000230226142506
:108BB000084A02F144015E540233CC18984204F88A
:108BC000015CF8DC1344FF2283F844200F2070BCC2
:108BD000C0E700BF8820002010B50A490A480A688B
:108BE000846800BF0B689A42F9D14FF47A70074B42
:108BF000D96D00FB01F31B1BB3FBF1F300FB02304B
:108C000010BD00BF1C15002010E000E088200020EF
:108C100038B50446FFF7E0FF0546FFF7DDFF401BD0
:108C2000A042FAD338BD10B5044604B910BD4FF4C4
:108C30007A70FFF7EDFF013CF7E706462DE987481C
:108C4000294C0B27013FFCD04FF01E0905254FF0A2
:108C5000020806F0400A06F0200B00E00025BAF1F9
:108C6000000F03D0E36883F40043E360BBF1000F1F
:108C700003D0E36883F48043E36016F0020218BF78
:108C8000E36848461CBF83F40053E3600192FFF79A
:108C9000CAFF019ABAF1000F03D0E36883F40043DE
:108CA000E360BBF1000F03D0E36883F48043E3602B
:108CB0001AB1E36883F40053E3604846FFF7B3FF5B
:108CC0007DB1013DCBD14FF4FA70FFF7ACFF4FF00F
:108CD0009609B8F1000FC1D14FF47A70FFF7A3FFE6
:108CE000B0E708F1FF38F4E700100140024A1368CA
:108CF00001331360704700BF1C1500200920FDE5FB
:108D00002820FBE5174B2DE9F0410746B3F860003A
:108D100090460C4608F082FC134908F0D7FC064642
:108D2000404608F07FFC114908F0D0FC01464FF0A6
:108D30007E5008F07FFD314608F0C0FB014630460A
:108D400008F078FD256806462946384608F0B4FB49
:108D50000146304608F0BAFC294608F0AFFB206017
:108D6000BDE8F08188200020BD378635DB0FC94083
:108D70002DE9F84F244C00252746244E94F8948082
:108D8000E8B2404531D3224B1B685B0339D500263E
:108D90004FF0500A33464FF0280BB146F4B2444529
:108DA0002FDAA4003A19526E55689D4215D0284614
:108DB000FEF70EF8EFF312838AF31288AA8C0BFBEE
:108DC000007092B20132C0F8BC20AA8ADBB292B223
:108DD00042F00102AA8283F311883C44636E01369B
:108DE0001B68A3F800902B46D8E704EB80035B6E6A
:108DF0002BB10B2803DCDB6836F8101098470135DF
:108E0000BCE7BDE8F88F00BF882000203E0F00209F
:108E1000D014002010B4184A137813F0010F03F097
:108E2000040003D11549096801291DDC14490C7897
:108E3000D4B1F0B9134C246864011AD49C0713D43C
:108E40004FF47A7043F0040313700F4B10BC1B886F
:108E50004B800E4B1A680E4B93F8743100FB0323C2
:108E600005204B60FFF776BE18B9012010BCFFF754
:108E700097BE10BC704700BF691500206C1500201C
:108E8000C421002060150020781500201C1500204A
:108E9000A00F002008B5114A1378590705D523F013
:108EA000050304201370FFF755FE0D4B1B7813B11B
:108EB00000220C4B1A7000230B4901200B724B72DD
:108EC0008B7240F2B631094A107050705160084AF6
:108ED00003201360BDE80840FAF7E1BC69150020E3
:108EE000C01D002010000020C42100204C000020E4
:108EF000481D002008B50C4B1B8813B90B4B188874
:108F000070B10020FAF7D6FC094B1B88DB0705D4AB
:108F1000084B1868003018BF012008BD012008BDAB
:108F2000FAF7BDFCF0E700BF7E15002072150020A7
:108F300070150020B817002070B44C1E4C2C2DD892
:108F4000DFE804F03C3C3C3C2C2C2C2C27273C2715
:108F500027272727272727272727272C2828282898
:108F6000282828283C27272727272C27283E3C2C41
:108F70003C28283E2C2C2727273C3C3C3C3C273CCB
:108F80003C273C2C2C2727272C2C2C2727273C2818
:108F90003C001AB144698569AC4202DB002070BC18
:108FA000704704EB44050669AD0001344461701953
:108FB000F5D071554260836070BC7047002AEDD0D7
:108FC000002BEBD044698569AC42E7DAE9E700BFE2
:108FD0002DE9F047C368B2F1000A04460E461A783C
:108FE00015BF4FF01E094FF01B094FF01D084FF041
:108FF0001A0814BF1C2719270D4618E0562A1FD03F
:109000004B2A24D0442A2DD15A78782A27D14C21B2
:10901000226B02331132E3602263002320461A469A
:10902000FFF78AFF2860C8B1E368051D1A78722A25
:10903000E4D1226B01330932E36022633946ECE765
:10904000226B01330932E36022634146E5E7226B7C
:1090500001330632E36022634946DEE705462846CF
:10906000BDE8F087BAF1000FF9D1462AF7D1B54231
:10907000F5D01D201E211C2207E01B2B0BD0192B25
:1090800000D132700436B542E9D0366833781A2BF5
:10909000F3D13070F6E73170F4E700BF10B4C36865
:1090A0000A461C78522C0DD04F2C02D0084610BC1A
:1090B00070472021046B033404630133C36010BC88
:1090C000002339E7046B1F2102340463F5E700BF76
:1090D000002A4DD070B505460E4614462378013B54
:1090E0004C2B2BD8DFE803F03636363F2A2A2727C9
:1090F0003636363636363636363636363636362A1C
:10910000363636363636363636362F2F36362A3619
:109110003636362B363636362A2736363636363615
:10912000363636363636362A2A362B2B2B2B2A362F
:10913000363636363600A468002CCFD170BD646850
:10914000002CCBD1FAE762681378052B03D1336882
:1091500001333360626831462846FFF7B9FFA468DF
:10916000002CBBD1EAE72B6801332B606268F2E781
:10917000704700BF7AB32DE9F0410D4604464FF029
:109180000008D0F80011AF1809E00B46BD4201F10C
:109190000101C4F80011E65484F8046119D0FF29D4
:1091A00015F8016BF1D1D4F80831D4F80C2184F80A
:1091B000FF802046984701210023D4F82421BD4296
:1091C0000A44C4F82421C4F80011E65484F8046168
:1091D000E5D1BDE8F081704770B4026811786E295E
:1091E00018D0A1F13003092B1ED80026002301322C
:1091F00003EB8303026001EB43041178A4F1300315
:10920000A1F13005092DF2D90EB1C4F13003184691
:1092100070BC7047531C03605178A1F13002092AD9
:1092200002D81A460126E1E70023F0E74369826984
:1092300010B593420FDA03EB430201699200013348
:109240008C18436105D041230C308B54FFF7C4FFC9
:109250006060204610BD0024204610BD10B5C368D4
:1092600004461A785F2A0DD06E2A0FD00C30FFF713
:10927000B3FF01300AD4E3681A785F2A06D10133BC
:10928000E36010BD01330020E36010BD4FF0FF30FC
:1092900010BD00BF38B5C3681A78542A01D0002029
:1092A00038BD0133C3600446FFF7D8FF051EF6DB67
:1092B000A26A6369A16901328B42A262EFDA03EB11
:1092C00043022169920001338818636102D00523AB
:1092D0008B54456038BD00BF70B504460C30FFF7B5
:1092E0007BFF061E4DDDE56863685B1B9E422BDC41
:1092F000A268AB195207E36004D5AA5D242A04BF13
:109300000133E360092E0CDD08221F4928460CF0CA
:10931000A1FC30B92B7A2E2B19D05F2B17D0242B20
:1093200015D06369A26993420EDA03EB4302216907
:10933000920001338818636106D02DB100238B544D
:1093400045608660E06270BD0020E06270BD6B7AAF
:109350004E2BE6D1236B6269A16916339E1B8A42AC
:109360002663F1DA02EB420321699B000132C8183F
:109370006261EAD000261525044ACE548560426019
:10938000E3E7002070BD00BF38B8010844B8010809
:1093900070B5C36804461A78C66A422A0D460FD1D2
:1093A0000133E3602046FFF797FF2A4603464B212F
:1093B0002046FFF7C1FDE36805461A78422AEFD040
:1093C000E662284670BD00BF2DE9F0410546C06841
:1093D0000378532B02D00020BDE8F081431CEB60E2
:1093E0004278A2B1831CEB6042785F2A5AD10023F5
:1093F0002A6A9342EFD2AA6AE9690132AA6251F855
:109400002300BDE8F081A2F14103192B4FD9AB68CD
:1094100003F00803002B14BF0124002401D100290C
:1094200069D1464B742103F1C40003E01C3383422D
:10943000D1D219788A42F9D15E69002E7BD06A694F
:10944000A9698A4263DA02EB4207D5F810E0BF004F
:1094500001321EEB0700D3F818806A6106D04FF086
:10946000180C0EF807C04660C0F80880E862002CAF
:109470004AD0DE681C692B6B914223442B6341DD8B
:1094800002EB420329699B000132C8186A6103D0CC
:109490001822CA5446608460EB681B78422B38D08F
:1094A000BDE8F081A2F13004E3B2092BABD8002172
:1094B0000DE0303B99428ED8E9680A78481C1AB111
:1094C000E8600A785F2A14D01946A2F13004E4B2A9
:1094D00001EBC103092CA2F1410002EB8303E8D99F
:1094E00019283FF678AF01EBC10302EB8303373B4A
:1094F000E0E701337CE7EB681B78433B012B98BF27
:1095000001248EE70020C7E75E689C68B3E700206F
:10951000ACE701462846FFF73BFF00283FF45BAF6E
:109520002B6A6A6A9342BBDAE9695A1C41F8230044
:109530002A62BDE8F081A9696A6998E7B0AC0108C0
:1095400038B5044629B9C3681A7832B15A1CC260CA
:109550001978682919D0762901D0002038BD04F186
:109560000C052846FFF738FEE3681A785F2AF4D125
:109570000133E3602846FFF72FFEE3681A785F2A7D
:10958000EBD101200344E36038BD04F10C00FFF788
:1095900023FEF2E7D0F810319BB10A685B68002A1D
:1095A0009B6809DB23B907E042B19B68013A1BB114
:1095B00019782F29F8D00023184670475B681846A1
:1095C00070470122C0F81821F6E700BF002941D0FA
:1095D00038B505460C4623784B2B27D8DFE803F037
:1095E0002E26262626302E2B2B26262626262626F7
:1095F00026262626262626262E2626262626262603
:10960000262626262626262E262626262E262626EA
:10961000262E2B26262626262626262626262626DD
:109620002E2E2626262E2E2E26262E2E6168284603
:10963000FFF7CCFF18B9A468002CCCD1002038BDAE
:10964000211D2846FFF7A6FF0028F7D003782F2B0F
:10965000F4D138BD00207047F0B5154652684B1C58
:10966000AC681344A34283B00E46074613D8EC6897
:109670000CB103B0F0BD95E80900324639461844F4
:1096800005F0A6FF2B686A6833449C546B681E443F
:109690006E6003B0F0BDEA68002AEAD11CB9022B63
:1096A0004FF0020402D96400A342FCD82146286886
:1096B0000CF0F6FB10B12860AC60D8E70190286888
:1096C0000BF0D8FF0122019BEA602B606B60AB605E
:1096D000CFE700BF2DE9F04188B00A4604461B4998
:1096E00001A80CF0FBFD01A80CF01EFE50B301AD6B
:1096F0004FF00008D4F800112F1809E00B46BD42C6
:1097000001F10101C4F80011E65484F8046119D094
:10971000FF2915F8016BF1D1D4F80831D4F80C21E8
:1097200084F8FF802046984701210023D4F82421A3
:10973000BD420A44C4F82421C4F80011E65484F858
:109740000461E5D108B0BDE8F08100BF5CB8010854
:1097500000222DE9F04FC36883B01D7804468D4286
:10976000019200F0C6818846DFF89C9401AE23E0A8
:10977000662A4CD0A2F13001092900F21782204656
:1097800001F0FEFA0546002800F07081E3681B78BE
:10979000492B00F0928067632A4600232E21204641
:1097A000FFF7CAFB306000285BD0E36800F10806D1
:1097B0001A78424500F007810125676B65631A78C6
:1097C0004C2A47D0542A51D0732AD1D15A78722AC0
:1097D00000F0E280702A00F0FD80204601F010FACF
:1097E0000546002800F042812B78312B43D0322BE4
:1097F0005CD0332B7BD1E3681A785F2A40F0C180BC
:109800000133E36045212046FFF7A2FFBCE05A7810
:10981000702AE2D19A1CE2609A78542A69D02046D4
:10982000FFF71CFD6FF00043984260D0431C5ED0F0
:1098300001306369A269934259DA2269591C03EB2A
:10984000430312EB8305616151D0062102F8231016
:109850006860A0E7204601F0E1FE05466763002D41
:109860009AD10025284603B0BDE8F08F2046FFF7C7
:1098700011FD0546F2E7D5F804B0236BDBF80820AC
:10988000DBF800A0023A134423635046494605F032
:1098900015FF002800F0E680DBF80C30032B26D8FB
:1098A000DFE813F02B0035013300A5006B68032BB4
:1098B0001DD8DFE803F022661C1C204600F0FEFBEA
:1098C0002A46034604212046FFF736FB0546C5E736
:1098D000742A82D15B786C2B7FF47FAF204600F036
:1098E000AFFDE36805465A78002A40F06981676356
:1098F000B7E70333E36000209BE72A4600233521C6
:109900002046FFF719FB0546A8E7BAF1000FEED095
:109910006B681B685A78632A00F0D2809AF800308E
:10992000662B00F0EF80204600F070F98346B149C5
:10993000504605F0C3FE002800F09D80AE49504619
:1099400005F0BCFE30B15046AC4905F0B7FE00282A
:1099500040F08380204601F013FAE36882461B78CA
:10996000492B00F0E98053465A4638212046FFF73C
:10997000E3FA2A46034637212046FFF7DDFA05467B
:109980006CE7204600F042F903462A46362120467D
:10999000FFF7D2FA054661E70233E360204600F0A4
:1099A0004FFD8246204601F0EBF9E36883461B78C1
:1099B000492B00F093800346294652462046FFF784
:1099C000BBFA05464AE7019D01332846E36003B030
:1099D000BDE8F08F0233E360204600F017F9002362
:1099E00002464A212046FFF7A7FA054636E7BAF1B4
:1099F000000F3FF47CAF8249504605F05FFE00281F
:109A00003FD09AF80030662B00F0BD806E2B7FF4BB
:109A10006EAF9AF80130772B02D0612B7FF467AFDD
:109A20005F212046FFF794FE8246204600F008FDA5
:109A3000E36883461A78452A00F0A180702A00F076
:109A4000A680692A7FF453AF5B786C2B7FF44FAF0D
:109A5000204600F0DBF803461FE0204600F0D6F871
:109A6000824680E7204600F0EBFC8DE728466763DE
:109A700003B0BDE8F08F45212046FFF769FE82461E
:109A800071E7204600F0C2F88246204600F0BEF89A
:109A90008346204600F0BAF803465A463B2120464A
:109AA000FFF74AFA524603463A212046FFF744FAA6
:109AB0002A46034639212046FFF73EFA0546CDE601
:109AC0001B78A3F16302012A03D9723B012B3FF6F5
:109AD00025AF204600F0B4FC834628E7204600F07E
:109AE000EDFA5A46034604212046FFF725FA0346BD
:109AF00062E70133C3602E21134603B0BDE8F04F87
:109B0000FFF71ABA204601F07BF883460FE7BAF157
:109B1000000F3FF436AF9AF80030702B17D06D2B42
:109B200015D05046374905F0C9FD00287FF429AF0C
:109B3000204600F065FA27E7204600F0BFFA5246BB
:109B4000034604212046FFF7F7F982460BE79AF80F
:109B500001209A42E5D1E3681A785F2A23D0504663
:109B6000284905F0ABFD00283FD0204600F04EF814
:109B700003461A4638212046FFF7DEF904E7013391
:109B8000E360002389E7204601F03AF87CE75A7841
:109B9000692A7FF4ACAE0233E36045212046FFF72B
:109BA000D7FD034679E70133E360BAE76F2A15D0A2
:109BB000692A7FF48DAE5A786C2A7FF40EAE0025A8
:109BC0000233E36045212046FFF7C2FD2A460346E3
:109BD00030212046FFF7B0F905463FE65A786E2A55
:109BE0007FF4FBAD0233E360C9E5204600F008FADC
:109BF0000346BEE764B8010868B801086CB80108FC
:109C000070B8010860B8010868BD0108C1680B7828
:109C10004C2B00F08780542B00F08680732B2DE9AD
:109C2000F041044637D0662B12D0A3F13002092A46
:109C300000F2B881204601F0A3F8054600286DD057
:109C4000E3681B78492B00F088802846BDE8F08146
:109C50004B78702B39D0204600F0D2FF0546002803
:109C60005CD00378312B61D0322B25D0332B55D1EA
:109C7000E3681A785F2A40F0B4810133E36045213C
:109C80002046FFF765FD03462A462046BDE8F04121
:109C90003621FFF751B94B78722B69D0702BDAD18E
:109CA0000231C160FFF7B2FF002302464A2120467D
:109CB000BDE8F041FFF740B94368032B2ED8DFE839
:109CC00013F0710090012D002D008B1CC3608B7868
:109CD000542B63D0FFF7C2FAC34333F000431DD0C7
:109CE00001306369A269934218DA03EB43022169E8
:109CF000920001338D186361A7D006238B546860EE
:109D0000A3E7742BA7D14B786C2BA4D100F098FB60
:109D1000E16805464B78002B40F04E81002528462F
:109D2000BDE8F08101F07ABCFFF7B4BA4768236B55
:109D3000BA683E68023A134423633046AA4905F0E4
:109D4000BDFC002800F0AB80FF68032FE6D8DFE8F9
:109D500017F02900FF0071003100204600F0AEF935
:109D60002A46034604212046BDE8F041FFF7E4B847
:109D70000231C16000F064FB0546204601F000F8A6
:109D8000E36806461B78492B00F0AE8003462A465E
:109D90002046BDE8F0410121FFF7CEB80331C16094
:109DA00000209EE72A462046BDE8F04100233521E9
:109DB000FFF7C2B8002EB1D08C49304605F07EFCCA
:109DC000002871D03378662B00F0B2806E2BA5D1BD
:109DD0007378772B01D0612BA0D15F212046FFF74C
:109DE000B7FC0646204600F02BFBE36807461A78CE
:109DF000452A00F09980702A00F09E80692A8DD152
:109E00005B786C2B8AD12046FFF700FF03463A4669
:109E10003B212046FFF790F8324603463A21204680
:109E2000FFF78AF82A46034639212046BDE8F0416B
:109E3000FFF782B8002E3FF471AF6B681B685A7849
:109E4000632A44D03378662B59D02046FFF7DEFED4
:109E500007466749304605F031FC90B36549304606
:109E600005F02CFC28B13046634905F027FC00289A
:109E70004AD1204600F084FFE36806461B78492B50
:109E800047D033463A4638212046FFF755F82A4650
:109E9000034637212046BDE8F041FFF74DB8204684
:109EA00000F0CEFA0346EFE62046FFF7AFFE064687
:109EB0002046FFF7ABFE07462046FFF7A7FE034606
:109EC000A5E745212046FFF743FC0646D9E71B7866
:109ED000A3F16302012A02D9723B012BB2D82046BA
:109EE00000F0AEFA0746B4E7204600F0E7F8324645
:109EF000034604212046FFF71FF8034647E72046A4
:109F000000F07EFE0746A4E72046FFF77FFE0646E8
:109F1000B7E7204600F0D2F8324603460421204637
:109F2000FFF70AF80646ACE70133E36000236EE76B
:109F3000204600F065FEBAE75A78692A7FF4EEAE53
:109F40000233E36045212046FFF702FC03465EE74B
:109F5000002E46D03378702B15D06D2B13D00027F0
:109F60003046264905F0AAFBB8B12046FFF74EFE61
:109F70000346002F3FF488AE1A4638212046FEF7EC
:109F8000DBFF034680E672789A42E8D1E3681A78EC
:109F90005F2AE5D10133E360E1E7204600F030F8C5
:109FA0000346E6E76F2B15D0692B7FF4AAAE4B78FA
:109FB0006C2B7FF450AE00250231E1602046452134
:109FC000FFF7C6FB2A46034630212046BDE8F04194
:109FD000FEF7B2BF4B786E2B7FF43DAE0231C1600D
:109FE00028E60027C1E700BF68BD010870B8010876
:109FF00064B8010868B801086CB8010860B80108C5
:10A000002DE9F041C26882B013780446452BC76A37
:10A0100049D00021012602AD45F8041D493B0F2B14
:10A020003AD8DFE803F03535391A39393939393951
:10A030003939393939080132D4F83480E2602046A0
:10A040006663FFF7E3FDE368C4F834801A78452AB5
:10A0500026D0002002B0BDE8F081204601F0DEFAF3
:10A060000028F6D0024600232F212046FEF764FF89
:10A07000286000F108050028EBD0E2681378452B32
:10A08000CCD101980132E260E76202B0BDE8F08114
:10A09000204600F013F8E3E7204600F0D1F9DFE7AF
:10A0A0000133E360DCE700230132C2602F211A464E
:10A0B00002B0BDE8F041FEF73FBF00BFC2681378B1
:10A0C000493B012B02D80132C26099E7002070475A
:10A0D0002DE9F043C26885B0137805464E3B0C2B42
:10A0E00070D8DFE803F01E6F6F6F6F5B6F176F6FD5
:10A0F0006F6F070001320021C26000F0B1FFEB6812
:10A1000006461978452900F099800022104605B0CE
:10A11000BDE8F08300F034FE0246104605B0BDE80D
:10A12000F0830132C26003A90122FEF751FF81468C
:10A130000028EAD000212846FEF7B0FF002780461D
:10A14000EA68BC4E1478002C00F0EF80442C00F03C
:10A15000D180A4F13003DBB21C2B40F2A880A4F123
:10A160006103192B40F2A880552C00F0E580532C98
:10A1700000F0CC80492C00F0E180542C00F01C81D0
:10A18000452C00F042814D2C40F0CF80002F00F094
:10A19000CC80531CEB6054781A46D4E75378742B68
:10A1A00031D00021FFF710F9EB68024619784929F0
:10A1B000B3D10133EB6028460192FFF721FF019AEA
:10A1C000034617E000F0DCFDEB68024619784929E8
:10A1D000A3D1002A99D0296A686A814295DAEC698C
:10A1E000481C44F82120286219784939012988BF80
:10A1F0000023DED928460421FEF79EFE02461046C3
:10A2000005B0BDE8F0834369816902328B42C260C8
:10A21000C0F2A8800024284600F0B2FD2246034682
:10A2200001212846FEF788FE296BEB68033129637C
:10A230001978024649297FF470AFCAE75A1CEA60D0
:10A240005978732900F0A080642900F0B98028466D
:10A25000FFF73EFF0446002879D00378452B00F035
:10A260009180472B00F08E80EB681A785F2A40F0CF
:10A2700089804FF0FF372846013340F80C3FFEF746
:10A28000ABFF0028FFF641AF7B1C7BD06B69AA694E
:10A2900093425CDA03EB43022969013392006B615C
:10A2A0008B1855D0462088549F605C6050E026FA99
:10A2B00003F3D9077FF553AF284600F061FD7FB364
:10A2C000012103463A462846FEF736FE0746532C40
:10A2D00023D0EA681478452C3FF43BAF2FB32B6AA8
:10A2E000696A8B4221DAE969581C41F823702862B7
:10A2F000147828E75378284603F0DF03542B11D055
:10A3000000F03EFD002FDBD10746E2E701212846A1
:10A31000FFF75AF8002FD3D10746EA68147812E7FE
:10A320000746D4E700F08CF8ECE700221046C9F8A5
:10A33000002005B0BDE8F0832846E1E7002FF4D007
:10A340000132EA602846FFF75BFE0421B9E70023EB
:10A35000324628460221FEF7EFFD0246104605B0C0
:10A36000BDE8F08303EB43020169920001338C18CE
:10A3700043613FF450AF002603202F4B8E54A06062
:10A38000636048E72346E3E79A1CEA609A785F2A0D
:10A3900032D06B69AA699342D9DA03EB4302296987
:10A3A000013392006B618B18D2D000270E24234812
:10A3B0008F549C605860CBE72846FEF76BFFA1E7FF
:10A3C0000233EB602846FEF749FF071EFFF69DAEFD
:10A3D0002846FFF77DFE044600283FF457AF037878
:10A3E000452B3FF453AF472B3FF450AFEB681A783F
:10A3F0005F2A7FF44BAF3EE72846033340F80C3F1B
:10A40000FEF7EAFE0028C4DA7FE6C9F80070002FE4
:10A410003FF47BAEB8F1000F04D0039BCDF80C8065
:10A42000C8F804301378452B7FF46FAE0132EA6030
:10A43000039A72E6FF03081084B8010874B8010893
:10A440002DE9F043C26883B013780446722B58D0CC
:10A45000562B56D04B2B54D0442B00F09F80A3F1A9
:10A4600030014A2900F28A80DFE811F02A012A012E
:10A470002A012A012A012A012A012A012A012A0184
:10A4800088008800880088008800880088000B0207
:10A4900088005201880088004C0160018800880013
:10A4A0008800880088006E012A018601C3018800A7
:10A4B0009401A201D101F30188008800880088007E
:10A4C0002A018800880088008800880088000C0124
:10A4D0000C010C010C010C010C010C010C010C0114
:10A4E0000C0188000C010C010C010C018800880093
:10A4F00088000C010C013E010C010C010C010C0147
:10A500000C01002201A92046FEF762FD0546002845
:10A5100034D0E36820461B78462B34D0FFF790FFF9
:10A52000286058B303781F3B012B30D9019A2AB316
:10A53000236A616A8B4221DAE069591C40F82320C2
:10A54000019D2162284603B0BDE8F0830123456BDD
:10A550004363FFF75BFB656302460023422120460D
:10A56000FEF7EAFC0546019040B1E3681A782AB18B
:10A570005A1CE2601B78452B00F0AA800025284673
:10A5800003B0BDE8F08300F04BFD2860C9E7019AF5
:10A59000436842602A6801922B60C7E75378782BA2
:10A5A000AFD0531CC3605378002BE7D0931CC3601B
:10A5B0005378463B302BE1D801A151F823F000BF7E
:10A5C00099AA00087DA500087DA500087DA50008C2
:10A5D0007DA500087DA500087DA500087DA50008D3
:10A5E0007DA500087DA500087DA500087DA50008C3
:10A5F0007DA500087DA500084DA500087DA50008E3
:10A600007DA500087DA500087DA500087DA50008A2
:10A610007DA500087DA500087DA500087DA5000892
:10A620007DA500087DA500087DA500086FAA00088B
:10A630007DA5000845AA000827AA0008FFA9000870
:10A64000D3A900087DA50008A7A9000885A90008CE
:10A650007DA500087DA500087DA500087DA5000852
:10A660004DA900087DA5000837A900087DA50008B0
:10A670007DA500080BA900084DA500087DA50008D0
:10A68000D5A800086069A569613BBB4903EB83035A
:10A69000A84201EB830380F2318200EB400126697E
:10A6A000890001307518606100F0288227207054FD
:10A6B0006B605968236B01320B44E26023635EE7F1
:10A6C0002046FFF705FD05460190002D3FF456AFEB
:10A6D000236A626A9342BFF651AFE1695A1C41F89E
:10A6E0002350019D22624AE70132E2602046FEF7D4
:10A6F000F3FD0023024628212046FEF71DFC0546F7
:10A700000190E2E7204600F08BFC05460190DCE773
:10A710000132E2602046FFF793FE00230246252126
:10A720002046FEF709FC05460190CEE70132E260C3
:10A730002046FFF785FE0023024626212046FEF72D
:10A74000FBFB05460190C0E70132E2602046FFF7BF
:10A7500077FE0546002800F0BB802046FFF770FE1C
:10A76000002800F0B58003462A462B212046FEF73C
:10A77000E3FB05460195A8E70132E2602046FFF7BA
:10A780005FFE0023024624212046FEF7D5FB054646
:10A7900001909AE70132E2602046FFF751FE002364
:10A7A000024623212046FEF7C7FB054601908CE7B1
:10A7B0005378A3F13002092A05D95F2B03D0413B1E
:10A7C000192B00F2BA8100212046FEF7FDFDE36857
:10A7D00001901B780546492B7FF4D1AE2046FFF748
:10A7E0006DFC2A46034604212046FEF7A5FB0546DC
:10A7F000C0E70132E2602046FFF722FE0023024656
:10A8000022212046FEF798FB054601905DE7204691
:10A81000FEF740FDE668019033780546492B7FF44A
:10A8200054AFA36B002B40F0A08100283FF4A6AEEC
:10A83000236A626A9342BFF6A1AEE1695A1C41F8ED
:10A84000230022622046019DFFF738FC2A4603467A
:10A85000C9E70132E2602046FEF73EFDE368019061
:10A860001B780546492B00F075812046FFF7E8FD6F
:10A87000019B024621212046FEF75EFB0546019022
:10A8800023E7511CE16053785F2B00F03B81303BA4
:10A89000092B00F245810B460133E3601A78303A08
:10A8A000092AF9D96269A069824211DA02EB4200F1
:10A8B0002669800001323518626109D05A1A07D022
:10A8C000002737546960AA601A785F2A00F08781F0
:10A8D00000254FE793785F2B00F07781FEF7A6FC09
:10A8E0000546002D3FF446AFE3681A785F2AEFD1A2
:10A8F0000133E3602046FFF7A3FD2A4603462D21DE
:10A900002046FEF719FB054634E7426983699A42FF
:10A9100080F2F4800C2303FB02F301690132CD18AD
:10A92000426100F0EB802720144AC8546A60236B10
:10A930000833236323E6FFF783FD002302464A2101
:10A940002046FEF7F9FA05460190BEE642698369A2
:10A950009A4280F2D3800C2303FB02F30169013297
:10A96000CD18426100F0CA802720054AC8546A60A9
:10A97000236B1133236302E674AD0108CCAF0108E9
:10A98000F4AF0108426983699A4280F2B7800C23D0
:10A9900003FB02F301690132CD18426100F0AE8081
:10A9A0002720904AC1E7426983699A4280F2A680D3
:10A9B0000C2303FB02F301690132CD18426100F060
:10A9C0009D802720884AC8546A60236B0433236320
:10A9D000D5E5426983699A4280F290800C2303FB9B
:10A9E00002F301690132CD18426100F0878027200F
:10A9F0007E4AC8546A60236B09332363BFE542690A
:10AA000083699A427ADA0C2303FB02F3016901326B
:10AA1000CD18426172D02720754AC8546A60236BF2
:10AA20000A332363ABE5426983699A4266DA0C23F1
:10AA300003FB02F301690132CD1842615ED0272089
:10AA40006C4AD6E7426983699A42BFF697AD0C23F8
:10AA500003FB02F301690132CD1842613FF48FAD6F
:10AA600000240E20644ACC54A8606A6087E54269DD
:10AA700083699A42BFF682AD0C2303FB02F301699E
:10AA80000132CD1842613FF47AAD002404205B4AC4
:10AA9000CC54A8606A6072E5436981698B427ADAB6
:10AAA0002C26006903EB43018900013345186361DB
:10AAB000019546549378303BDBB2092B94BF0123B8
:10AAC00000232B817BD92046FFF7BAFC019B6860ED
:10AAD0005B68002B3FF452AD04F10C00FEF77CFBE9
:10AAE000E268137813B1531CE3601378A3F1730386
:10AAF000B3FA83F3019D5B096B8140E50023019369
:10AB00005B68FFDE00250131E1602046FFF798FC1D
:10AB10002A4603462A212046FEF70EFA054629E674
:10AB20000123656B20466363FFF770F86563054694
:10AB300000283FF4CDAEE368C6E62046FFF7C8FA2A
:10AB40000546019000283FF419AD0378182B7FF4D7
:10AB5000BFAD14E52046FFF7B1FA2A4603460421AB
:10AB60002046FEF7E9F901907FE62046D4F81490DC
:10AB7000D4F82080A76A256BFFF7A0FAE268127864
:10AB8000492A0BD02563E660C4F81490C4F82080ED
:10AB9000A762019D99E500231B70FFDE019B002B3E
:10ABA0003FF4ECAC226A616A8A42BFF6E7ACE56921
:10ABB000511C45F82230019A0346216213E604F144
:10ABC0000C00FEF709FB019D7DE701230332466B74
:10ABD000C2604363FFF71AF86663054681E61946CB
:10ABE00091E700BFE0AF0108B8AF01087CAF0108F2
:10ABF000A4AF010890AF010890B8010888B8010817
:10AC0000F8B5C36884461F7827B35A1CC2605A78C7
:10AC10001F78002A58D09A1CC260762F044693F8F9
:10AC200001E043D0632F16D1BEF1760F13D1436BF1
:10AC3000856BB3FA83F35B098363FFF701FCA36BB6
:10AC40000246002B52D0002334212046FEF774F92F
:10AC5000A563F8BDBE4643200022274D04E08CBF0B
:10AC600018465A1C82422DD0831A03EBD37302EB91
:10AC7000630319016C5829442678BE42EFD16478E9
:10AC80007445ECD1DCF81430DCF81820934219DA62
:10AC900003EB4302DCF8104092000133A018CCF81B
:10ACA000143013D03123A3544160F8BDAEF1300508
:10ACB000EBB2092BCFD8FEF70FFB6369A2690146FF
:10ACC000934204DB0020F8BD9646C4E7F8BD03EBD1
:10ACD0004302266992000133B0186361F2D0002963
:10ACE000F0D03223B35445608160F8BD3321204653
:10ACF000FEF722F9ACE700BF08B00108002330B529
:10AD0000C26883B00193137843B3452B26D02E2B12
:10AD100024D0044601AD16E04F2B16D02046FFF795
:10AD20008FFBD8B1024600232E212046FEF704F9FE
:10AD3000286098B1E26800F10805137843B1452B0B
:10AD400006D02E2B04D0522BE6D15378452BE5D1DB
:10AD5000019818B1836823B103B030BD002003B05F
:10AD600030BD426811782729F6D15268117C092933
:10AD7000F2D15168226B521A22634360ECE700BFA4
:10AD8000F8B5C16804460B78A3F13002092A20D92E
:10AD9000A3F16102192A25D9A3F14302012A2CD972
:10ADA0004C2B00F08880552B33D14B786C2B33D053
:10ADB000742B2ED14B1CC3604B78742B5AD0422B72
:10ADC0004FF000050CD129462046BDE8F840FEF7BB
:10ADD000DFBAFEF781FA0546E3681B78422BF2D012
:10ADE0002846F8BDFFF70CFF054618B10378312B54
:10ADF00000F0B280E3681B78F0E7C56A25B12A78D5
:10AE0000002A6CD0182A6AD0432B00F0BF80442B54
:10AE10006FD000252846F8BD4B1CC3604B786C2BC7
:10AE2000CDD10231C160FFF769FF0646F0B1E2689B
:10AE30001378452BC3D10132E2602046FEF70EFAAB
:10AE4000002813DB6369A26993420FDA03EB430224
:10AE50002169920001338D186361CBD045238B5457
:10AE60006E60A860236A626A93421CDBE368002577
:10AE70001B78B3E70231C160FEF7F0F90028F5DB7B
:10AE80006369A2699342F1DA03EB430221699200FC
:10AE900001338D186361ADD047238B546860236AFA
:10AEA000626A9342E2DAE069591CE26840F8235092
:10AEB0002162137892E70131C160FEF70DFA054671
:10AEC0000028A6D0E26813785F2B87D12046013294
:10AED00040F80C2FFEF780F900288BDA99E7236BF6
:10AEE000AA68134423630B78432B4FD0442B7FF481
:10AEF00066AF4B78303B052B8BD801A252F823F07C
:10AF000055AF000819AF000851AF000813AE000894
:10AF10004DAF000849AF000802276369A269881C89
:10AF20009342E06056DA03EB43022069920001335A
:10AF30008618636105D0002D4FD0082383543771E4
:10AF4000B5608B78354649E70527E6E70427E4E74F
:10AF50000327E2E70127E0E74268236B91680733A4
:10AF60000B4410681E49236304F0A8FB00287FF4FB
:10AF700041AF2046FEF7B0F92A4603463621204667
:10AF8000FDF7DAFFE36805461B7827E74B78313B8E
:10AF9000042B3FF63EAFDFE803F015031B19170043
:10AFA00002276369A269881C9342E06012DA03EB0E
:10AFB000430220699200013386186361C1D065B1F4
:10AFC0000723BBE70127ECE70527EAE70427E8E7C3
:10AFD0000327E6E78B78002500E78B78FEE600BFC5
:10AFE000A0B8010870B5C36804461A784A2A0DD083
:10AFF00071B90D462046FFF781FE78B103462A4617
:10B000002046BDE870402921FDF796BF0133C3609B
:10B010002046FFF715FA05460028EBD1002070BD49
:10B02000C3681A78462A01D00020704710B55A1C10
:10B03000C2605A780121592A04BF0233C360044612
:10B04000FFF7D0FF01462046FEF728F8E3681A789C
:10B05000452A01D0002010BD0133E36010BD00BFC0
:10B060002DE9F047C36805461A78472A1FD0542AAD
:10B070001DD00E46FFF72CF8044610B32EB3AB6874
:10B08000DB0722D42378A3F11C02042A40D94C2BDD
:10B090003ED0022B16D1A3681A78A2F11C01042914
:10B0A00040F283824C2A00F08082A3600AE0296B80
:10B0B00001F114022A631A78542A2BD0472A00F08F
:10B0C0009F8000242046BDE8F087EB681B78002BAA
:10B0D000F8D0452BF6D021460A78202A00F21381B9
:10B0E0001C2A80F01281042A40F001814A686AB16A
:10B0F0001378082B03F1FF3100F2F680072B80F064
:10B10000F680012902D89268002AF1D10121EFE0EE
:10B110006468B7E75A1CEA605A78002AD1D09A1CB2
:10B12000EA605B78433B332BCBD801A252F823F083
:10B130006BB50008C3B00008C3B0000855B50008DF
:10B14000C3B000083FB5000829B5000813B50008D2
:10B15000C3B00008C3B00008C3B00008C3B0000803
:10B16000C3B00008C3B00008C3B00008C3B00008F3
:10B17000FDB40008E3B40008C3B00008C9B4000877
:10B18000B3B40008C3B00008C3B00008C3B00008DF
:10B19000C3B00008C3B00008C3B00008C3B00008C3
:10B1A000C3B00008C3B00008C3B00008C3B00008B3
:10B1B0007FB40008C3B00008C3B00008C3B00008E3
:10B1C000C3B0000859B40008C3B00008C3B00008F9
:10B1D000C3B00008C3B00008C3B00008C3B0000883
:10B1E000C3B00008C3B00008C3B00008C3B0000873
:10B1F000C3B00008C3B00008C3B0000833B40008EF
:10B200005A1CEA605A78002A3FF45BAF9A1CEA6045
:10B210005A78413A312A3FF654AF01A151F822F051
:10B2200015B30008C3B00008C3B00008C3B00008DD
:10B23000C3B00008C3B00008C3B00008C3B0000822
:10B24000C3B00008C3B00008C3B00008C3B0000812
:10B25000C3B00008C3B00008C3B00008C3B0000802
:10B26000C3B0000815B40008C3B00008E9B3000873
:10B27000C3B00008D3B30008C3B00008C3B00008CF
:10B28000C3B00008C3B00008C3B00008C3B00008D2
:10B29000C3B00008C3B00008C3B00008C3B00008C2
:10B2A000C3B00008C3B00008C3B00008C3B00008B2
:10B2B000C3B00008C3B00008C3B00008C3B00008A2
:10B2C000C3B00008C3B00008C3B00008C3B0000892
:10B2D000C3B00008C3B00008C3B00008C3B0000882
:10B2E000C3B000082DB30008342B7FF40FAF00214A
:10B2F0002846FFF777FE2246034603212846BDE88D
:10B30000F047FDF719BE4C2AF1D1496800297FF4B6
:10B31000E3AEEDE700212846FFF7A2FE0023024638
:10B3200017212846BDE8F047FDF706BE05F10C00E1
:10B33000FDF752FF01287FF7C4AEEB681A78002AA8
:10B340003FF4BFAE5F1CEF601B785F2B7FF4B9AE9C
:10B3500000224FF040099046461E3B78002B3FF4F8
:10B36000B0AE242B00F028813C46002104E014F804
:10B37000013F23B1242B02D00131B142F7DB6C69CC
:10B38000A869844280F213812869631C04EB440499
:10B390006B6110EB840300F00A8100F824805F6089
:10B3A0009960EF68761A0F44EF60002A00F021815F
:10B3B0003F212846FDF7C0FD024600283FF481AE3C
:10B3C000002ECADC2846BDE8F04700233E21FDF7E9
:10B3D000B3BD2846FEF77CFE002302461321284613
:10B3E000BDE8F047FDF7A8BD9A7800212846002A5D
:10B3F00000F00181DA1CEA609B786E2B40F0FB8044
:10B40000FFF72EFE0023024649212846BDE8F047FB
:10B41000FDF792BD2846FEF75BFE04462846FDF781
:10B4200005FF2246034616212846BDE8F047FDF7F2
:10B4300083BD76212846FEF783F800283FF441AE0D
:10B4400000212846FFF70CFE002302461021284663
:10B45000BDE8F047FDF770BD68212846FEF770F89B
:10B4600000283FF42EAE00212846FFF7F9FD002307
:10B4700002460F212846BDE8F047FDF75DBD0021DB
:10B480002846FEF75DF800283FF41BAE0021284651
:10B49000FEF756F800283FF414AE00212846FFF7C7
:10B4A000DFFD0023024611212846BDE8F047FDF7E5
:10B4B00043BD2846FEF70CFE002302461521284610
:10B4C000BDE8F047FDF738BD0F3129632846FEF788
:10B4D000B7FF0023024609212846BDE8F047FDF7E3
:10B4E0002BBD0A3129632846FEF7AAFF0023024636
:10B4F0000A212846BDE8F047FDF71EBD2846FEF7A5
:10B500009FFF002302460D212846BDE8F047FDF7C6
:10B5100013BD2846FEF794FF002302461221284659
:10B52000BDE8F047FDF708BD2846FEF789FF002378
:10B5300002460C212846BDE8F047FDF7FDBC284631
:10B54000FEF7C6FD0023024614212846BDE8F04759
:10B55000FDF7F2BC2846FEF773FF002302460E21DA
:10B560002846BDE8F047FDF7E7BC2846FEF768FF30
:10B57000044605F10C00FDF72FFE0028FFF6A1ADF3
:10B58000EB681A785F2A7FF49CAD0133EB602846A4
:10B59000FEF756FF2B6B0246591D296323462846AA
:10B5A000BDE8F0470B21FDF7C7BC5B6874E5EB68AD
:10B5B00000240B44EB6085E57B78532B27D05F2B71
:10B5C00023D0242B7FF47DAD18466969AB6999427D
:10B5D0001FDA2C694F1C01EB410114EB81036F61F1
:10B5E00017D004F821905860EF68023E0237EF60F0
:10B5F000DBE61A46E4E6FFF733FD00230246482166
:10B600002846BDE8F047FDF797BC2E20DDE72F2048
:10B61000DBE7EB6800240233EB6053E5F8B5C26862
:10B6200013784C2B01D00020F8BD531CC360517817
:10B6300005465F293AD05A293FD0FEF701FF00287E
:10B64000F1D00378272B46D0EE6833786E2B4BD0A1
:10B650003C21452B4ED0002BE5D0334601E0002C99
:10B66000E1D00133EB601C78452CF8D19C1B6B6951
:10B67000AA6993422DDA03EB43022F69013392004A
:10B680006B61BB1825D026B31CB34FF0000E07F832
:10B6900002E05E609C6002462846FDF74DFCEB68C8
:10B6A0001A78452ABFD10133EB60F8BD931CC36003
:10B6B00092785A2A18BF002007D10133EB6000218D
:10B6C0002846FFF7CDFCEB681A78452AEBD000201E
:10B6D000F8BD0023DFE743681A7C002AB4D05A681B
:10B6E0002B6B9B1A2B63AFE7721CEA6073783D21CA
:10B6F0001646AEE70024BAE72DE9F04F044695B0B0
:10B70000002A00F0DB80D0F81871002F40F0C280D2
:10B710001378884615464D2B01F2EA81DFE813F0D5
:10B7200059043B043B04A403A4048804E9048E03E5
:10B730007C03300356030A03E4029802BE0272023D
:10B740004C02F0012602CA01A40158017E01320117
:10B750000B01F200F200F200D400D400D400D400B7
:10B76000D400D400D400D806D806D400D400AC0647
:10B77000FF069606200704078C0704077B057B0558
:10B7800032060806E205E809AF05910656064E00A6
:10B7900084045009E308E308B208B2088C0848059D
:10B7A0003A05E8081405C20918099C09E809CF07F9
:10B7B0006608F5071B081204D4005205AB681B7815
:10B7C000382B7BD16A6853681B685978632902F06B
:10B7D000508105F108034146204603F0C9FB0646A7
:10B7E000002857D16B681A78312A02F071835B68A0
:10B7F000C749186803F062FFAB6820B95A6811782E
:10B80000032902F0AB835A684146204603F04CFB03
:10B810006F68C0497B68D3F80090484603F04EFF3C
:10B820000646002842F07582D4F80011FF2902F084
:10B8300050845B234A1CC4F80021635484F804310B
:10B84000AB6841469A68204602F000FDD4F800112A
:10B85000FF2902F02B845D234A1CC4F800216354A5
:10B8600084F804316B681A78312A13D15B689A68BE
:10B87000012A0FD15B681B783E2B0BD1D4F8001145
:10B88000FF2902F0888429234A1CC4F8002163544C
:10B8900084F8043115B0BDE8F08FD4F82031002BC6
:10B8A000C1F2A884002B02F038848068013B10B1FB
:10B8B00002782F2AF6D00FB1C4F810610123C4F822
:10B8C000183115B0BDE8F08FD4F814C1002114ABC5
:10B8D000D4F8102143F840CD0595C4F814310691F1
:10B8E00007926A684146204602F0B0FC069B002B96
:10B8F00001F08D83049BC4F81431002FCAD0C4F822
:10B900001061C7E7D0F814C1BCF1000FDED0624669
:10B9100005E08B4201F0BC861268002AD6D0906800
:10B920000028F9D151680978A1F1190EBEF1020F72
:10B93000EFD90746CAE7AF686D68002FAAD04FF06D
:10B940000008D0F800112F4408E00B460131BD4239
:10B95000C4F80011E65484F804619BD0FF2915F85F
:10B96000016BF2D1D4F80831D4F80C2184F8FF80AF
:10B97000204698470121D4F8242100230A44C4F822
:10B980002421E4E7644E4FF00009D0F8001106F1DD
:10B99000110A09E00B4601315645C4F80011E7547D
:10B9A00084F8047101F09A82FF2916F8017FF1D121
:10B9B000D4F80831D4F80C2184F8FF902046984739
:10B9C0000121D4F8242100230A44C4F82421E3E708
:10B9D000524E4FF00009D0F8001106F1190A09E0A3
:10B9E0000B4601315645C4F80011E75484F8047140
:10B9F00001F0AC82FF2916F8017FF1D1D4F80831AB
:10BA0000D4F80C2184F8FF90204698470121D4F8FF
:10BA1000242100230A44C4F82421E3E7404E4FF0D8
:10BA20000009D0F8001106F1150A09E00B460131B2
:10BA30005645C4F80011E75484F8047101F05582AA
:10BA4000FF2916F8017FF1D1D4F80831D4F80C2180
:10BA500084F8FF90204698470121D4F82421002340
:10BA60000A44C4F82421E3E72E4E4FF00009D0F831
:10BA7000001106F1160A09E00B4601315645C4F8DB
:10BA80000011E75484F8047101F06782FF2916F869
:10BA9000017FF1D1D4F80831D4F80C2184F8FF905B
:10BAA000204698470121D4F8242100230A44C4F8F1
:10BAB0002421E3E71C4E4FF00009D0F8001106F1F5
:10BAC000130A09E00B460131B245C4F80011E754EE
:10BAD00084F8047101F07C80FF2916F8017FF1D110
:10BAE000D4F80831D4F80C2184F8FF902046984708
:10BAF0000121D4F8242100230A44C4F82421E3E7D7
:10BB00000A4E4FF00009D0F8001106F11A0A19E0A8
:10BB100064B8010860BA0108EFB90108BBB90108AF
:10BB2000D7B90108A3B901088FB9010863B90108A1
:10BB30000B4601315645C4F80011E75484F80471EE
:10BB400001F05480FF2916F8017FF1D1D4F80831B3
:10BB5000D4F80C2184F8FF90204698470121D4F8AE
:10BB6000242100230A44C4F82421E3E7B54E4FF012
:10BB70000009D0F8001106F10F0A09E00B46013167
:10BB80005645C4F80011E75484F8047101F0278089
:10BB9000FF2916F8017FF1D1D4F80831D4F80C212F
:10BBA00084F8FF90204698470121D4F824210023EF
:10BBB0000A44C4F82421E3E7A34E4FF00009D0F86B
:10BBC000001106F1110A09E00B4601315645C4F88F
:10BBD0000011E75484F8047101F00F80FF2916F872
:10BBE000017FF1D1D4F80831D4F80C2184F8FF900A
:10BBF000204698470121D4F8242100230A44C4F8A0
:10BC00002421E3E7914E4FF00009D0F8001106F12E
:10BC1000150A09E00B4601315645C4F80011E754F6
:10BC200084F8047100F0B887FF2916F8017FF1D17C
:10BC3000D4F80831D4F80C2184F8FF9020469847B6
:10BC40000121D4F8242100230A44C4F82421E3E785
:10BC50007F4E4FF00009D0F8001106F1120A09E0FA
:10BC60000B460131B245C4F80011E75484F8047161
:10BC700000F0A087FF2916F8017FF1D1D4F8083130
:10BC8000D4F80C2184F8FF90204698470121D4F87D
:10BC9000242100230A44C4F82421E3E76D4E4FF029
:10BCA0000009D0F8001106F1100A09E00B46013135
:10BCB0005645C4F80011E75484F8047100F0738706
:10BCC000FF2916F8017FF1D1D4F80831D4F80C21FE
:10BCD00084F8FF90204698470121D4F824210023BE
:10BCE0000A44C4F82421E3E75B4E4FF00009D0F882
:10BCF000001106F10D0A09E00B4601315645C4F862
:10BD00000011E75484F8047100F05B87FF2916F8EE
:10BD1000017BF1D1D4F80831D4F80C2184F8FF90DC
:10BD2000204698470121D4F8242100230A44C4F86E
:10BD30002421E3E7494E4FF00009D0F8001106F145
:10BD4000180A09E00B460131B245C4F80011E75466
:10BD500084F8047100F0E886FF2916F8017FF1D11C
:10BD6000D4F80831D4F80C2184F8FF902046984785
:10BD70000121D4F8242100230A44C4F82421E3E754
:10BD8000374E4FF00009D0F8001106F10B0A09E018
:10BD90000B460131B245C4F80011E75484F8047130
:10BDA00000F0CF87FF2916F8017BF1D1D4F80831D4
:10BDB000D4F80C2184F8FF90204698470121D4F84C
:10BDC000242100230A44C4F82421E3E7254E4FF040
:10BDD0000009D0F8001106F1080A09E00B4601310C
:10BDE000B245C4F80011E75484F8047100F0CD8620
:10BDF000FF2916F8017FF1D1D4F80831D4F80C21CD
:10BE000084F8FF90204698470121D4F8242100238C
:10BE10000A44C4F82421E3E7D0F80011FF2901F017
:10BE200080844A1C7E23C4F80021635484F80431C2
:10BE30004146AA68204602F009FA2BE5AA6802F0FA
:10BE400005FA27E57FB901084FB901084BB9010888
:10BE500023B9010837B9010814B90108EFB801087E
:10BE6000D8B80108E3B801080022D0F81431C0F8AE
:10BE700014216E680093002E00F051860DF1100918
:10BE8000174696464B46D0F810C131781A60A1F19A
:10BE90001C02042A5E60C3F808E0C3F80CC007F176
:10BEA0000107184640F22F864C2900F02C86042901
:10BEB000C4F8143101F0C28702291AD1D6F808B0AB
:10BEC0009BF80030462B02F03C802B4609EB071E06
:10BED00001965D467646A2469B462B78A3F11C024E
:10BEE000042A41F262804C2B01F05F8054465D468B
:10BEF000019EAA684146204602F0A8F93378042B37
:10BF000002F02780202509EB071959F8086C013F3A
:10BF100086B9D4F80011FF2902F04A804B1CC4F8FE
:10BF2000003159F80C2C65542046414684F80451E0
:10BF300002F09CF9A9F11009002FE6D1009BC4F88A
:10BF40001431A7E4D24E6A6802F080F94FF000097C
:10BF5000D4F8001106F1050A09E00B460131B2459B
:10BF6000C4F80011E75484F8047100F0D786FF2963
:10BF700016F8017BF1D1D4F80831D4F80C2184F8FB
:10BF8000FF90204698470121D4F8242100230A4439
:10BF9000C4F82421E3E76A6802F058F918F00409AC
:10BFA00001F0AF82D4F80011FF2901F0A1854A1CED
:10BFB0002E23C4F80021635484F80431AD682B7833
:10BFC000462B01F0D1832A464146204602F03EF935
:10BFD00060E411F0040841F09080AF686D68002FB4
:10BFE0003FF458ACD0F800112F4409E00B46013162
:10BFF000BD42C4F80011E65484F804613FF44AAC31
:10C00000FF2915F8016BF1D1D4F80831D4F80C21CF
:10C0100084F8FF80204698470121D4F8242100238A
:10C020000A44C4F82421E3E70123C0F8183131E4BD
:10C03000D0F81C31002B41F00A81291DFDF7AAFA26
:10C0400000283FF43BAC03782F2B01F00184D4F897
:10C05000105102462B684146C4F81031204602F0C8
:10C06000F5F8C4F8105115E40023D0F81491D0F875
:10C070004471C0F81431C0F8445111F0040F6E68D7
:10C0800005D033781BB9B268062A01F043853246E1
:10C090004146204602F0DAF894F804313C2B01F0D6
:10C0A0007982D4F80031FF2B01F09084591C3C2296
:10C0B000C4F80011E25484F804214146AA682046DD
:10C0C00002F0C4F894F804313E2B01F03E82D4F81B
:10C0D0000031FF2B01F06784591C3E22C4F8001187
:10C0E000E25484F80421C4F81491C4F84471FFF7B1
:10C0F000D1BBD5F80490B9F1000F01F08580654DF2
:10C100004FF00008D0F80011AF1D09E00B460131D7
:10C11000AF42C4F80011E65484F8046100F0868749
:10C12000FF2915F8016BF1D1D4F80831D4F80C21AE
:10C1300084F8FF80204698470121D4F82421002369
:10C140000A44C4F82421E3E7534E4FF00009D0F825
:10C15000001106F10A0A09E00B4601315645C4F800
:10C160000011E75484F8047100F00587FF2916F8E0
:10C17000017BF1D1D4F80831D4F80C2184F8FF9078
:10C18000204698470121D4F8242100230A44C4F80A
:10C190002421E3E7D0F800112D79FF2901F0AF82C7
:10C1A0004B1CC4F80031655484F80451FFF772BB8E
:10C1B0006A6802F04BF8AA684146204602F046F849
:10C1C000FFF768BB354E6A6802F040F84FF000098F
:10C1D000D4F8001106F1080A09E00B460131564572
:10C1E000C4F80011E75484F8047100F00D85FF29AC
:10C1F00016F8017FF1D1D4F80831D4F80C2184F875
:10C20000FF90204698470121D4F8242100230A44B6
:10C21000C4F82421E3E76A680AB102F017F8AB68B2
:10C22000002B3FF437ABD4F80061FD2E01F2C08142
:10C230001B4F07F1020B0AE0B24601365F45C4F816
:10C24000006104F80A9084F8049100F0C986FF2E7A
:10C2500017F8019BF0D14FF000033146012684F816
:10C26000FF30D4F80C21D4F8083120469847D4F890
:10C2700024314FF0000A3344C4F82431DEE7094E7C
:10C280004FF00009D0F8001106F1090A16E000BFCE
:10C29000A4B80108B4BA01089CBA01081BBB010884
:10C2A00038BA010847BA01080B4601315645C4F8AF
:10C2B0000011E75484F8047100F09685FF2916F800
:10C2C000017FF1D1D4F80831D4F80C2184F8FF9023
:10C2D000204698470121D4F8242100230A44C4F8B9
:10C2E0002421E3E7D24E4FF00009D0F8001106F107
:10C2F000090A09E00B4601315645C4F80011E7541C
:10C3000084F8047100F09985FF2916F8017FF1D1B6
:10C31000D4F80831D4F80C2184F8FF9020469847CF
:10C320000121D4F8242100230A44C4F82421E3E79E
:10C33000D5F804A0BF4D4FF00008DAF80870D0F827
:10C34000001105F1080909E00B460131A945C4F8BF
:10C350000011E65484F8046100F00885FF2915F8FF
:10C36000016FF1D1D4F80831D4F80C2184F8FF80A2
:10C37000204698470121D4F8242100230A44C4F818
:10C380002421E3E76A68AE680AB101F05FFFD4F8E0
:10C390000031FF2B01F0B5825A1C7B25C4F8002127
:10C3A0004146E5543246204684F8045101F04EFFE0
:10C3B000D4F80011FF2901F0E9814A1C7D23C4F85B
:10C3C0000021635484F80431FFF764BAD5F804906F
:10C3D000AE6899F80030312B00F0CC87332B41F058
:10C3E000D786D0F80011FF2901F0C78428234A1C02
:10C3F000C4F80021635484F80431D9F80430D4F827
:10C40000285104A91A46C4F828112046414604932D
:10C410000595FFF771F9D4F80011059BFF29C4F8C1
:10C42000283101F0998429234A1CC4F8002163545F
:10C4300084F8043132464146204602F035FDFFF7CC
:10C4400029BA6A6802F0F2FCFFF724BA11F0200F53
:10C4500040F053876A681AB118F0400601F0D181A4
:10C4600028F0600805F108024146D4F8143120464E
:10C4700002F0E8FBFFF70EBA11F004086B6840F019
:10C48000138693E8A000002F3FF404AAD0F800110F
:10C490002F4409E00B460131BD42C4F80011E654B7
:10C4A00084F804613FF4F6A9FF2915F8016BF1D176
:10C4B000D4F80831D4F80C2184F8FF80204698473E
:10C4C0000121D4F8242100230A44C4F82421E3E7FD
:10C4D0006968D0F81C710B78002F40F0E285052BBD
:10C4E00001F0C881232B00F08A862A789A4200F056
:10C4F0008686242B7FF4E8A900234A68D4F8141117
:10C5000014A840F8401DD4F810110595C4F8140182
:10C5100006930791002A7FF4E5A9FFF7E2B96A685C
:10C5200001F094FEFFF7B6B90027D0F8142114AB40
:10C5300043F8402DC0F81431D0F81061AA68059571
:10C540000697079601F082FE069B23B92A464146CC
:10C55000204601F08BFE049BC4F81431FFF79AB912
:10C56000D0F814A1002251460DF15009D0F8103135
:10C5700049F840ADCDF800A0C0F814910595069299
:10C580000793002901F0A3834B681B78193B022B0A
:10C5900001F29D83AC4601270E464D4604E07368C8
:10C5A0001B78193B022B1CD8B3684FEA071AABB9AA
:10C5B000032F01F2FD8096E80F000DF1500E0EEBF7
:10C5C0000A0BABF1400E8EE80F0001234BF8405CE4
:10C5D00009EB0A05C4F814510137B3603668002E20
:10C5E000DDD1DCF8082041462046654601F02EFEEC
:10C5F000009A069BC4F81421002B7FF44BA9012F4D
:10C600000CD009EB071959F80C2C013F4146204684
:10C6100001F02CFE012FA9F11009F4D12A1D414689
:10C62000D4F81431204602F031FAFFF733B900BFD5
:10C6300047BA01083BBA0108B5F90A30002B40F0AF
:10C6400073866A68D54B5168994200F06986414605
:10C65000204601F0FBFDD4F80031FF2B01F0B4823D
:10C66000591C2022C4F80011E25484F80421B5F9C1
:10C670000830002B00F09585C94D4FF00008AF1D24
:10C6800009E00B460131BD42C4F80011E65484F8BC
:10C6900004613FF4FFA8FF2915F8016BF1D1D4F82C
:10C6A0000831D4F80C2184F8FF80204698470121F6
:10C6B000D4F8242100230A44C4F82421E3E7B94E26
:10C6C0004FF00008D0F8001106F10E0909E00B4602
:10C6D0000131B145C4F80011E75484F8047100F049
:10C6E000B383FF2916F8017FF1D1D4F80831D4F8CB
:10C6F0000C2184F8FF80204698470121D4F824219A
:10C7000000230A44C4F82421E3E7A74E4FF00009B0
:10C71000D0F8001106F11A0A09E00B46013156451E
:10C72000C4F80011E75484F8047100F0F082FF2986
:10C7300016F8017FF1D1D4F80831D4F80C2184F82F
:10C74000FF90204698470121D4F8242100230A4471
:10C75000C4F82421E3E76968FCF738FF4FF00009CB
:10C76000002801F05F8303782F2B40F05784436843
:10C77000002B00F05384806809F101090028F2D1F0
:10C780006B6800934FF0000A09F1FF330193C4F87E
:10C790002071009A4146204601F058FD019BBB42A2
:10C7A00040F3AB81814DD4F8001105F1020B09E093
:10C7B0000B460131AB45C4F80011E65484F804611E
:10C7C00000F09B81FF2915F8016BF1D1D4F80831F5
:10C7D000D4F80C2184F8FFA0204698470121D4F812
:10C7E000242100230A44C4F82421E3E7704E4FF0CB
:10C7F0000009D0F8001106F1160A09E00B460131D4
:10C80000B245C4F80011E75484F8047100F05F8366
:10C81000FF2916F8017FF1D1D4F80831D4F80C21A2
:10C8200084F8FF90204698470121D4F82421002362
:10C830000A44C4F82421E3E75E4E4FF00009D0F823
:10C84000001106F10E0A09E00B4601315645C4F805
:10C850000011E75484F8047100F0A083FF2916F852
:10C86000017FF1D1D4F80831D4F80C2184F8FF907D
:10C87000204698470121D4F8242100230A44C4F813
:10C880002421E3E76A681178272900F0158600263D
:10C89000D4F80011FF2901F0C78028234A1CC4F8EE
:10C8A0000021635484F804316A684146204601F04F
:10C8B000CDFCD4F80031FF2B01F09B802922591CBC
:10C8C000C4F80011E25484F804212B783D2B00F0C9
:10C8D000E686082E00F07F86AA684146204601F0D1
:10C8E000B5FCFEF7D7BF0123C0F81831FEF7D2BF61
:10C8F0006A6804A8304909F0F1FC04A809F014FDA5
:10C9000000283EF4C7AF04AD4FF00008D4F8001182
:10C910002F1809E00B460131BD42C4F80011E6545E
:10C9200084F804613EF4B6AFFF2915F8016BF1D12C
:10C93000D4F80831D4F80C2184F8FF8020469847B9
:10C940000121D4F8242100230A44C4F82421E3E778
:10C950001A4E4FF00009D0F8001106F11C0A09E048
:10C960000B4601315645C4F80011E75484F80471B0
:10C9700000F0FA82FF2916F8017FF1D1D4F80831CE
:10C98000D4F80C2184F8FF90204698470121D4F870
:10C99000242100230A44C4F82421E3E714AE01084B
:10C9A00028BA01080BBB010803BA010838BA01080C
:10C9B00007BA01088BBA01085CB80108DBBA0108A4
:10C9C000AB681A783A2A7EF479AF9B681B783B2BC8
:10C9D0007EF474AF05F108036A6802F0C9FA0646EE
:10C9E00000287EF457AFD5F804A0AA68DAF804103E
:10C9F00093680868D649D2F804905F689D6802F091
:10CA00005DFE002801F0E4820422D2492046FCF7B2
:10CA1000B1FBD9F8043083B141464A46204602F0C2
:10CA200043FAD4F80011FF2901F0EE8320234A1CB9
:10CA3000C4F80021635484F804313A464146204644
:10CA400001F004FC002D3EF425AF2A464146204665
:10CA500002F02AFAFEF71EBFBF4E4FF00009D0F8D1
:10CA6000001106F1080A09E00B4601315645C4F8E9
:10CA70000011E75484F8047100F0D980FF2916F8FA
:10CA8000017FF1D1D4F80831D4F80C2184F8FF905B
:10CA9000204698470121D4F8242100230A44C4F8F1
:10CAA0002421E3E7AD4E4FF00009D0F8001106F164
:10CAB0001D0A09E00B460131B245C4F80011E754E4
:10CAC00084F8047100F0FC81FF2916F8017FF1D190
:10CAD000D4F80831D4F80C2184F8FF902046984708
:10CAE0000121D4F8242100230A44C4F82421E3E7D7
:10CAF0000123C0F81831FEF7CDBE01374F457FF452
:10CB000046AEFEF7C7BE7668002E01F07080042F97
:10CB100003F1100302467FF4B8A9C4F814010123FD
:10CB2000C4F81831FEF7B6BE8D4E41466A682046FD
:10CB300001F08CFB4FF00009D4F8001106F1040A53
:10CB400008E00B460131B245C4F80011E75484F8FF
:10CB5000047113D0FF2916F8017BF2D1D4F8083103
:10CB6000D4F80C2184F8FF90204698470121D4F88E
:10CB7000242100230A44C4F82421E4E7AA6841469A
:10CB8000204601F063FBFEF785BE6A6841462046F9
:10CB900001F05CFBFEF77EBE6A684146204601F06C
:10CBA00055FBFEF777BE6A684146204601F04EFB12
:10CBB000FEF770BE6A684146204601F047FBFEF76B
:10CBC00069BE6A684146204601F040FBFEF762BE3E
:10CBD0006A684146204601F039FBFEF75BBE6A6891
:10CBE0004146204601F032FBFEF754BE6A684146DA
:10CBF000204601F02BFBFEF74DBE6A6841462046F9
:10CC000001F024FBFEF746BE4146AA68204601F02B
:10CC10001DFBD4F80011FF2900F05F854A1C5D233D
:10CC2000C4F80021635484F80431FEF733BED4F80D
:10CC30001C3141460133C4F81C316A68204601F0BA
:10CC400005FBD4F81C31474E013B4FF00009D4F8E6
:10CC50000011C4F81C3106F1020808E00B4601314E
:10CC60004645C4F80011E75484F8047113D0FF2935
:10CC700016F8017BF2D1D4F80831D4F80C2184F8ED
:10CC8000FF90204698470121D4F8242100230A442C
:10CC9000C4F82421E4E7AA6804A80132324909F063
:10CCA0001DFB04A809F040FB18B304AD4FF00008C9
:10CCB000D4F800112F1808E00B460131AF42C4F838
:10CCC0000011E65484F8046115D0FF2915F8016BB2
:10CCD000F2D1D4F80831D4F80C2184F8FF80204632
:10CCE00098470121D4F8242100230A44C4F82421C0
:10CCF000E4E7D4F80011FF2900F05F854A1C7D238A
:10CD0000C4F80021635484F80431FEF7C3BD6A6897
:10CD10004146204601F09AFAFEF7BCBD4146AA689A
:10CD2000204601F093FAD4F80011FF2900F00A859B
:10CD30004A1C5D23C4F80021635484F80431FEF7D3
:10CD4000A9BD6A684146204601F080FAFEF7A2BDFF
:10CD500070B8010868BA0108FBBA0108BBBA01083B
:10CD60000CB9010808BB01085CB80108DAF80450E6
:10CD70002B78613B192B09D8FF2900F095872023D8
:10CD80004A1CC4F80021635484F80431EB1913F8E9
:10CD9000013C202B08BF07F1FF37002F3EF47AAD8E
:10CDA0004FF00008D4F800112F4409E00B46013180
:10CDB000AF42C4F80011E65484F804613EF46AAD51
:10CDC000FF2915F8016BF1D1D4F80831D4F80C2102
:10CDD00084F8FF80204698470121D4F824210023BD
:10CDE0000A44C4F82421E3E7D4F844213AB1D4F842
:10CDF000101114AB43F8481D0392C4F810316B684E
:10CE00001A78042A00F00D83D4F8285104A81A4691
:10CE1000C4F828014146204604930595FEF76CFCB2
:10CE2000059AD4F84431C4F82821002B3EF432ADE1
:10CE3000029BC4F81031FEF72DBDAA68414620467A
:10CE400001F004FAFEF726BD6A6804A80132D7494A
:10CE500009F044FA04A809F067FA18B304AD4FF0DA
:10CE60000008D4F800112F1808E00B460131BD422C
:10CE7000C4F80011E65484F8046115D0FF2915F8B0
:10CE8000016BF2D1D4F80831D4F80C2184F8FF807A
:10CE9000204698470121D4F8242100230A44C4F8ED
:10CEA0002421E4E7D4F80011FF2900F004844A1C8F
:10CEB0007D23C4F80021635484F80431FEF7EABCF2
:10CEC0006A684146204601F0C1F9FEF7E3BC6A6892
:10CED0004146204601F0BAF9FEF7DCBC6A684146DB
:10CEE000204601F0B3F9FEF7D5BCB14E4146AA6821
:10CEF000204601F0ABF94FF00009D4F8001106F11B
:10CF0000050A08E00B4601315645C4F80011E75404
:10CF100084F8047113D0FF2916F8017BF2D1D4F8FC
:10CF20000831D4F80C2184F8FF902046984701215D
:10CF3000D4F8242100230A44C4F82421E4E76A68D1
:10CF40004146204601F082F9FEF7A4BC6A684146DA
:10CF5000204601F07BF9FEF79DBC6A6841462046F9
:10CF600001F074F9FEF796BC6A684146204601F06C
:10CF70006DF9FEF78FBC41466A68204601F066F9FC
:10CF8000D4F80011FF2900F02A844A1C2923C4F890
:10CF90000021635484F80431FEF77CBC6A68414682
:10CFA000204601F053F9FEF775BC042F06F1100E70
:10CFB000A6F1100400F0248794E80F0086E80F0023
:10CFC0000023CAF814614EF8104C4EF81C5C4EF861
:10CFD000183C4EF814CC76466D680137FEF77DBFDD
:10CFE000AA6841462046D4F8245101F02FF9D4F81C
:10CFF00024319D427EF44EACD4F80031B3427EF42D
:10D0000049AC0AF1FF33C4F80031FEF743BC2A46AD
:10D010004146204601F02AF9FEF76CBC6B6800938C
:10D02000B9F1000F7FF4AEABFEF734BC4A4604A85A
:10D030005E4909F053F904A809F076F918B304AD74
:10D040004FF00008D4F800112F1808E00B4601310A
:10D05000AF42C4F80011E65484F8046115D0FF29EA
:10D0600015F8016BF2D1D4F80831D4F80C2184F80A
:10D07000FF80204698470121D4F8242100230A4448
:10D08000C4F82421E4E7D4F80011FF2900F0DF847C
:10D090004A1C7D23C4F80021635484F80431FEF750
:10D0A000F9BB0027FFF71EBADF689D68002F3EF42A
:10D0B000F1AB4FF00008D0F800112F4409E00B4607
:10D0C0000131BD42C4F80011E65484F804613EF415
:10D0D000E1ABFF2915F8016BF1D1D4F80831D4F890
:10D0E0000C2184F8FF80204698470121D4F82421A0
:10D0F00000230A44C4F82421E3E76E68AF6837448C
:10D10000BE42BEF4C7AB4FF000080DE0D4F80011EA
:10D11000FF2936D04B1CC4F80031655484F8045103
:10D120000136B7427EF6B6ABBB1B032B3578EDDD7F
:10D130005F2DEBD173785F2BE8D1B378552BE5D118
:10D14000F31C9F42E2D9002006E0A5F137029F427E
:10D1500002EB001000F0C985994613F8015BA5F1B8
:10D160003002D1B20929A5F1410EF0D9BEF1050F67
:10D17000A5F16102E9D9052A00F24587A5F1570218
:10D18000E5E7D4F80831D4F80C2184F8FF80204674
:10D1900098470123D4F8242100211A44C4F82421FB
:10D1A000B9E7044D9846AF1D10E000BF5CB8010818
:10D1B000D0B9010830BA01080B460131BD42C4F8AC
:10D1C0000011E65484F804613EF464ABFF2915F8BD
:10D1D000016BF1D1D4F80831D4F80C2184F8FF8028
:10D1E000204698470121D4F8242100230A44C4F89A
:10D1F0002421E3E72B782F2B7EF466AB01460D4606
:10D20000D4F814C1FEF762BBD74DD0F800112F1D22
:10D2100009E00B460131AF42C4F80011E65484F82E
:10D2200004613EF437ABFF2915F8016BF1D1D4F856
:10D230000831D4F80C2184F8FF902046984701214A
:10D24000D4F8242100230A44C4F82421E3E7C74E7C
:10D250004FF00008D0F8001106F1050908E00B4670
:10D260000131B145C4F80011E75484F8047113D0BA
:10D27000FF2916F8017BF2D1D4F80831D4F80C213B
:10D2800084F8FF80204698470121D4F82421002308
:10D290000A44C4F82421E4E76A6804A80132B449C6
:10D2A00009F01CF804A809F03FF800283EF4F2AA9F
:10D2B00004AD4FF00008D4F800112F1809E00B4618
:10D2C0000131AF42C4F80011E65484F804613EF421
:10D2D000E1AAFF2915F8016BF1D1D4F80831D4F88F
:10D2E0000C2184F8FF80204698470121D4F824219E
:10D2F00000230A44C4F82421E3E721F0600805F183
:10D3000008024146D0F8143101F09CFC6A68002AFA
:10D310003EF4C0AA4146204600F098FFFEF7BABA94
:10D32000D4F80011FFF7A3B9924E4FF00009D0F8DE
:10D33000001106F1050A09E00B460131B245C4F8B7
:10D340000011E75484F804713FF47BA9FF2916F813
:10D35000017BF1D1D4F80831D4F80C2184F8FF9086
:10D36000204698470121D4F8242100230A44C4F818
:10D370002421E3E7D9F804307F491F68384602F0DA
:10D380009DF996F800A018B9BAF1030F00F01E85B8
:10D39000BAF1380F00F000867849384602F08EF96D
:10D3A0000546002800F036817549384602F086F9B6
:10D3B000002800F0B9824A464146204601F036FD79
:10D3C000002F3FF437A86F49384602F077F900285C
:10D3D00000F0878338466C4902F070F90546002852
:10D3E0007FF428A8D4F80031FF2B00F0DE84282534
:10D3F000581CC4F800014146E5543246204684F8E2
:10D40000045100F023FFD4F80011FF2900F07084CC
:10D4100029234A1CC4F80021635484F80431FEF720
:10D4200039BA58680DF11009D4F828310246049031
:10D43000C4F82891414620460593FEF75DF9059A08
:10D44000D4F84431C4F8282113B1029BC4F8103138
:10D4500094F804313C2B00F0DB83D4F80011FF2951
:10D4600000F069843C234A1CC4F80021635484F80A
:10D4700004316B68D4F828519B6841461A46C4F8B9
:10D480002891204604930595FEF736F994F8043167
:10D49000059A3E2BC4F8282100F0AD83D4F8001182
:10D4A000FF2900F09C843E234A1CC4F800216354E9
:10D4B00084F80431FEF7EEB95268167C002E3FF472
:10D4C000E7A9062E40F23983072E7FF4E1A9AA6866
:10D4D000117800297FF4DCA9916801297FF4D8A98B
:10D4E0003C2B7FF4D5A953681B78302B00F028869D
:10D4F000312B7FF4CDA904222449FBF73BFEFEF734
:10D50000C9B9234ED4F8001106F1020A09E00B460E
:10D510000131B245C4F80011E75484F804713EF4B7
:10D520004DADFF2916F8017BF1D1D4F80831D4F8BC
:10D530000C2184F8FF90204698470121D4F824213B
:10D5400000230A44C4F82421E3E7D4F80011FF299A
:10D5500000F0E68420224B1CC4F80031625484F8A9
:10D560000421FEF7B6BD00BFACBA0108D0B801086F
:10D570005CB8010820BA010854BA010828BB0108A8
:10D5800060B8010858BA010868BD010884BA0108EA
:10D59000ACB80108D4F80011FF2900F067842022FC
:10D5A0004B1CC4F80031625484F80421FEF77BBDA3
:10D5B0000027A7553146D4F80831D4F80C2120466D
:10D5C0009847D4F824313E460133C4F80071C4F8BA
:10D5D0002431FEF72DBED4F80011FF2900F0678436
:10D5E0005B234A1CC4F80021635484F8043141468B
:10D5F000AA68204600F02AFED4F80011FF2900F0A6
:10D6000014835D234A1CC4F80021635484F8043158
:10D61000FEF740B931462046FBF7D8FF28B907E0AE
:10D6200043682BB18068013510B103782F2BF7D0F8
:10D630002A4604A8D54908F051FE04A808F074FE53
:10D6400000283EF427A904AD4FF00008D4F80011DB
:10D650002F1809E00B460131BD42C4F80011E65411
:10D6600084F804613EF416A9FF2915F8016BF1D185
:10D67000D4F80831D4F80C2184F8FF80204698476C
:10D680000121D4F8242100230A44C4F82421E3E72B
:10D690006A684146204600F0D9FDFEF7FBB8FF2935
:10D6A00000F0D4832D234A1CC4F80021635484F86D
:10D6B0000431FFF70EB90025D4F80831D4F80C2155
:10D6C00084F8FF50204698470122D4F82431294697
:10D6D0001344C4F82431FFF7EBBB0025D4F808311C
:10D6E000D4F80C2184F8FF50204698470122D4F842
:10D6F000243129461344C4F82431FFF790BA002698
:10D70000D0F8083180F8FF60D0F80C219847D4F8A1
:10D71000243131460133C4F80061C4F82431FEF7E6
:10D720003FBD0026D0F80831D0F80C2180F8FF600A
:10D7300098470122D4F8243131461344C4F82431E7
:10D74000FEF770BB0025D4F80831D4F80C2184F81A
:10D75000FF50204698470122D4F82431294613442B
:10D76000C4F82431FFF7E5BA0D2289492046FBF7BA
:10D7700001FDA96820460131FBF7ACFF0322854972
:10D780002046FBF7F7FC6D68FEF71DBC0025D4F8BA
:10D790000831D4F80C2184F8FF5020469847012224
:10D7A000D4F8243129461344C4F82431FEF706BEC8
:10D7B0000123C4F81831FEF76DB80025D4F80831FC
:10D7C000D4F80C2184F8FF50204698470122D4F861
:10D7D000243129461344C4F82431FFF790BA0025B8
:10D7E000D4F80831D4F80C2184F8FF50204698472B
:10D7F0000122D4F8243129461344C4F82431FFF718
:10D80000C5BBD4F8143114A941F8403D28F0600894
:10D81000D4F81031C4F814112046414606960793F7
:10D82000059500F013FD049B069EC4F81431002EEC
:10D830007EF430A8D4F80011FF2900F00B842023D7
:10D840004A1CC4F80021635484F80431FEF70ABE70
:10D85000D4F82031002BFEF6FAAB002B00F09F82AB
:10D860008068013B00283EF429A802782F2AF4D0D2
:10D87000FEF724B8D0F830E1D0F82C21BEF1000F2B
:10D8800014DD1368994200F0F7833B4602F108006B
:10D89000A44607E052F833408146A14200F1080057
:10D8A00000F0D38101339E45F4D16446D4F834317D
:10D8B0009E4580F2BB840EF1010302EBCE09C4F851
:10D8C000303142F83E10D4F810E109F104097246F3
:10D8D000002A00F08E84D4F83C01D4F8403100F1E5
:10D8E000010E984280F2A284D4F83831C4F83CE1A9
:10D8F00003EBC00350685860C9F8003012689946BD
:10D90000E6E700251946D4F80C21D4F8083184F84C
:10D91000FF50204698470122D4F824112B46114489
:10D92000C4F82411FEF739BD002E00F04D84BAF181
:10D930002F0F40F08884736873B3074607E0013700
:10D94000B66856B333782F2B27D173682BB31A7868
:10D950004A2AF4D159682046FBF738FE98B103787B
:10D960002F2B40F06C844368002B00F06484034646
:10D97000002004E01A782F2A05D15A681AB19B6852
:10D980000130002BF6D10744DAE700BF5CB801088C
:10D99000B0B80108C0B801081F4639462046FBF759
:10D9A00099FEFDF777BF00251946D4F80C21D4F86D
:10D9B000083184F8FF50204698470121D4F82421EB
:10D9C0002B460A44C4F82421FEF787BB00261946DB
:10D9D000D4F80C21D4F8083184F8FF602046984729
:10D9E0000121D4F8242133460A44C4F82421FEF747
:10D9F0005EBB0022194684F8FF20D4F80831D4F821
:10DA00000C212046984729230121237084F80431F2
:10DA10002A78D4F824313D2A0B44C4F82431C4F8C0
:10DA200000117EF456AF3DE60027D4F8083184F8A3
:10DA3000FF70D4F80C2120469847D4F82431394699
:10DA40000133C4F80071C4F82431FEF726BF002565
:10DA5000D4F80831D4F80C2184F8FF5020469847B8
:10DA60000122D4F8243129461344C4F82431FFF7A5
:10DA700010BB1B78A3F16301012903D9723B012B71
:10DA80003DF6A7AE4146204601F0D0F9D4F800118A
:10DA9000FF2900F071823C234A1CC4F80021635422
:10DAA00084F80431AB6841465A68204600F0CEFB4A
:10DAB0000222D5492046FBF75DFBAB6841469A68D8
:10DAC000204600F0C3FBD4F80011FF2900F0DF81ED
:10DAD00029234A1CC4F80021635484F80431FDF75B
:10DAE000D9BE32464146204600F0B0FBFDF7D2BE1B
:10DAF0000026D4F80831D4F80C2184F8FF602046C1
:10DB000098470122D4F8243131461344C4F8243113
:10DB1000FEF74EBABD49706808F034FC00287EF468
:10DB2000B6AAAA684146204600F090FB0222B849F6
:10DB30002046FBF71FFBFEF7D6BAAA681778002F1E
:10DB40007EF4A6AE3D2B00F0EF82AA684146204647
:10DB5000023E00F07BFB042E3DF69CAEDFE806F0B3
:10DB60002618110A030020460322AA49FBF702FBEC
:10DB7000FDF790BE20460222A749FBF7FBFAFDF70E
:10DB800089BE20460222A549FBF7F4FAFDF782BEC2
:10DB9000D4F80011FF2900F01A836C234A1CC4F842
:10DBA0000021635484F80431FDF774BED4F80011E9
:10DBB000FF2900F0DB8275234A1CC4F8002163545E
:10DBC00084F80431FDF766BE00261946D4F80C210E
:10DBD000D4F8083184F8FF60204698470121D4F832
:10DBE000242133460A44C4F82421FEF73ABDC4F880
:10DBF0001431FEF794BFD4F80011FF2900F04482DD
:10DC000020234A1CC4F80021635484F8043145E4FD
:10DC1000D4F80011FF2900F06E8220234A1CC4F8BA
:10DC20000021635484F8043117E40025D4F8083146
:10DC300084F8FF50D4F80C2120469847D4F82431BA
:10DC400029460133C4F82431DBE46446D4F82801C2
:10DC5000D8B1026891420AD0034604E05B68A3B1E0
:10DC60001A68914203D09542F8D19842F6D0043117
:10DC70002046FBF78FFC00283DF420AE03782F2BC5
:10DC80003DF40BAE0146FEF72DBCD9F80430D4F8B4
:10DC9000106104312046C4F81031FBF77BFC0028EA
:10DCA0003DF40AAE0127E9E70025D4F8083184F8ED
:10DCB000FF50D4F80C2120469847D4F82431294647
:10DCC0000133DAF80450C4F82431FFF758B8AA68D1
:10DCD0004146204600F0BAFA009A069BC4F8142187
:10DCE000002B3EF49BACFDF7D5BD5F25FFF70EBAC8
:10DCF0000025D4F8083184F8FF50D4F80C212046D0
:10DD00009847D4F8243129460133C4F82431FFF769
:10DD10007FBB4846424901F0D1FC20B13A4641461A
:10DD2000204601F083F8AB6841469A68204601F02E
:10DD3000BBF8FDF797BD0026D4F8083184F8FF60E2
:10DD4000D4F80C2120469847D4F8243131460133C9
:10DD5000C4F82431FFF786BB0025D4F8083184F8D5
:10DD6000FF50D4F80C2120469847D4F82431294696
:10DD70000133C4F82431FEF756BB0025D0F8083132
:10DD800080F8FF50D0F80C219847D4F82431294668
:10DD90000133C4F80051C4F82431FEF727BB4068B2
:10DDA00000283DF48BADFEF752B984F8FF00194608
:10DDB000D4F80C21D4F8083120469847D4F824210F
:10DDC0002B460132C4F82421FFF711BB73681A787F
:10DDD000012A00F0538196F800A0FFF7DDBA002574
:10DDE000D4F8083184F8FF50D4F80C212046984725
:10DDF000D4F8243129460133C4F82431FFF753BB4A
:10DE00005446FEF78CBE00BF5CBA0108C4B80108D6
:10DE1000CCB8010878BA010874BA010870BA0108D0
:10DE200064B801086A684146204601F03DF8204682
:10DE30000322E249FBF79EF9FDF72CBD14AB43F832
:10DE400048CD0396C4F81031FEF753B80027D4F834
:10DE5000083184F8FF70D4F80C2120469847D4F894
:10DE6000243139460133C4F824311BE40026D4F8A8
:10DE7000083184F8FF60D4F80C2120469847D4F884
:10DE8000243131460133C4F82431FFF788BB002523
:10DE9000D4F8083184F8FF50D4F80C212046984774
:10DEA000D4F8243129460133C4F8243110E6002681
:10DEB000D4F8083184F8FF60D4F80C212046984744
:10DEC000D4F8243131460133C4F82431FFF788BB3C
:10DED0005A68916801297DF48AAC526812783E2A0A
:10DEE0007DF485ACD4F80011FF290FD1D4F80831A6
:10DEF00084F8FF60D4F80C21204698473146D4F8C6
:10DF00002431C4F800610133C4F8243128234A1CA9
:10DF1000C4F80021635484F804316B68FDF767BCD2
:10DF20000025D4F8083184F8FF50D4F80C2120469D
:10DF30009847D4F8243129460133C4F82431FFF737
:10DF400009BBDBF804B0BBF1000F3EF4E8ADFDF710
:10DF5000BCBF029BC4F81031FDF7D4BF93684146A3
:10DF60001B782046292B1CBF0123C4F818315268A6
:10DF700000F09AFFFDF74CBC0026D4F8083184F875
:10DF8000FF60D4F80C2120469847D4F8243131465C
:10DF90000133C4F824317EE572684146204600F022
:10DFA00083FF4A464146204600F040FFFDF772BC21
:10DFB000D4F8083184F8FF60D4F80C212046984743
:10DFC000D4F8243131460133C4F82431FDF7A6BF1B
:10DFD0004A464146204600F067FF524641462046E9
:10DFE00000F024FF3A464146204600F05DFF2046FF
:10DFF00003227349FBF7BEF82A464146204600F04B
:10E0000053FFFDF747BC4F457FF66FAE5F2D7FF4A2
:10E010006CAEFF283FF67AA8D4F80011C5B2FF29EC
:10E020000FD1D4F8083184F8FF80D4F80C212046B1
:10E0300098470021D4F82431C4F800810133C4F892
:10E0400024314B1CC4F800314E46655484F8045109
:10E05000FFF766B8D4F8083184F8FF60D4F80C21D3
:10E0600020469847D4F8243131460133C4F8006182
:10E07000C4F82431FFF7E3BB9146E7E5B2681278B4
:10E08000292A08BF1E46A6E60025D4F8083184F8E0
:10E09000FF50D4F80C2120469847D4F82431294663
:10E0A0000133C4F80051C4F82431A9E50026D4F89E
:10E0B000083184F8FF60D4F80C2120469847D4F842
:10E0C000243131460133C4F80061C4F82431FDF72E
:10E0D000C2BB84F8FF00D4F80831D4F80C212046E4
:10E0E0009847D4F8243131460133C4F80061C4F8AC
:10E0F0002431FDF79EBB0026D4F8083184F8FF6078
:10E10000D4F80C2120469847D4F824313146013305
:10E11000C4F80061C4F824317FE5416800293DF46A
:10E12000CAAB0B78FEF7DEB9D0F80011FF290DD08D
:10E130002D234A1CC4F80021635484F8043104E5FB
:10E1400005222049FBF716F8FDF7A4BBD0F80831EB
:10E1500080F8FF70D0F80C219847D4F82431394664
:10E160000133C4F80071C4F82431E1E70025D4F884
:10E17000083184F8FF50D4F80C2120469847D4F891
:10E18000243129460133C4F80051C4F8243112E582
:10E190000027FFF710B90025D4F8083184F8FF50A4
:10E1A000D4F80C2120469847D4F82431294601336D
:10E1B000C4F80051C4F82431FDF765BBA8BA0108C2
:10E1C00064BA01087CBA01083746FFF7E6BB0025B0
:10E1D000D4F8083184F8FF50D4F80C212046984731
:10E1E000D4F8243129460133C4F80051C4F824314D
:10E1F000D3E4C9F8002004312046FBF7CBF900280E
:10E200007FF43CADFDF75ABBD4F8083184F8FF60C9
:10E21000D4F80C2120469847D4F8243131460133F4
:10E22000C4F80061C4F82431FEF700BC0123C4F82F
:10E230001831FDF72FBB18460744FFF781BB0020BC
:10E240000744FFF77DBB0746FFF7A7BB10B5D0F823
:10E25000283182B0C0F828D104468DE80C00FDF7C3
:10E260004BFA019BC4F8283102B010BD2DE9F047EC
:10E27000137882B0033B154604468846492B00F2CA
:10E280002982DFE813F0E90127022702270227028B
:10E290002702270227022702270227022702270236
:10E2A0002702270227022702270227022702270226
:10E2B0002702EE018401AA01EE018401AA01CF0127
:10E2C000DC016F008D009D00AC00D000F50027023E
:10E2D0002702270227021A0127025E0127022702CE
:10E2E00027022702270227022702270227022702E6
:10E2F00027022702270227022702270227022702D6
:10E3000027022702270227022702270227022702C5
:10E3100027022702270227024A00D64D4FF00008A5
:10E32000D0F8001105F1110708E00B460131BD429C
:10E33000C4F80011E65484F804612ED0FF2915F8C2
:10E34000016FF2D1D4F80831D4F80C2184F8FF80A1
:10E35000204698470121D4F8242100230A44C4F818
:10E360002421E4E7D0F80011FF2900F0FE814A1CC7
:10E370002023C4F80021635484F80431AB6841467B
:10E380001A46D4F82851C4F828D120468DE8280030
:10E39000FDF7B2F9019BC4F8283102B0BDE8F0875F
:10E3A00011F00405F9D1D0F80031FF2B00F02282E2
:10E3B0002A22591CC4F80011E25484F80421ECE725
:10E3C000D0F80011FF2900F0BF814A1C2623C4F8B1
:10E3D0000021635484F8043102B0BDE8F087D0F81E
:10E3E0000011A54D4FF00008AF1C08E00B460131AD
:10E3F000BD42C4F80011E65484F80461CDD0FF2971
:10E4000015F8016BF2D1D4F80831D4F80C2184F856
:10E41000FF80204698470121D4F8242100230A4494
:10E42000C4F82421E4E7954D4FF00008D0F800111E
:10E4300005F1080708E00B460131BD42C4F80011A0
:10E44000E65484F80461A8D0FF2915F8016FF2D1D1
:10E45000D4F80831D4F80C2184F8FF80204698477E
:10E460000121D4F8242100230A44C4F82421E4E73C
:10E47000834D4FF00008D0F8001105F10A0708E0BD
:10E480000B460131BD42C4F80011E65484F8046122
:10E4900083D0FF2915F8016BF2D1D4F80831D4F8F4
:10E4A0000C2184F8FF80204698470121D4F82421CC
:10E4B00000230A44C4F82421E4E790F80431282B0F
:10E4C0000BD0D0F80031FF2B00F02C812022591CFA
:10E4D000C4F80011E25484F804216B68D4F8285180
:10E4E00041461A46C4F828D120468DE82800FDF799
:10E4F00003F9644D019B0027D4F80011C4F82831BA
:10E5000005F1030809E00B4601314545C4F8001147
:10E51000E65484F804613FF440AFFF2915F8016B1D
:10E52000F1D1D4F80831D4F80C2184F8FF702046DA
:10E5300098470121D4F8242100230A44C4F8242157
:10E54000E3E7514E4FF00009D0F8001106F10A0A36
:10E5500009E00B4601315645C4F80011E75484F830
:10E56000047100F0C480FF2916F8017BF1D1D4F8C2
:10E570000831D4F80C2184F8FF90204698470121F7
:10E58000D4F8242100230A44C4F82421E3E73F4DB2
:10E590004FF00008D0F8001105F1090709E00B461B
:10E5A0000131BD42C4F80011E65484F804613FF41F
:10E5B000F4AEFF2915F8016FF1D1D4F80831D4F881
:10E5C0000C2184F8FF80204698470121D4F82421AB
:10E5D00000230A44C4F82421E3E72D4D4FF000083E
:10E5E000D0F80011AF1D09E00B460131BD42C4F85F
:10E5F0000011E65484F804613FF4CFAEFF2915F80A
:10E60000016BF1D1D4F80831D4F80C2184F8FF80E3
:10E61000204698470121D4F8242100230A44C4F855
:10E620002421E3E7D0F80031FF2B00F0D180202235
:10E63000591CC4F80011E25484F80421C2E6D0F851
:10E640000031FF2B00F0B2802022591CC4F80011C9
:10E65000E25484F80421C4E66B68D0F828511A46C5
:10E6600091E60C4D4FF00008D0F8001105F10907B4
:10E670001CE000BF4BBB010860BB010863BB010885
:10E6800070BB01087CBB010880BB010837BB0108D7
:10E6900044BB01082BBB01080B460131AF42C4F853
:10E6A0000011E65484F804613FF477AEFF2915F8B1
:10E6B000016FF1D1D4F80831D4F80C2184F8FF802F
:10E6C000204698470121D4F8242100230A44C4F8A5
:10E6D0002421E3E7D0F828312A46C0F828D1019355
:10E6E0000095FDF709F8019BC4F8283155E66B68E1
:10E6F000D4F828511A464146C4F828D120468DE85E
:10E700002800FCF7F9FFD4F80011019BFF29C4F899
:10E7100028313AD04A1C2923C4F80021635484F8D4
:10E7200004313AE600261946D0F80C21D0F8083119
:10E7300080F8FF609847D4F8242133460132C4F8AA
:10E740000061C4F82421C1E60025D4F80831D4F8CA
:10E750000C2184F8FF50204698470122D4F8243138
:10E7600029461344C4F8243130E60026D0F8083195
:10E77000D0F80C2180F8FF6098470122D4F82431AA
:10E7800031461344C4F82431F2E50025D4F80831A9
:10E79000D4F80C2184F8FF50204698470122D4F881
:10E7A000243129461344C4F82431B4E7002519461E
:10E7B000D0F80C21D0F8083180F8FF509847D4F8F1
:10E7C00024212B460132C4F80051C4F824213BE730
:10E7D00000251946D0F80C21D0F8083180F8FF50F8
:10E7E0009847D4F824212B460132C4F80051C4F8CC
:10E7F00024211CE71946D0F80C21D0F8083180F804
:10E80000FF509847D4F824212B460132C4F8005118
:10E81000C4F82421CCE500BF002A00F0A1802DE936
:10E82000F04F1E46D0F8183189B0054643BB0F465D
:10E8300014464FF0010802E0D5F8183103BBA36875
:10E84000DBB9626813782EB9A3F11C01042914D92D
:10E850004C2B12D0E168292BC4F80880D5F8109110
:10E86000C5F810110FD02A2B18D0022B21D0394611
:10E870002846FFF7FBFCC5F810912468002CDBD17B
:10E8800009B0BDE8F08F236808323946284600F009
:10E89000D9F9C5F8109109B0BDE8F08F23680432AA
:10E8A0003946284600F0F2F8C5F8109109B0BDE8E5
:10E8B000F08F0026D5F81481C5F8146152683946E6
:10E8C0002846FFF7C3FC17F0040AC5F8148123D0CB
:10E8D000D5F80011FF2900F0C1804A1C2E23C5F88D
:10E8E00000216B5485F8043163689C682378462BBB
:10E8F00037D0A3F11C02042A0BD94C2B09D0224695
:10E9000039462846FFF7A2FCC5F8109109B0BDE8CA
:10E91000F08F64682378ECE7584ED5F8001106F1C3
:10E92000020B09E00B4601315E45C5F8001105F800
:10E93000038085F80481D7D0FF2916F8018BF1D127
:10E94000D5F80831D5F80C2185F8FFA0284698475E
:10E950000121D5F8242100230A44C5F82421E3E746
:10E960007047474E4FF0000BD5F8001106F10D0A25
:10E9700009E00B460131B245C5F8001105F80380E6
:10E9800085F8048113D0FF2916F8018BF1D1D5F851
:10E990000831D5F80C2185F8FFB0284698470121A9
:10E9A000D5F8242100230A44C5F82421E3E7A2680E
:10E9B00001A80132334907F091FC01A807F0B4FC2B
:10E9C00028B301AE4FF0000BD5F8001106EB000A9A
:10E9D00009E00B460131B245C5F8001105F8038086
:10E9E00085F8048115D0FF2916F8018BF1D1D5F8EF
:10E9F0000831D5F80C2185F8FFB028469847012149
:10EA0000D5F8242100230A44C5F82421E3E7D5F8EA
:10EA100000111D4E4FF0000B06F1030A0AE00B46F1
:10EA20000131B245C5F8001105F8038085F804816D
:10EA30003FF46FAFFF2916F8018BF0D1D5F80831FC
:10EA4000D5F80C2185F8FFB0284698470121D5F864
:10EA5000242100230A44C5F82421E2E7D5F808312F
:10EA6000D5F80C2185F8FF60284698470122D5F893
:10EA7000243131461344C5F824312FE7ACB80108DE
:10EA8000B0B801085CB80108C0B801082DE9F84F1A
:10EA900004460F46904663B11E461A46936893B3E8
:10EAA0001268002AFAD11346394632462046FFF74B
:10EAB000B3FED4F80011FF2900F08D804B1C2022FA
:10EAC000FF2BC4F80031625484F8042168D05B2223
:10EAD000591CC4F80011E25484F80421D8F800202D
:10EAE0002AB139462046FFF7B1FBD4F80011FF29BF
:10EAF00000F082804A1C5D23C4F80021635484F82E
:10EB00000431BDE8F88F526812782A2A3FD0DFF826
:10EB100030911D46D4F8001109F1020B0AE00B46B2
:10EB2000CB4501F10101C4F8001104F803A084F8F9
:10EB300004A11AD0FF2919F801ABF0D1D4F808319B
:10EB4000D4F80C2184F8FF50204698470121002377
:10EB5000D4F82421CB450A44C4F82421C4F8001178
:10EB600004F803A084F804A1E4D100233246394616
:10EB70002046FFF751FED4F80031FF2B4DD0591C31
:10EB80002922C4F80011E25484F8042193E73246A4
:10EB900039462046FFF740FED4F80031FF2B96D1CE
:10EBA0000022194684F8FF20D4F80831D4F80C214B
:10EBB000204698475B230121237084F80431D4F860
:10EBC0002431D8F800200B44C4F82431C4F80011D3
:10EBD000002A86D18EE70025D4F80831D4F80C211C
:10EBE00084F8FF50204698470123D4F82421294671
:10EBF0001A44C4F8242162E70025D4F80831D4F877
:10EC00000C2184F8FF50204698470122D4F8243183
:10EC100029461344C4F824316DE700251946D4F879
:10EC20000C21D4F8083184F8FF5020469847012180
:10EC3000D4F824212B460A44C4F82421A0E700BFBD
:10EC4000A4BA01082DE9F043044683B00E461746E6
:10EC50001D464BB39B683BBB2A460120DFF8C8E149
:10EC600006E011F4606F5BD11268EAB19368DBB91A
:10EC700053681B78193BDBB2122B00FA03F1F3D86F
:10EC800011EA0E0FEDD094F80431202B4ED0D4F8B9
:10EC90000031FF2B00F0B580591C2022C4F8001170
:10ECA000E25484F8042143E00022D4F8148113468E
:10ECB000C4F8142131462A462046FFF7ADFDD4F8AA
:10ECC0000011FF2956D04B1C2822C4F80031625491
:10ECD00084F80421386878B1D4F8283102460090CD
:10ECE000C4F828D1314620460193FCF705FD019A6E
:10ECF000D4F80031C4F82821FF2B4DD05A1C29200C
:10ED0000C4F800213146E0542A4684F80401012366
:10ED10002046FFF781FDC4F8148103B0BDE8F083FD
:10ED200094F8043103F0FD02282AAED1D4F8001182
:10ED3000FF2954D04A1C28234FF00009C4F80021B1
:10ED40006354D4F8148184F80431C4F814914B4608
:10ED50002A4631462046FFF75FFDD4F80031FF2BED
:10ED60002CD0591C2922FF29C4F80011E25484F840
:10ED70000421A8D14FF00009D4F80831D4F80C21AF
:10ED800084F8FF90204698470123D4F8242149466F
:10ED90001A44C4F8242197E700271946D4F80C2117
:10EDA000D4F8083184F8FF70204698470122D4F83F
:10EDB00024113B461144C4F82411A0E71946D4F8A5
:10EDC0000C21D4F8083184F8FF902046984701219F
:10EDD000D4F824214B460A44C4F82421C2E74FF05A
:10EDE0000008D4F80831D4F80C2184F8FF802046BC
:10EDF00098470122D4F8243141461344C4F8243101
:10EE000099E74FF000081946D4F80C21D4F80831DE
:10EE100084F8FF80204698470121D4F824214346F6
:10EE20000A44C4F8242138E7073104002DE9F041F1
:10EE3000157882B0312D134604460DD0D0F82851F4
:10EE4000C0F828D18DE82800FCF756FC019BC4F8D7
:10EE5000283102B0BDE8F08153689F685D68002FDB
:10EE6000F7D04FF00008D0F800112F4408E00B460F
:10EE70000131BD42C4F80011E65484F80461E8D0C1
:10EE8000FF2915F8016BF2D1D4F80831D4F80C2120
:10EE900084F8FF80204698470121D4F824210023DC
:10EEA0000A44C4F82421E4E7F0B5137883B0012BB9
:10EEB00015460E46044629D9302B27D0062B25D0DF
:10EEC000D0F80011FF2931D04A1C2823C4F80021B2
:10EED0006354D4F82871314684F804312A46C4F8C2
:10EEE00028D120468DE8A000FCF706FCD4F80011DC
:10EEF000019BFF29C4F8283128D04A1C2923C4F8D3
:10EF00000021635484F8043103B0F0BDD4F82831F3
:10EF100031462A46C4F828D1204601930095FCF7D3
:10EF2000EBFB019BC4F8283103B0F0BD0027D4F8F7
:10EF30000831D4F80C2184F8FF7098470122D4F8E6
:10EF4000243139461344C4F82431BEE70025D4F8EF
:10EF50000831D4F80C2184F8FF502046984701224C
:10EF6000D4F8243129461344C4F82431C6E700BF3D
:10EF70002DE9F84F526812681578662D02D00020EE
:10EF8000BDE8F88F1B68D0F82071D3F80890D3F84B
:10EF9000048099F800300E463B2B4FF0FF3304BF3E
:10EFA000D9F80850D9F80490C0F82031537818BF28
:10EFB00000254C3B0446262B2BD8DFE803F0902A93
:10EFC0002A2A2A2A902A2A2A2A2A2A2A2A2A2A2A3B
:10EFD0002A2A2A2A2A2A2A2A2A2A2A2A2A2A6A2A51
:10EFE0002A2A2A2A2F00424631462046FFF71EFFD2
:10EFF0004A4631462046FFF757FFD4F80011FF2953
:10F0000000F0B0804A1C2923C4F80021635484F81E
:10F010000431C4F820710120BDE8F88FD0F8001148
:10F02000FF2900F0C2804A1C2823C4F80021204692
:10F0300063544A46314684F80431644DFFF734FF87
:10F04000424631462046FFF7F1FE4FF0000AD4F861
:10F05000001105F1040808E00B460131A845C4F889
:10F060000011E65484F80461D3D0FF2915F8016B30
:10F07000F2D1D4F80831D4F80C2184F8FFA020464E
:10F0800098470121D4F8242100230A44C4F82421FC
:10F09000E4E74F4DD0F8001105F1040B09E00B46F1
:10F0A00001315D45C4F8001104F803A084F804A1FF
:10F0B00099D0FF2915F801ABF1D14FF00003D4F836
:10F0C0000C2184F8FF302046D4F8083198470121FC
:10F0D000D4F8242100230A44C4F82421E1E7D0F81D
:10F0E0000011FF294FD02823481C4A46C4F80001CC
:10F0F000DFF8E09063542046314684F80431FFF78E
:10F10000D3FE314642462046FFF790FE09F1030B3D
:10F11000D4F8001109E00B460131CB45C4F80011C9
:10F1200004F803A084F804A115D0FF2919F801AB55
:10F13000F1D14FF00003D4F80C2184F8FF302046C1
:10F14000D4F8083198470121D4F8242100230A4437
:10F15000C4F82421E1E7424631462046FFF766FE27
:10F160002A4646E70025D4F80831D4F80C2184F863
:10F17000FF50204698470122D4F8243129461344F1
:10F18000C4F824313FE74FF0000AD0F8083180F886
:10F19000FFA0D0F80C219847D4F824315146013310
:10F1A000C4F800A1C4F824319DE70025D0F8083147
:10F1B000D0F80C2180F8FF5098470122D4F8243170
:10F1C00029461344C4F824312EE700BF94BB01083C
:10F1D0008CBB0108A8BA01082DE9F04FE7B090F800
:10F1E000009000AFB9F15F0F05467960164600F058
:10F1F000F3800822BE49284607F0C4F848B92B7AA4
:10F200002E2B00F0D8805F2B00F0D580242B00F04F
:10F21000D2804FF00008284607F086F84FEA400AEF
:10F22000830003EB0A0292000832ADEB020D0024CA
:10F23000EB4611220A3323F00703ADEB030DB8634D
:10F24000B8F1010F2844C7F824B0C7F830D0C7F888
:10F250002CA07D613D62B861FA61BC627C63FC6395
:10F260003C647C64BC64FC6400F0BD80C0F0D18070
:10F27000EA7AB8F1020F05F10B0314BF4FF044090D
:10F280004FF043095F2A3B6200F0B68018463B60AE
:10F2900007F04AF8BAF1000F3B6840F3C38001223F
:10F2A000BA62002800F0BE8000228BF800205A4687
:10F2B000CBF80430CBF808004946002307F11400CE
:10F2C000F9F73AFE3C6A0546204607F02DF8231868
:10F2D0003B6214F80090B9F1000F40F08780002DD8
:10F2E00000F084807B6807F150042A4607F5C2715C
:10F2F00007F5C870C4F80831C4F80C61C4F800916F
:10F3000084F80491C4F81091C4F81491C4F82091C1
:10F31000C4F82491C4F81891C4F81C91C4F8289139
:10F32000C4F82C91C4F83091C4F83491C4F83891E1
:10F33000C4F83C91C4F84091F9F7CAFED4F83421DE
:10F34000E846D3000833ADEB030D6846D4F840110E
:10F35000D4F8283101FB02F1CA000832ADEB020DEE
:10F3600007F10C062A46C4F82C01C4F840112046C7
:10F370001121C4F838D13B61FD60C4F84491C4F850
:10F380002861FCF7B9F93B692046C4F82831D4F864
:10F390000011C54604F80190D4F80831D4F80C21C6
:10F3A0009847D4F8180107F5CE77B0FA80F04009F5
:10F3B000BD46BDE8F08F6B7A442B02D0492B7FF419
:10F3C00028AFAA7A5F2A7FF424AF492B14BF4FF0ED
:10F3D00003084FF002081EE743785A2B7FF409AF69
:10F3E0004FF0010817E7B9F15F0F1DD0002007F5B6
:10F3F000CE77BD46BDE8F08F2A7B5A2A7FF446AF10
:10F400000D35214607F114003D62FBF729FE024647
:10F4100052E707F11400FBF713F83B6A054693F82F
:10F42000009058E7002247E76B785A2BDED102356F
:10F43000414607F114003D62FBF712FEFB690546E9
:10F44000DB0750D5386A90F80090B9F12E0F7FF4A1
:10F4500042AF4378A3F16102192A38D95F2B36D025
:10F46000303B092B3FD8024603782E2B11D153781D
:10F47000303B092B0DD893780232A3F130010929D2
:10F48000F3D812F8013FA3F130010929F9D92E2B45
:10F49000EDD0B96AFB6A3A62994216DAD7F824E0ED
:10F4A0004B1C01EB4101BB621EEB81030DD0121A14
:10F4B0000BD00EF8214058609A602A464D2107F182
:10F4C0001400F9F739FD0546BCE70023F5E7811C78
:10F4D0000A4611F8013BA3F1610EBEF1190FF7D9ED
:10F4E0005F2BF5D0C1E73B6A93F80090F3E600BFCD
:10F4F00038B801082DE9F04184B078B301B16AB39E
:10F50000002416460D466A4627491F46009401947A
:10F5100002940394FFF760FE00283ED0039BD3B112
:10F520004FF00108009C5CB33DB3204606F0FCFEA2
:10F53000336898421BD2421C2146284600F048F806
:10F54000204606F097F82C460FB100233B6020467A
:10F5500004B0BDE8F081DDF80880E3E713B30024D0
:10F560006FF0020220461A6004B0BDE8F081284620
:10F5700006F080F8C6F80080E6E7002EFAD1E3E74F
:10F5800087B1B8F1010F04D06FF0010300243B6094
:10F59000DDE74FF0FF333B60D9E7009806F06AF8EB
:10F5A000002FF1D10024D2E75996000860B108B5C8
:10F5B00039B1FFF711FE00280CBF6FF001000020E9
:10F5C00008BD6FF0020008BD6FF00200704700BF79
:10F5D000844641EA000313F0030349D1403A23D3A0
:10F5E0000B6803604B6843608B688360CB68C360C3
:10F5F0000B6903614B6943618B698361CB69C361AB
:10F600000B6A03624B6A43628B6A8362CB6AC36292
:10F610000B6B03634B6B43638B6B8363CB6BC3637A
:10F6200040304031403ADBD230320BD30B680360BC
:10F630004B6843608B688360CB68C36010301031C7
:10F64000103AF3D20C3205D351F8043B40F8043B96
:10F65000043AF9D2043208D0D2071CBF11F8013B9A
:10F6600000F8013B01D30B8803806046704700BF60
:10F67000082A13D38B07B1D010F00303AED0C3F127
:10F680000403D21ADB071CBF11F8013B00F8013B51
:10F69000A4D331F8023B20F8023B9FE7043AD9D3C8
:10F6A000013A11F8013B00F8013BF9D20B780370E5
:10F6B0004B7843708B7883706046704780EA010C0A
:10F6C0001CF0030F37D110F0030C20F0030021F0E1
:10F6D000030150F8042B08BF51F8043B0ED08CF006
:10F6E000030C6FF07F434FEACC0C23FA0CFC51F86B
:10F6F000043B42EA0C0243EA0C0300BFA2F1013CC6
:10F700009A4201BF2CEA020C1CF0803F50F8042BF7
:10F7100051F8043BF2D04FEA02604FEA122201286E
:10F7200028BFB0EB036F08BF1B0AF4D003F0FF0340
:10F73000000EC01A704710F0030F0AD010F8012B0A
:10F7400011F8013B012A28BF9A42F4D0A2EB030032
:10F7500070474DF8045D50F8042B01F0030521F0CB
:10F76000030151F8043B022D26D04DD822F07F45ED
:10F77000B5EB132FA2F1013C2CEA020C0DD11CF0C9
:10F78000803C08BF51F8043B0AD185EA0205B5EB7D
:10F79000036F0CD150F8042BE8E74FEA13235BE02A
:10F7A0003CF07F4C54D10B784FEA126554E04FEA9D
:10F7B000126503F0FF034FE04FEA0245A2F1013C5E
:10F7C0004FEA15452CEA020CB5EB134F18D11CF08B
:10F7D000803C08BF51F8043B07D185EA0205B5EB30
:10F7E000034F09D150F8042BE6E75FEA0C4C2FD108
:10F7F0000B884FEA12452FE04FEA03434FEA1245C8
:10F800004FEA134328E000BF02F0FF05B5EB136F8A
:10F81000A2F1013C2CEA020C0DD11CF0803C08BF87
:10F8200051F8043B0AD185EA0205B5EB032F0AD152
:10F8300050F8042BE8E74FEA13630DE012F0FF0FD6
:10F8400006D051F8043B4FEA122523F07F4303E032
:10F850004FF0000020BC704705F0FF0203F0FF00EE
:10F86000012828BF904204BF2D0A1B0AF4D0A2EB46
:10F87000000020BC704700BF81F0004102E000BFE3
:10F8800083F0004330B54FEA41044FEA430594EA60
:10F89000050F08BF90EA020F1FBF54EA000C55EA9B
:10F8A000020C7FEA645C7FEA655C00F0E2804FEA6C
:10F8B0005454D4EB5555B8BF6D420CDD2C4480EA4E
:10F8C000020281EA030382EA000083EA010180EA7E
:10F8D000020281EA0303362D88BF30BD11F0004FCC
:10F8E0004FEA01314FF4801C4CEA113102D0404202
:10F8F00061EB410113F0004F4FEA03334CEA13333D
:10F9000002D0524263EB430394EA050F00F0A78054
:10F91000A4F10104D5F1200E0DDB02FA0EFC22FA4F
:10F9200005F2801841F1000103FA0EF2801843FA43
:10F9300005F359410EE0A5F120050EF1200E012A34
:10F9400003FA0EFC28BF4CF0020C43FA05F3C01872
:10F9500051EBE37101F0004507D54FF0000EDCF1EB
:10F96000000C7EEB00006EEB0101B1F5801F1BD394
:10F97000B1F5001F0CD349085FEA30004FEA3C0C98
:10F9800004F101044FEA445212F5800F80F09A808E
:10F99000BCF1004F08BF5FEA500C50F1000041EB92
:10F9A000045141EA050130BD5FEA4C0C404141EB96
:10F9B000010111F4801FA4F10104E9D191F0000FBD
:10F9C00004BF01460020B1FA81F308BF2033A3F140
:10F9D0000B03B3F120020CDA0C3208DD02F1140C37
:10F9E000C2F10C0201FA0CF021FA02F10CE002F172
:10F9F0001402D8BFC2F1200C01FA02F120FA0CFC6B
:10FA0000DCBF41EA0C019040E41AA2BF01EB0451B3
:10FA1000294330BD6FEA04041F3C1CDA0C340EDCB1
:10FA200004F11404C4F1200220FA04F001FA02F3F4
:10FA300040EA030021FA04F345EA030130BDC4F1B2
:10FA40000C04C4F1200220FA02F001FA04F340EAA7
:10FA50000300294630BD21FA04F0294630BD94F058
:10FA6000000F83F4801306BF81F480110134013D3F
:10FA70004EE77FEA645C18BF7FEA655C29D094EAB0
:10FA8000050F08BF90EA020F05D054EA000C04BF2E
:10FA90001946104630BD91EA030F1EBF0021002019
:10FAA00030BD5FEA545C05D14000494128BF41F0B8
:10FAB000004130BD14F580043CBF01F5801130BD1C
:10FAC00001F0004545F0FE4141F470014FF00000A7
:10FAD00030BD7FEA645C1ABF194610467FEA655C58
:10FAE0001CBF0B46024650EA013406BF52EA0335FA
:10FAF00091EA030F41F4002130BD00BF90F0000FE8
:10FB000004BF0021704730B54FF4806404F1320423
:10FB10004FF000054FF0000150E700BF90F0000FDC
:10FB200004BF0021704730B54FF4806404F1320403
:10FB300010F0004548BF40424FF000013EE700BFD3
:10FB400042004FEAE2014FEA31014FEA02701FBF63
:10FB500012F07F4393F07F4F81F06051704792F035
:10FB6000000F14BF93F07F4F704730B54FF46074AF
:10FB700001F0004521F0004120E700BF50EA0102FA
:10FB800008BF704730B54FF000050AE050EA0102A7
:10FB900008BF704730B511F0004502D5404261EB17
:10FBA00041014FF4806404F132045FEA915C3FF458
:10FBB000DCAE4FF003025FEADC0C18BF03325FEAF1
:10FBC000DC0C18BF033202EBDC02C2F1200300FAA6
:10FBD00003FC20FA02F001FA03FE40EA0E0021FACB
:10FBE00002F11444C1E600BF70B54FF0FF0C4CF4B5
:10FBF000E06C1CEA11541DBF1CEA135594EA0C0F6B
:10FC000095EA0C0F00F0DEF82C4481EA030621EAA5
:10FC10004C5123EA4C5350EA013518BF52EA0335E0
:10FC200041F4801143F4801338D0A0FB02CE4FF092
:10FC30000005E1FB02E506F00042E0FB03E54FF0C2
:10FC40000006E1FB03569CF0000F18BF4EF0010EBA
:10FC5000A4F1FF04B6F5007F64F5407404D25FEAB6
:10FC60004E0E6D4146EB060642EAC62141EA555169
:10FC70004FEAC52040EA5E504FEACE2EB4F1FD0CAB
:10FC800088BFBCF5E06F1ED8BEF1004F08BF5FEA29
:10FC9000500E50F1000041EB045170BD06F00046DB
:10FCA00046EA010140EA020081EA0301B4EB5C0488
:10FCB000C2BFD4EB0C0541EA045170BD41F4801180
:10FCC0004FF0000E013C00F3AB8014F1360FDEBFA5
:10FCD000002001F0004170BDC4F10004203C35DA81
:10FCE0000C341BDC04F11404C4F1200500FA05F304
:10FCF00020FA04F001FA05F240EA020001F00042A5
:10FD000021F0004110EBD37021FA04F642EB06011A
:10FD10005EEA430E08BF20EAD37070BDC4F10C0444
:10FD2000C4F1200500FA04F320FA05F001FA04F208
:10FD300040EA020001F0004110EBD37041F10001F4
:10FD40005EEA430E08BF20EAD37070BDC4F12005FF
:10FD500000FA05F24EEA020E20FA04F301FA05F267
:10FD600043EA020321FA04F001F0004121FA04F20F
:10FD700020EA020000EBD3705EEA430E08BF20EADF
:10FD8000D37070BD94F0000F0FD101F00046400019
:10FD900041EB010111F4801F08BF013CF7D041EA9B
:10FDA000060195F0000F18BF704703F0004652009F
:10FDB00043EB030313F4801F08BF013DF7D043EA70
:10FDC0000603704794EA0C0F0CEA135518BF95EA26
:10FDD0000C0F0CD050EA410618BF52EA4306D1D1AD
:10FDE00081EA030101F000414FF0000070BD50EACC
:10FDF000410606BF1046194652EA430619D094EA56
:10FE00000C0F02D150EA013613D195EA0C0F05D13F
:10FE100052EA03361CBF104619460AD181EA030193
:10FE200001F0004141F0FE4141F470014FF000004B
:10FE300070BD41F0FE4141F4780170BD70B54FF0E6
:10FE4000FF0C4CF4E06C1CEA11541DBF1CEA135566
:10FE500094EA0C0F95EA0C0F00F0A7F8A4EB050448
:10FE600081EA030E52EA03354FEA013100F088803F
:10FE70004FEA03334FF0805545EA131343EA126308
:10FE80004FEA022245EA111545EA10654FEA0026BD
:10FE90000EF000419D4208BF964244F1FD0404F576
:10FEA000407402D25B084FEA3202B61A65EB0305D2
:10FEB0005B084FEA32024FF480104FF4002CB6EB8F
:10FEC000020E75EB030E22BFB61A754640EA0C000F
:10FED0005B084FEA3202B6EB020E75EB030E22BF4F
:10FEE000B61A754640EA5C005B084FEA3202B6EB90
:10FEF000020E75EB030E22BFB61A754640EA9C004F
:10FF00005B084FEA3202B6EB020E75EB030E22BF1E
:10FF1000B61A754640EADC0055EA060E18D04FEADC
:10FF2000051545EA16754FEA06164FEAC30343EA7C
:10FF300052734FEAC2025FEA1C1CC0D111F4801F49
:10FF40000BD141EA00014FF000004FF0004CB6E742
:10FF500011F4801F04BF01430020B4F1FD0C88BFE1
:10FF6000BCF5E06F3FF6AFAEB5EB030C04BFB6EBEC
:10FF7000020C5FEA500C50F1000041EB045170BDDF
:10FF80000EF0004E4EEA113114EB5C04C2BFD4EB0C
:10FF90000C0541EA045170BD41F480114FF0000E90
:10FFA000013C90E645EA060E8DE60CEA135594EA0C
:10FFB0000C0F08BF95EA0C0F3FF43BAF94EA0C0F0F
:10FFC0000AD150EA01347FF434AF95EA0C0F7FF484
:10FFD00025AF104619462CE795EA0C0F06D152EAD8
:10FFE00003353FF4FDAE1046194622E750EA4106BC
:10FFF00018BF52EA43067FF4C5AE50EA41047FF4CD
:020000040801F1
:100000000DAF52EA43057FF4EBAE12E74FF0FF3C31
:1000100006E000BF4FF0010C02E000BF4FF0010C02
:100020004DF804CD4FEA410C7FEA6C5C4FEA430C7B
:1000300018BF7FEA6C5C1BD001B050EA410C0CBFCA
:1000400052EA430C91EA030F02BF90EA020F00202C
:10005000704710F1000F91EA030F58BF994208BF93
:1000600090422CBFD8176FEAE37040F00100704750
:100070004FEA410C7FEA6C5C02D150EA013C07D1A7
:100080004FEA430C7FEA6C5CD6D152EA033CD3D0F2
:100090005DF8040B704700BF8446104662468C46EC
:1000A0001946634600E000BF01B5FFF7B7FF00281F
:1000B00048BF10F1000F01BD4DF808EDFFF7F4FF48
:1000C0000CBF012000205DF808FB00BF4DF808EDD3
:1000D000FFF7EAFF34BF012000205DF808FB00BFF6
:1000E0004DF808EDFFF7E0FF94BF012000205DF818
:1000F00008FB00BF4DF808EDFFF7CEFF94BF0120CD
:1001000000205DF808FB00BF4DF808EDFFF7C4FFC5
:1001100034BF012000205DF808FB00BF4FEA410C0E
:100120007FEA6C5C02D150EA013C0AD14FEA430CF1
:100130007FEA6C5C02D152EA033C02D14FF000002E
:1001400070474FF0010070474FEA410212F500126C
:1001500015D211D56FF47873B3EB625212D94FEA0E
:10016000C12343F0004343EA505311F0004F23FAF8
:1001700002F018BF404270474FF00000704750EA4D
:10018000013005D111F0004008BF6FF0004070470A
:100190004FF00000704700BF53B94AB9002908BFAB
:1001A00000281CBF4FF0FF314FF0FF3001F000B9C5
:1001B000ADF1080C6DE904CE00F006F8DDF804E0BE
:1001C000DDE9022304B070472DE9F0478C460E4666
:1001D0000446089D002B50D18A4217466CD9B2FACA
:1001E00082FEBEF1000F0BD0CEF1200C01FA0EF60C
:1001F00020FA0CFC02FA0EF74CEA060C00FA0EF498
:100200003A0CBCFBF2F9BBB202FB19CC09FB03FAB6
:100210004FEA144848EA0C46B2450AD9F61909F1E2
:10022000FF3180F02581B24540F22281A9F1020917
:100230003E44A6EB0A06B6FBF2F002FB106600FB9A
:1002400003F3A4B244EA0644A34209D9E41900F135
:10025000FF3280F00B81A34240F2088102383C4417
:100260000021E41A40EA0940002D62D0002324FA5C
:100270000EF42C606B60BDE8F0878B4207D9002D2F
:1002800055D0002185E841000846BDE8F087B3FA63
:1002900083F1002940F08F80B34202D3824200F202
:1002A000FC80841A66EB03060120B446002D40D082
:1002B00085E81010BDE8F08712B90127B7FBF2F707
:1002C000B7FA87FEBEF1000F35D10121F61B4FEAC8
:1002D000174C1FFA87F8B6FBFCF20CFB126608FB02
:1002E00002F0230C43EA0646B04207D9F61902F1A0
:1002F000FF3302D2B04200F2D2801A46361AB6FB61
:10030000FCF00CFB106608FB00F8A3B243EA0644BD
:10031000A04507D9E41900F1FF3302D2A04500F24D
:10032000B9801846A4EB080440EA02409CE729463D
:100330002846BDE8F08707FA0EF7CEF1200326FA2B
:1003400003F24FEA174CB2FBFCF11FFA87F80CFBE3
:10035000112206FA0EF620FA03F301FB08F93343E3
:100360001E0C46EA0246B14500FA0EF409D9F61908
:1003700001F1FF3280F08C80B14540F28980023972
:100380003E44A6EB0906B6FBFCF00CFB106200FB3A
:1003900008F99EB246EA0246B14507D9F61900F1BE
:1003A000FF3371D2B1456FD902383E44A6EB09063E
:1003B00040EA01418FE7C1F1200722FA07F88B409C
:1003C00048EA030326FA07F44FEA134EB4FBFEF99A
:1003D0001FFA83FC0EFB19448E4020FA07F809FB34
:1003E0000CFA48EA06084FEA184646EA0444A245D1
:1003F00002FA01F200FA01F608D9E41809F1FF3017
:1004000044D2A24542D9A9F102091C44A4EB0A0432
:10041000B4FBFEF00EFB104400FB0CFC1FFA88F846
:1004200048EA0444A44507D9E41800F1FF3E29D264
:10043000A44527D902381C4440EA0940A0FB0289A0
:10044000A4EB0C0CCC45C246CE4615D312D055B108
:10045000B6EB0A036CEB0E0606FA07F7CB401F4318
:10046000CE402F606E600021BDE8F0871046F7E6B1
:100470008946DEE64645EAD2B8EB020A69EB030E8E
:100480000138E4E77046D7E718468FE78146BDE7B5
:10049000114676E702383C4444E7084606E7023A4C
:1004A0003E442BE703685A004CBF43F0004323F05F
:1004B00000431844704700BF61B32DE9F84F01F1C4
:1004C000FF3A90460646D146002707EB090404EBA5
:1004D000D4746410E50071190846FFF7E3FFA245E4
:1004E000834605F10800304409D0FFF7DBFFC34520
:1004F00000F1FF3005D8404509D2671CE5E7C34548
:1005000005D9A74202D004F1FF39DEE700210846F1
:10051000BDE8F88F08467047012807D0022807D0A9
:10052000044B00280CBF1846002070470248704753
:1005300002487047290C01082D0C0108310C0108F4
:1005400030B5254B83B004468D1E73B301A92846F0
:10055000AFF3008018B301992A46FFF7ADFF0146BB
:10056000E8B1FFF79FFF4B68A064012B11D0002B6F
:1005700022DB081DFFF796FF0023E0642365036874
:10058000002B1EDBFFF78EFF00232061184603B00F
:1005900030BD052300221846226103B030BD092377
:1005A00000221846226103B030BD0C4B0C4918469E
:1005B000C91AC9100191CFE70123081DE064236522
:1005C000DDE7C3F30360FFF7A7FF0028206114BF36
:1005D00000230923DAE700BF000000003CC4010843
:1005E00064C60108036810B5DA07044606D49B0701
:1005F00000F1480009D500F057FC2368590709D5D8
:100600001A070ED5DB0613D510BD00F045FC236894
:100610005907F5D404F1D00000F04EFC23681A0706
:10062000F0D404F5A87000F04FFC2368DB06EBD48F
:1006300004F5E870BDE8104000F08ABC036803B11F
:1006400003441846704700BF09207047704700BF39
:1006500070B504460D4608E02A6C236962612146A4
:100660002A4601209847082808D1296C2046FFF720
:1006700067FF06460028EFD004F08CFD0728FBD169
:100680003046296CFFF7E2FF281D00F0F9FB00BFA0
:100690002DE9F04705460027ADF5727D03AC0E1D30
:1006A00092460FCE0FC40FCE0FC40FCE0FC496E8E4
:1006B0000F00D5F80C80D5F8189084E80F0002AC34
:1006C0002846216C2760FFF73BFFBAF1000F074671
:1006D00014BF0A2609267FB1A36B46F010018DE8EE
:1006E00010022A46636401202B46C04778BB384677
:1006F0000DF5727DBDE8F087236C4FF4F0726B61ED
:1007000021467AA8FEF764FF2B697AAA294630466B
:100710009847889B82468DE81002314663642A46DA
:100720002B460120C04790B94FF4F0727AA92046B9
:10073000FEF74EFFBAF1080F06D1216C2846FFF7ED
:10074000FFFE09260746C6E7BAF1070F05D00927BD
:1007500038460DF5727DBDE8F0873846216CFFF70D
:1007600075FF03A800F08CFB406C7047F0B54FF0AC
:10077000FF3ECB6BF9B00B640E1D01AD0F46044676
:100780000FCE0FC50FCE0FC50FCE0FC596E80F00C9
:1007900085E80F00CDF800E006E023696A462146AF
:1007A00098470828054608D110992046FFF7C8FE4B
:1007B0000028F2D0092079B0F0BD6846FFF712FF9B
:1007C000062DF7D139462046FFF742FF30B4DD6BE6
:1007D000C160826119461D64002230BC58E700BF29
:1007E00070B54369C6680B6426B10122FFF750FF5C
:1007F00004F0D0FC03690A4604460D460146022077
:100800009847072807D0082803D129462046FFF734
:100810001FFF04F0BFFC3046296CFFF717FF281DAF
:1008200000F02EFBC2682AB110B4CC6B00220C641D
:1008300010BC2DE79AE700BF704700BF836813B173
:10084000014601201847704700B5042907D8DFE8A2
:1008500001F00309060909000BB90F2A05D9022086
:100860005DF804FB01205DF804FB00EB8202526896
:100870001846019B1A605DF804FB00BF002310B509
:1008800084B003AC0A4600941946FFF7DDFF0398D5
:1008900004B010BD00B5042907D8DFE801F0030952
:1008A000060909000BB90F2A05D902205DF804FBDF
:1008B00001205DF804FB019900EB820209681846EB
:1008C00051605DF804FB00BF002310B584B004AC98
:1008D00044F8042D00940A461946FFF7DBFF04B0E4
:1008E00010BD00BFF0B54FF0FF3ED36BADF50F7DEF
:1008F0001364151D17AC07460E460FCD0FC40FCD60
:100900000FC40FCD0FC495E80F0084E80F00CDF899
:1009100058E012E00C2116A86A46FFF7D5FF3146D1
:1009200016A8B84778B9049B16AA694608209847C4
:100930000528044608D0092805D026996846FFF7FF
:10094000FFFD0028E6D0092416A8FFF74BFE20463D
:100950000DF50F7DF0BD00BF2DE9F04FCC6C914639
:1009600022688BB004340D460792089400F0030B04
:100970001E46002B60D10323120207928DF82560DA
:100980008DF824302B6DBBF1020F08BFAC6B13F058
:10099000010340D1019300F008030393D4F80080D1
:1009A000B8F1000F39D0022E43D0B4F80080678828
:1009B0000434AB6C27F0010A0F2148469A44FFF734
:1009C0005DFF824533D828F001039A4450452CBF7F
:1009D000002001207F0007F0020708F0010847EA25
:1009E0000807012F3ED035D3022F1CD1236823F0F6
:1009F00000420292BBF1000F76D128B10399002981
:100A00007ED0002A00F0A680002B77DB029B01330A
:100A100004EB8304C2E700230193022E3EDDFFF7BF
:100A200013FE002840D009200BB0BDE8F08F002055
:100A3000D0E767680834BCE7022BA3DC0221130C63
:100A40008DF825301204DBB204EB830407928DF895
:100A5000241097E7BBF1000F02D0002840F0BD80C2
:100A600004349BE7BBF1000F25D1A8B194E80C003A
:100A7000991C4FEAD272D6D005F158010133069184
:100A800000F0A380201DFFF7D9FD06AB01462846E4
:100A900004F06EF9002877D108347FE707A94846AB
:100AA00000F0F0FA0028BED1019B002B5CD1082099
:100AB0000BB0BDE8F08F0D2148462F6AFFF7DEFE30
:100AC0008742E9D1AB6A9C42E6D12046FFF7EAFCB7
:100AD0000F2102464846FFF7F7FE48462A46002106
:100AE000FFF7F2FE07209FE70D2148462F6AFFF728
:100AF000C5FE874258D02368002B87DA043485E787
:100B0000029B3BB305F15803271DCDF810B0DDF86B
:100B10000C80A346DDF808A01C46059602E0B2450D
:100B2000B04616D038460694FFF788FD06AB01465E
:100B30000022284604F01CF908F1010604370028B9
:100B4000EDD0029B5C464345DDF810B0059ED2D146
:100B500000E05C4648460D21FFF790FE069B2862A8
:100B6000AC626B6206205FE70F214846FFF786FE06
:100B70000E2102464846FFF7A7FE4846294A0F21A4
:100B8000FFF7A2FE07204FE707460D214846FFF773
:100B900075FE022F28621DD12B46069A43F82C2F92
:100BA0006B62AC6206203FE7AB6A9C42A3D1042291
:100BB00000270299A318A962EF622A636B63236876
:100BC000BB421DDB0123019320E748460D21FFF7BF
:100BD00055FE2862069B6B62E3E72046FFF762FC46
:100BE00004340646AC63284604F01EF900283FF49E
:100BF0001AAF484632460F21FFF766FE072013E77B
:100C00000846013004EB8000FFF74CFC0F21024640
:100C10004846FFF759FE48462A463946FFF754FE34
:100C2000072001E7854F0108002395E6012393E69D
:100C3000022391E6F0B50446C5B004290DD8DFE8DB
:100C400001F055030C310F00012B4FEA124695B20B
:100C500064D17219102A40F29D80022045B0F0BD87
:100C6000002BFAD1102AF8D82368D80600F1C880E2
:100C700022AE30460192012500F074F90023A06BEA
:100C8000019A05FA03F1114203D00168043046F8D5
:100C900023100133042BF4D1A063304600F058F93F
:100CA0000020DBE7032BD8D1150C97B2EB19102BE2
:100CB000D3D823681E0700F1B78022AE304600F07B
:100CC00025F9ED00A06B5FB1043D0346711900EBFF
:100CD000C70053F8042B834241F8042FF9D118467A
:100CE000A063304600F0F0F80020B7E7002BB4D145
:100CF0000127A56B96B2201D07FA03F1314203F1DB
:100D0000010302D0296804350160102B00F10400B2
:100D1000F2D112F400503BD1A5639FE7052B9CD183
:100D20007719202F99D80F2E66D92F46002D3AD14A
:100D30002A460027002AA06B72DD00EBC2020146A2
:100D400044A800EBC6008C3851F8045B914240F88F
:100D5000045FF9D1084697B1102E324638BF1022F1
:100D600044A901EBC202A2F5C4727900043A00EB77
:100D7000810150F8045B884242F8045FF9D1012BED
:100D800048D00F2EA16333D917B102A800F094F810
:100D9000002063E70F2E3FF660AF00272268D107DF
:100DA00017D4002F60D02268510745D4012B4DD0B5
:100DB0000F2E06D822A8019300F07AF8019B002F8D
:100DC000B6D002A8019300F07BF8019BC6F1100297
:100DD000B0E722F00101052B2160019320463BD0B2
:100DE00022F0030240F8482B00F05AF8019BD8E7A4
:100DF00022A800F059F8C7E7102FCED9103FCDE751
:100E000023F01003236004F5E870019200F0AAF8C3
:100E1000019A2DE70431A16322A800F03DF8B7E75D
:100E2000002F99D10146AAE723F00803236004F5B7
:100E3000A87000F06BF840E7204622F0040240F86A
:100E4000D02B019300F03CF8019BAFE722A801935F
:100E500000F026F8019BB9E741F0020140F8481B79
:100E600000F026F8019B9CE7012B03D00F2E3FF6E4
:100E70005FAF9FE722A8019300F012F8019B57E7AC
:100E800000F1340191E838009C46A6464CF8045D18
:100E900090E8FF0FE54600BD90EC210B704700BFC6
:100EA00080EC210B704700BF90EC200B704700BF17
:100EB00080EC200B704700BFD0EC200B704700BFC8
:100EC000C0EC200B704700BFF0EC0201F0EC021107
:100ED000F0EC0221F0EC0231F0EC0241F0EC0251B6
:100EE000F0EC0261F0EC0271F0EC0281F0EC0291A6
:100EF000F0EC02A1F0EC02B1F0EC02C1F0EC02D196
:100F0000F0EC02E1F0EC02F1704700BFE0EC02010E
:100F1000E0EC0211E0EC0221E0EC0231E0EC0241F5
:100F2000E0EC0251E0EC0261E0EC0271E0EC0281E5
:100F3000E0EC0291E0EC02A1E0EC02B1E0EC02C1D5
:100F4000E0EC02D1E0EC02E1E0EC02F1704700BF1E
:100F5000B0FC0181B0FC0191B0FC01A1B0FC01B179
:100F6000704700BFA0FC0181A0FC0191A0FC01A181
:100F7000A0FC01B1704700BFEC4600B52DE9005060
:100F80002DE9FF1F4FF000032DE90C0001A9FFF729
:100F9000EDFBDDF840E012B0704700BFEC4600B555
:100FA0002DE900502DE9FF1F4FF000032DE90C0043
:100FB00001A9FFF715FCDDF840E012B0704700BF53
:100FC000EC4600B52DE900502DE9FF1F4FF000035E
:100FD0002DE90C0001A9FFF725FCDDF840E012B077
:100FE000704700BFEC4600B52DE900502DE9FF1F0A
:100FF0004FF000032DE90C0001ABFFF7E7FBDDF834
:1010000040E012B0704700BFEC4600B52DE900503B
:101010002DE9FF1F4FF000032DE90C0001AAFFF797
:1010200061FCDDF840E012B0704700BF027A1AB9E7
:10103000437A43B9B02070470368013A02721A023A
:101040000260180E704703214268013B10B44372DE
:101050001368141D01721A024460026010BC180E5D
:10106000704700BF002300B585B003AA009219465F
:101070000C22FFF7E9FB039805B05DF804FB00BF05
:10108000F0E700BF2DE9F04306460F464FF0000899
:1010900085B03846FFF7CAFFB028044623D00506BE
:1010A00027D400230DF10C09194685000D22CDF837
:1010B00000903046FFF7C8FBEDB2039B600605F1D8
:1010C00004054CBF5D1BED1800230D221946CDF819
:1010D000009030460395FFF7DDFB3846FFF7A6FF8B
:1010E000B0280446DBD1B8F1000F00F09480002056
:1010F0001CE000F0F003802B5CD0902B19D0A02BCB
:101100002CD0B02B3ED0C02B6BD000F0F803D02BEE
:101110000BD100F00702013242F400220523012125
:101120003046FFF787FD0028B3D0092005B0BDE8A1
:10113000F08300F00D030D2BF7D0002303AD00F07A
:101140000F02194600953046FFF77EFB00230095FD
:1011500019460D223046FFF79DFB9AE7C3434FF433
:101160007F6203F007031A410023010702F47F6244
:1011700048BF42F4804219463046FFF75BFD002825
:10118000D3D186E7B12857D0B22868D0B32800F071
:10119000958000F0FC03B42BC7D0012300F00702B8
:1011A0001A4442F4002219463046FFF743FD002856
:1011B000BBD16EE73846FFF739FF24020443B4F58C
:1011C000004FB2D000232401A2B219463046FFF7E7
:1011D00031FD0028A9D114F4004F18BF4FF00108C9
:1011E00057E7C6287DD0C72800F0868000F0F803B6
:1011F000C02B00F09480C82800F09F80C92894D1AB
:101200003846FFF713FF020300F00F0002F47022CC
:101210000130024382E703AC43460E22414600946C
:101220003046FFF711FB0094304643460F224146FB
:10123000FFF730FB404679E73846FFF7F7FE002816
:101240003FF473AF10F0F0037FF46FAF024619461E
:101250003046FFF7EFFC00287FF467AF19E7002363
:101260000DF10C090D221946CDF800903046FFF71C
:10127000EBFA3846FFF7DAFE02064FF002040CD50F
:10128000039B00F07F00A040034438460393FFF720
:10129000CDFE030604F10704F2D40023039900F005
:1012A0007F02A24001F501718C18CDF8009019461B
:1012B0000D2230460394FFF7EDFAEAE63846FFF7D1
:1012C000B5FE0123010300F00F0001F47021C218E4
:1012D0000A4330461946FFF7ADFC00287FF425AFDE
:1012E000D7E63846FFF7A2FE010300F00F00032304
:1012F00001F47021421CEBE73846FFF797FE002807
:101300003FF413AF10F0F0037FF40FAF0246042157
:101310003046FFF78FFC00287FF407AFB9E60323C0
:1013200000F00F02013242F4202219463046FFF746
:1013300081FC00287FF4F9AEABE63846FFF776FE75
:1013400000F0F00200F00F031032013343EA0232E2
:10135000E4E600BF30B503240D46C36C85B05A687F
:101360008DF80C40DC791202083301A9284601925D
:101370008DF80D400293FFF785FE05B030BD00BF2C
:1013800008B5FFF77DFE806C08BD00BF08B5FFF70C
:1013900077FEC06CC37900EB8300083008BD00BF46
:1013A00008B503F0F7FE00BF08B5FFF7F9FF00BF6F
:1013B000704700BFD0400B1C1141203A03D49C461B
:1013C000134118436346524293401843704700BF8D
:1013D0004A0011D212F5001211D20DD56FF47873B4
:1013E000B3EB62520ED44FEAC12343F0004343EA09
:1013F000505323FA02F070474FF00000704750EA54
:10140000013002D14FF0FF3070474FF000007047BD
:101410004FEA4102B2F1E04324BFB3F5001CDCF116
:10142000FE5C0DD901F0004C4FEAC0024CEA50704E
:10143000B2F1004F40EB830008BF20F0010070477D
:1014400011F0804F21D113F13872BCBF01F0004080
:10145000704741F480114FEA5252C2F11802C2F1B2
:10146000200C10FA0CF320FA02F018BF40F0010033
:101470004FEAC1234FEAD32303FA0CFC40EA0C00E5
:1014800023FA02F34FEA4303CCE77FEA625307D122
:1014900050EA01331EBF4FF0FE4040F44000704759
:1014A00001F0004040F0FE4040F40000704700BFF3
:1014B00080F0004002E000BF81F0004142001FBF09
:1014C0005FEA410392EA030F7FEA226C7FEA236C12
:1014D0006AD04FEA1262D2EB1363C1BFD218414007
:1014E00048404140B8BF5B42192B88BF704710F09D
:1014F000004F40F4000020F07F4018BF404211F040
:10150000004F41F4000121F07F4118BF494292EAA7
:10151000030F3FD0A2F1010241FA03FC10EB0C00D3
:10152000C3F1200301FA03F100F0004302D5494260
:1015300060EB4000B0F5000F13D3B0F1807F06D30D
:1015400040084FEA310102F10102FE2A51D2B1F105
:10155000004F40EBC25008BF20F0010040EA0300FA
:101560007047490040EB000010F4000FA2F10102A7
:10157000EDD1B0FA80FCACF1080CB2EB0C0200FA31
:101580000CF0AABF00EBC25052421843BCBFD0407F
:101590001843704792F0000F81F4000106BF80F4F9
:1015A00000000132013BB5E74FEA41037FEA226CBC
:1015B00018BF7FEA236C21D092EA030F04D092F087
:1015C000000F08BF0846704790EA010F1CBF0020BB
:1015D000704712F07F4F04D1400028BF40F0004018
:1015E000704712F100723CBF00F50000704700F038
:1015F000004343F0FE4040F4000070477FEA22625F
:1016000016BF08467FEA23630146420206BF5FEA2F
:10161000412390EA010F40F4800070474FF000032F
:1016200004E000BF10F0004348BF40425FEA000CF6
:1016300008BF704743F0964301464FF000001CE09E
:1016400050EA010208BF70474FF000030AE000BFF4
:1016500050EA010208BF704711F0004302D5404232
:1016600061EB41015FEA010C02BF844601460020A4
:1016700043F0B64308BFA3F18053A3F50003BCFABF
:101680008CF2083AA3EBC25310DB01FA02FC63446C
:1016900000FA02FCC2F12002BCF1004F20FA02F273
:1016A00043EB020008BF20F00100704702F1200266
:1016B00001FA02FCC2F1200250EA4C0021FA02F2C7
:1016C00043EB020008BF20EADC7070474FF0FF0CCC
:1016D0001CEAD0521EBF1CEAD15392EA0C0F93EAC7
:1016E0000C0F6FD01A4480EA010C400218BF5FEA69
:1016F00041211ED04FF0006343EA501043EA5111DC
:10170000A0FB01310CF00040B1F5000F3EBF4900D5
:1017100041EAD3715B0040EA010062F17F02FD2AD9
:101720001DD8B3F1004F40EBC25008BF20F00100BC
:10173000704790F0000F0CF0004C08BF49024CEAD3
:10174000502040EA51207F3AC2BFD2F1FF0340EA65
:10175000C250704740F400004FF00003013A5DDCD6
:1017600012F1190FDCBF00F000407047C2F1000217
:10177000410021FA02F1C2F1200200FA02FC5FEA04
:10178000310040F1000053EA4C0308BF20EADC704E
:10179000704792F0000F00F0004C02BF400010F4C0
:1017A000000F013AF9D040EA0C0093F0000F01F06D
:1017B000004C02BF490011F4000F013BF9D041EA8F
:1017C0000C018FE70CEAD15392EA0C0F18BF93EA91
:1017D0000C0F0AD030F0004C18BF31F0004CD8D1BB
:1017E00080EA010000F00040704790F0000F17BF42
:1017F00090F0004F084691F0000F91F0004F14D088
:1018000092EA0C0F01D142020FD193EA0C0F03D1DF
:101810004B0218BF084608D180EA010000F00040E2
:1018200040F0FE4040F40000704740F0FE4040F4BD
:10183000400070474FF0FF0C1CEAD0521EBF1CEA5C
:10184000D15392EA0C0F93EA0C0F69D0A2EB03027A
:1018500080EA010C49024FEA402037D04FF0805314
:1018600043EA111143EA10130CF000408B4238BFD9
:101870005B0042F17D024FF4000C8B4224BF5B1AE7
:1018800040EA0C00B3EB510F24BFA3EB510340EA35
:101890005C00B3EB910F24BFA3EB910340EA9C00E3
:1018A000B3EBD10F24BFA3EBD10340EADC001B0153
:1018B00018BF5FEA1C1CE0D1FD2A3FF650AF8B42F7
:1018C00040EBC25008BF20F0010070470CF0004C04
:1018D0004CEA50207F32C2BFD2F1FF0340EAC2502F
:1018E000704740F400004FF00003013A37E792F0F0
:1018F000000F00F0004C02BF400010F4000F013A4E
:10190000F9D040EA0C0093F0000F01F0004C02BF48
:10191000490011F4000F013BF9D041EA0C0195E7B1
:101920000CEAD15392EA0C0F08D142027FF47DAF4A
:1019300093EA0C0F7FF470AF084676E793EA0C0F3A
:1019400004D14B023FF44CAF08466EE730F0004C38
:1019500018BF31F0004CCAD130F000427FF45CAFC8
:1019600031F000437FF43CAF5FE700BF4FF0FF3C36
:1019700006E000BF4FF0010C02E000BF4FF0010C89
:101980004DF804CD4FEA40024FEA41037FEA226C52
:1019900018BF7FEA236C11D001B052EA530C18BF74
:1019A00090EA010F58BFB2EB030088BFC81738BFD9
:1019B0006FEAE17018BF40F0010070477FEA226CC7
:1019C00002D15FEA402C05D17FEA236CE4D15FEAC3
:1019D000412CE1D05DF8040B704700BF84460846F7
:1019E0006146FFE70FB5FFF7C9FF002848BF10F1B8
:1019F000000F0FBD4DF808EDFFF7F4FF0CBF0120FD
:101A000000205DF808FB00BF4DF808EDFFF7EAFF86
:101A100034BF012000205DF808FB00BF4DF808ED41
:101A2000FFF7E0FF94BF012000205DF808FB00BF36
:101A30004DF808EDFFF7D2FF94BF012000205DF8BC
:101A400008FB00BF4DF808EDFFF7C8FF34BF0120C9
:101A500000205DF808FB00BF4FEA40024FEA410357
:101A60007FEA226C02D15FEA402C08D17FEA236C26
:101A700002D15FEA412C02D14FF0000070474FF0D5
:101A8000010070474FEA4002B2F1FE4F0FD34FF012
:101A90009E03B3EB12620DD94FEA002343F00043DB
:101AA00010F0004F23FA02F018BF404270474FF089
:101AB0000000704712F1610F01D1420205D110F010
:101AC000004008BF6FF0004070474FF000007047C3
:101AD00042000ED2B2F1FE4F0BD34FF09E03B3EB98
:101AE000126209D44FEA002343F0004323FA02F0C4
:101AF00070474FF00000704712F1610F01D14202B0
:101B000002D14FF0FF3070474FF00000704700BF28
:101B10007BB972B90029BEBF00204FF0004106E03A
:101B200008BF00281CBF6FF000414FF0FF30FFF7E7
:101B30003FBCADF1080C6DE904CE002909DB002B98
:101B40001ADBFEF741FBDDF804E0DDE9022304B017
:101B50007047404261EB4101002B1BDBFEF734FB79
:101B6000DDF804E0DDE9022304B0404261EB41010D
:101B7000524263EB43037047524263EB4303FEF769
:101B800023FBDDF804E0DDE9022304B0404261EB11
:101B900041017047524263EB4303FEF715FBDDF84A
:101BA00004E0DDE9022304B0524263EB43037047D3
:101BB00010B500210446FFF727FF20B92046BDE8F5
:101BC000104000F009B804F1004000F005F8404270
:101BD00061EB410110BD00BFD0B5FDF7B1FF0022A0
:101BE0000E4B06460F46FDF7FFFFFFF7F1FB0446DD
:101BF000FDF784FF00220A4BFDF7F6FF02460B4675
